:1000000054464953000100004CD30200B3B5926638
:100010001779010519080709413931531779010189
:1000200019080709413931531779000119080709DF
:1000300041393153030000000000000000000000BF
:100040005446435300200000389A0200000000008C
:10005000008001100121000025210000010A02009A
:10006000292100002B2100002D2100003D2100004E
:100070003D2100003D2100003D2100002F21000016
:10008000312100003D210000332100003D700000BF
:1000900007740000372100003D210000296A00108C
:1000A00037210000815100008551000037730000A6
:1000B000372100007B6C00006D6300008951000057
:1000C000356A00003721000037210000895E0000FA
:1000D0000000000000000000000000000000000020
:1000E0000000000000000000000000000000000010
:1000F0000000000000000000000000000000000000
:1001000000000000000000000000000000000000EF
:1001100000000000000000000000000000000000DF
:1001200000000000000000000000000000000000CF
:1001300000000000000000000000000000000000BF
:1001400000000000000000000000000000000000AF
:1001500000F003F800F020F8FEE70D480168890878
:100160008900002001C101C101C101C17047000027
:1001700048700010FEE7FEE7FEE7FEE7FEE7FEE759
:10018000FEE7FEE7FEE703480047FEE7FEE7000064
:10019000202100003D21000000F002F800F068F886
:1001A0000AA090E8000C82448344AAF10107DA45D2
:1001B00001D100F05DF8AFF2090EBAE80F0013F0BC
:1001C000010F18BFFB1A43F001031847482602002D
:1001D000982602000A444FF0000C10F8013B13F07F
:1001E000070408BF10F8014B1D1108BF10F8015B90
:1001F000641E05D010F8016B641E01F8016BF9D183
:1002000013F0080F1EBF10F8014BAD1C0C1B09D1D9
:100210006D1E58BF01F801CBFAD505E014F8016B4B
:1002200001F8016B6D1EF9D59142D6D370470000DD
:10023000103A24BF78C878C1FAD8520724BF30C812
:1002400030C144BF04680C607047000000230024E4
:1002500000250026103A28BF78C1FBD8520728BFD6
:1002600030C148BF0B6070471FB51FBD10B510BD32
:10027000DFF80CD0FFF7F8FF07F00AFA1EF0DAFB00
:100280000080011003B4FFF7F1FF03BC1EF0DAFB9E
:1002900008B500200346024600900121022000F02C
:1002A00068FB08BD38B5FF4D0024FF48AC81EC81E8
:1002B0002C8240698047E861FF202872FB480023B8
:1002C0001A46046044608460C4600461012068725E
:1002D0002C70AC7001460220009400F04AFB012013
:1002E00038BD38B5EF4D02282C7A22460DD00528AE
:1002F00010D0A24208BF38BD002003460246214666
:10030000009000F036FB2C7238BD022914BF012486
:100310000224EEE7022914BF04240824E9E708B503
:10032000009313460A460146012000F022FB08BD57
:1003300008B50346009103220221012000F019FBB9
:1003400008BD38B500240DF0EDFE002818BF0124CB
:1003500012F04CFB002818BF0224D2480178A142B9
:1003600008BF38BD047000200346022100902246D9
:10037000084600F0FEFA38BD38B5CA4D0446687824
:10038000A04208BF38BD07F09DF96C70002C0CBF6F
:10039000052106210020034602460090022000F0BD
:1003A000E8FA38BD08B500210B4602460091072146
:1003B000022000F0DEFA08BD08B500210B46024617
:1003C00000910821022000F0D4FA08BD08B50021F0
:1003D0000091002814BF01220022002303210220E3
:1003E00000F0C7FA08BD08B5002003460246009099
:1003F0000421022000F0BDFA08BDAA4B0028DA78DB
:1004000014BF01210021D9708A4208BF7047021C25
:1004100018BF012208B50020034600900A210220DF
:1004200000F0A7FA08BD9F4B00289A7814BF01215D
:10043000002199708A4208BF7047021C18BF012230
:1004400008B50020034600900921022000F091FA2F
:1004500008BD94488078002818BF0120704701200B
:100460009049087170478F48007970478D49002086
:10047000087170472DE9F04104460127002503F07B
:100480000700884E8846012804BF0020308248D0EB
:10049000022846D1308A844904280BD2002818BF8C
:1004A000B06902D148688047B06110F8011B217023
:1004B000B0612FE0062809D288688047318A80B26F
:1004C000C1F10501C900C840207023E0082808D206
:1004D00008698047318AC1F10701C900C84020700E
:1004E00018E00C2808D248698047318AC1F10B0115
:1004F000C900C84020700DE00E2808D288698047E6
:10050000318AC1F10D01C900C840207002E0FF200E
:1005100020700027308A401C80B230820E2828BF0D
:10052000012588F800503846BDE8F08130B403F06A
:1005300007000024DFF86CC1012804BFACF80C40B0
:10054000ACF810401BD013F0070F18D1554BBCF876
:1005500010009B89022805D2120242EA1322ACF84D
:100560000C2009E003449D1EB5F5806F04DADCF829
:100570001C502B4403F8022C401CACF810000C70EB
:1005800030BC00207047F0B40746002003F0070499
:10059000444D0646012C04BF2E826E6125D0DFF843
:1005A00004C1022CBCF80EC003D013F0070F0DD00D
:1005B0001BE02A8A0CEB0203B3F5806F15D2E869C1
:1005C000C05C3870501C288201200EE0120242EA02
:1005D0001C22EA816B69012B05D1B2F5806F24BF23
:1005E00040F2FF32EA815A1C6A610E70F0BC70471B
:1005F00038B503F0070000240D46012809D1294829
:1006000000231A460482848119460220009400F0D7
:10061000B0F92C70002038BD2DE9F04182B01746AA
:100620000C0005464FF0000800F0028126782049B2
:10063000012E18BF022E05D0032E5AD0002E00F036
:10064000F780BDE06078421E05EB001000F8102C2A
:10065000607805EB001000F80F6C08686288438D25
:10066000C08C5A4392FBF0F0627805EB021222F83C
:100670000E0C0868A288018D808C514391FBF0F02C
:10068000617805EB011121F80C0C6178A07905EB7C
:10069000011121F80A0C6178207A05EB011121F88B
:1006A000080C07E0008000108846020094850010C6
:1006B000008500106178607A05EB011121F8060CC5
:1006C0006178A07B05EB011121F8040CE079052885
:1006D000607805EB001010F8021C0CBF41F001011E
:1006E00021F0010100F8021C002E69D102B0BDE822
:1006F000F0816078421E05EB001000F8102C627843
:10070000032005EB021202F80F0C08686288438D83
:10071000C08C5A4392FBF0F0627805EB021222F88B
:100720000E0C0868A288018D808C514391FBF0F07B
:10073000617805EB011121F80C0C06F0C3FF0528C8
:1007400021D107B36178B87905EB011121F80A0CC2
:100750006178387A05EB011121F8080C6178787A14
:1007600005EB011121F8060CF8790528607805EBF6
:10077000001010F8021C0CBF41F0010121F0010132
:1007800000F8021C17E0607805EB001020F80A8CD6
:10079000607805EB001020F8088C607805EB0010FD
:1007A00020F8068C607805EB001010F8021C21F090
:1007B000010100F8021C607805EB001020F8048CA1
:1007C000012E18BF032E06D00DF08CFA002804BFAE
:1007D00002B0BDE8F08106F075FF05281CBF02B02D
:1007E000BDE8F081012E04BFC0208DF8000005D0C7
:1007F000022E0CBFC220C1208DF8000060788DF859
:10080000010060880123000A8DF80200A0788DF8AD
:100810000300A0880622000A8DF8040020798DF8D4
:1008200005006946072011F02EF802B0BDE8F081FE
:1008300085F8008085F80180A5F80280A5F804807D
:10084000A5F80680A5F80880A5F80A80A5F80C8010
:10085000A87B20F00100A87302B0BDE8F0814A49EE
:10086000002048717047484840797047002818BFF9
:1008700001204549887170474348807970470028B6
:1008800018BF01204049C87170473F48C079704780
:100890003D49488170473C48408970473A490120AA
:1008A00048717047394B03EB80004254704700B5E4
:1008B00085B001788DF8001042788DF8012083789A
:1008C0008DF80230C3788DF8033003798DF8043049
:1008D00043798DF8053080798DF8060000208DF879
:1008E00007000290039001232748522904D046298B
:1008F00008BF012A05D008E08179002908BF83716B
:1009000003E0C179002908BFC37106F0FEFF01288A
:100910000CD11EF0ADF8012801BF9DF8000046285B
:100920009DF80100012804BF05B000BD68461EF017
:10093000A4F805B000BD70471349002818BF012076
:10094000487270471048407A7047012818BF7047B6
:100950000F48012904BF416841F4007105D0002906
:1009600006BF416821F40071704741607047094833
:10097000704708B5DDF808C0CDF800C0DFF818C032
:10098000DCF800C0E04708BD00800010948500102E
:10099000001000406C410200884602007047F64893
:1009A000D0F8500300F00100704770B5F24D04001C
:1009B0000AD002F030FB38B9D5F8500310F0010F1F
:1009C0001CBF0020A86005D10120A860002C08BF32
:1009D00000202DD0D5F8600310F0010F0BD1D5F811
:1009E000600340F00100C5F86003D5F8600320F013
:1009F0000100C5F86003E148016811F0010F07D15B
:100A0000016841F001010160016821F0010101600C
:100A100004F0D0FB00281CBFD5F8500310F0010FE4
:100A200005D004F0C1FB002818BF04F0CFFB012063
:100A3000286270BDD048006A002818BF01207047A6
:100A4000C00000F1804000F5A04041637047C00045
:100A500000F1804000F5A040006B00F4807070470A
:100A60001021C00000F1804000F5A04041637047B4
:100A700030B48209C24B00F00F0000EB400053F885
:100A800022404FF4847505EB8015D1F800C044F87E
:100A900005C053F822204FF4867303EB8010496899
:100AA000115030BC70478209B54850F82200D0F888
:100AB000402161F30D22C0F840217047B049800900
:100AC00051F82000D0F84001C0F305207047AA4932
:100AD000D1F8402160F31742C1F840217047A64881
:100AE000D0F84001C0F3074070474FF4A072C0F344
:100AF000011302EB8312DFF888C200F00F038009B4
:100B000003EB43035CF82000002900EB83108158BD
:100B100014BF41F0010121F0010181507047984A52
:100B2000810952F8212000F00F0101EB410102EB95
:100B30008111C0F301104FF4A07202EB801008582D
:100B400000F0010070478E4A810952F82110D1F857
:100B5000E01100F00F00012201F0070102FA00F09D
:100B6000084018BF012070474FF4A072C0F3011372
:100B700002EB8312DFF808C200F00F03800903EBD9
:100B800043035CF82000002900EB8310815814BF58
:100B900041F0020121F0020181507047784A810939
:100BA00052F8212000F00F0101EB410102EB81110D
:100BB000C0F301104FF4A07202EB80100858C0F38C
:100BC0004000704781096F4A01EB410102EBC1010E
:100BD00000F00F0201EBC201C0F3011051F8200038
:100BE0007047684982091CD00122B2EB901F18BFE0
:100BF000704765480068C0F3080088616348026870
:100C0000C2F308420A620068C0F308004862604804
:100C10000268C2F308428A620068C0F30800C86232
:100C200070475548D0F82421C2F308020A60D0F872
:100C3000E421C2F308428A60D0F8E421C2F308023A
:100C4000CA60D0F8A422C2F308420A61D0F8A40214
:100C5000C0F30800486170472DE9F00301228309C1
:100C600000F00F01C0F3011CC0F3011622EA0C0CC6
:100C700000290BBF02254D1E00224FEA0C124FF037
:100C8000080404EBCC043F4F03EB430C07EBCC0C04
:100C90000CEBC101DFF8E88051F826604FF4587C76
:100CA00058F823100CEBC50551F805C000F00F00F3
:100CB0001CF0010F00EB40004FF4927C0CEB801C09
:100CC00040F2FF1729D02C48D0F844034FF03209E6
:100CD0000005000D06FB09F60EBF0120B6FBF0F083
:100CE000401CFF2888BFFF204E594FF0FF0909FA2A
:100CF00004F9C0B226EA0906A0403043485158F82A
:100D0000230050F80C3007FA02F123EA01021143E4
:100D100040F80C10BDE8F003704751F80C0007FADA
:100D200002F39843C6F3080303FA02F2104341F8B2
:100D30000C00BDE8F003704710B50020FFF78CFFF2
:100D40000120FFF789FF1120FFF786FF0220FFF740
:100D500083FF1220FFF780FF4020FFF77DFF412037
:100D6000FFF77AFF5120FFF777FF4220FFF774FF6C
:100D7000BDE8104052206FE700500040605B00402B
:100D8000884102004886001024590040E459004080
:100D9000A45A00402DE9F04707464FEA9016FF4855
:100DA0000D0050F826404FF000002062C4F84001CA
:100DB000C4F80002C4F84002C4F8C002C4F800033A
:100DC00008BFBDE8F08728682060686860606168D7
:100DD0000120002908BF6060F1490860A868A06090
:100DE000E868E0602869A0616869E061E8696062BC
:100DF000286AE06221206063E063686A2064A86A70
:100E00006064E86AA064286BE064686B2066A86B85
:100E1000A066E86B6067286CA067686CE067A86CE8
:100E2000C4F88000E86CC4F88400286DC4F8880019
:100E3000686DC4F88C00A86DC4F89000E86DC4F823
:100E4000A400286EC4F8A800686EC4F8AC00A86EB0
:100E5000C4F8B000E86EC4F8B400286FC4F8B80055
:100E6000686FC4F8BC004FF0FF30C4F8E400A86F0E
:100E7000C4F8F000E86FC4F8F400D5F88000C4F8B6
:100E8000FC004FF4107205F1840104F580701DF030
:100E9000F9FDD5F8C40220F48030C4F84003D5F839
:100EA000C802C4F84C03D5F8CC02C4F85003D5F8F6
:100EB000D002C4F85403D5F8D402C4F85803D5F8C6
:100EC000D802C4F85C03002005EBC002D2F8DC3283
:100ED00004EBC001C1F86033D2F8E022C1F864230A
:100EE000401C0328F0DBD5F8F402C4F87803D5F8E9
:100EF000F802C4F87C03D5F8FC02C4F80004D5F865
:100F00000003C4F80404D5F80403C4F80804D5F8B1
:100F10000803C4F80C04D5F80C03C4F8100400222C
:100F2000002104EBC20805EBC20000EB8103D3F8FB
:100F3000109308EB810CCCF83094D3F83893CCF8AC
:100F40005894D3F86033CCF88034491C0229ECDB88
:100F500005EB8200D0F8883304EB8201C1F8A83495
:100F6000D0F89C33C1F8BC34D0F8B003C1F8D00439
:100F7000521C052AD4DB002E14BF8A488A48006818
:100F800030F0FF0105D1D4F8901060F30301C4F8EC
:100F90009010D4F8500320F00100C4F85003D4F8A6
:100FA000600320F00100C4F86003D4F8680320F067
:100FB0000100C4F86803D4F8700320F00100C4F8FD
:100FC00070033846BDE8F0470BE678480078704774
:100FD00076484078704775498870704773488078C4
:100FE00070477349D1F8542360F30902C1F85423C0
:100FF00070476F48D0F85403C0F3090070476B493D
:101000004860704769484068704768498860704721
:101010006648806870476549C86070472DE9F05F91
:1010200004460027384614F4803F18BF012014F40A
:10103000003F18BF40F0040014F4802F18BF40F0A8
:10104000020014F4002F18BF40F0100014F4001F29
:1010500018BF40F0400014F4800F18BF40F00800A3
:1010600014F4000F18BF40F02000DFF84081DFF8D3
:10107000409198F8021010EA0105D9F8400320F4D5
:101080008030C9F8400336D0D8F80C60D9F848034E
:10109000002740F00100C9F84803D9F8480320F0C0
:1010A0000100C9F84803D9F8400340F48030C9F87A
:1010B00040034FF0630ADFF8FCB016E004F0C1F91A
:1010C0005046D9F8481311F0010F0AD0D9F844035B
:1010D0000005000D1CBFBBFBF0F0C8F8080001279D
:1010E00003E0011EA0F10100EBDC301EA6F10106B9
:1010F00001DD002FE2D0D9F8500320F00100C9F83B
:101100005003D9F8600320F00100C9F86003D9F852
:10111000680320F00100C9F86803D9F8700320F0D3
:101120000100C9F87003244A106820F00100106023
:101130002248016821F00101016021490B6823F078
:1011400001030B60F7B315F0010F05D0D9F8503348
:1011500043F00103C9F8503315F0040F05D0D9F856
:10116000703343F00103C9F8703315F0020F05D056
:10117000D9F8603343F00103C9F8603315F0100F5C
:1011800005D0D9F8683343F00103C9F8683315F086
:10119000400F19D00B6843F0010314E088410200AE
:1011A00004580040F0FE0400E0FE0400208000101F
:1011B0000050004080F0FA02605B0040685B004035
:1011C000705B00401AE00B6015F0080F03D0116847
:1011D00041F00101116015F0200F03D0016841F0CA
:1011E0000101016088F80150012088F80000D9F859
:1011F000400340F48030C9F8400321E0002088F823
:101200000100ADB1022088F80000D9F8400340F495
:101210008030C9F84003D9F8480340F00100C9F80C
:101220004803D9F8480320F00100C9F8480307E053
:10123000D9F8401321F48031C9F8401388F8000030
:10124000D9F8400114F0010F20F00D0018BF40F054
:10125000010014F0040F18BF40F0040014F0020F56
:1012600018BF40F00800C9F84001D9F8000214F096
:10127000100F14BF40F0010020F00100C9F8000277
:10128000D9F8400214F0200F14BF40F0010020F004
:101290000100C9F84002D9F8C00214F0400F14BF91
:1012A00040F0010020F00100C9F8C002D9F80003A5
:1012B00014F0800F14BF40F0010020F00100C9F8C5
:1012C0000003FF4814F4805F016814BF41F001017E
:1012D00021F001010160FB4814F4005F016814BFB4
:1012E00041F0010121F001010160F74814F4804F41
:1012F000016814BF41F0010121F001010160F348D0
:1013000014F4004F016814BF41F0010121F0010104
:101310000160EF49086814F4807F20F00D0018BFC9
:1013200040F0010014F4806F18BF40F0040014F482
:10133000007F18BF40F0080008600020FFF78CFC19
:101340000120FFF789FC1120FFF786FC0220FFF740
:1013500083FC1220FFF780FC4020FFF77DFC41203A
:10136000FFF77AFC5120FFF777FC4220FFF774FC6F
:10137000BDE8F05F52206FE42DE9F04F840900F0E2
:101380000F0343EA8411D34D4FEA911CC1F30118B6
:1013900055F82C6003EB430C06EB8C174FF4A0764A
:1013A00006EB8818024657F80870002017F0010F66
:1013B00010D141F010018F09C1F3011155F82770C8
:1013C00006EB811107EB8C17795811F0010F08BF5C
:1013D000BDE8F08F55F82410CF6907F0080801EB3D
:1013E0008C17D7F80011DFF8F0A204EB440C0AEBDD
:1013F000CC0C1FFA81F902F00F05002103EB430624
:101400000CEBC505C2F3011A43EA011242EA841249
:10141000DFF8C0C2C2F3811B5CF82BC0C2F3011B12
:101420004FF4A0720CEB861C02EB8B125CF80220CE
:1014300012F0010F1AD007EB811C55F82A20DCF8B6
:1014400044B1B8F1000FCBF3080B0EBF4FF0000C06
:10145000DCF844C1CCF3023C02EBC20E0EEB0212EC
:1014600000EB42000BFA0CF202FB0900491C0229B6
:10147000CAD3BDE8F08F2DE9F0418509AA0195484E
:101480009309002450F82300D0F8401111F0010F07
:1014900034D0914E03EB430306EBC30302F00F0677
:1014A00003EBC603C2F3011211F0040F53F822201C
:1014B000D0F8003101F0080C9EB2D0F84431C3F3EB
:1014C000080318BFC1F30744C769C1F3052117F02A
:1014D000080F1ABFD0F84401C0F302300020BCF15D
:1014E000000F18BF491C03FA00F001FB004002EB9B
:1014F000C201704301EB021100EB4104012040EAFC
:101500008510FFF739FF0646022040EA8510FFF7F5
:1015100033FFA1190844BDE8F08110B50020FFF7A2
:10152000AAFF4FF47A7148434CF25031B0FBF1F00E
:1015300010BD6A484068C0F30C00704770B504469F
:101540000020FFF798FF05464020FFF794FF35B3D2
:10155000624BB0B141F288310844A84211D9421B14
:10156000186800F01F0104FB01F000EBC00C0CEB4D
:101570000010B2EB400F04D932204843B2FBF0F028
:10158000441CB4F5005F28BF41F6FF7402D2002C62
:1015900008BF0124586864F30C00586070BDB4F5AE
:1015A000005F28BF41F6FF7402D2002C08BF01245F
:1015B0004B48016864F30C01016070BD2DE9F041F6
:1015C000464F0646386810F01F0508BF0125002069
:1015D000FFF751FFDFF80C810446002E18BF002CE6
:1015E0003FD0414900204A68002A08BF0122330940
:1015F000B3FBF2F1D7F850C31CF0010F1BD0B3EBD3
:10160000420F1DD33949B1FBF2F3B6FBF2F10A09DF
:10161000B3FBF4F1102928BF0F218A4298BF11466D
:1016200039B1012984BF01FB1430B0FBF1F007D9B7
:1016300008E0012109E0B8FBF6F2A24288BF101BC6
:101640000029F6D0102988BF0F21D7F85C2361F359
:101650000302C7F85C2332216943B0FBF1F0FFF7C6
:101660006DFF7868C0F30C00684300EBC00101EB2C
:10167000001004EB4000B8FBF0F0BDE8F08170B55D
:10168000164D0024D5F8500310F0010F08D016486D
:10169000D5F85C13406801F00F01484304012DE0C8
:1016A0000020FFF7E8FE02462868696800F01F0086
:1016B000C1F30C01414301EBC10000EB011017E045
:1016C000005A0040405A0040C05A0040005B0040B1
:1016D00040590040884102004886001000500040F8
:1016E000045800400008AF2F2080001080F0FA025C
:1016F00012EB40001CBFFE49B1FBF0F4204670BD68
:10170000002818BF0120FB49D1F85C2360F30302D5
:10171000C1F85C237047F748D0F85C0300F00F0075
:1017200070478109F44A00F00F0000EB400052F8C6
:1017300021104FF4807202EB80100858EF4980B2FC
:10174000B1FBF0F0401C400870472DE9F041EA4B36
:101750008209DFF8A8C353F8223000F00F0731B137
:10176000BCFBF1F1491C4A08B2F5004F01D347F622
:10177000FF72BCFBF2F1491C4D08D3F880104FEA10
:10178000520C01F00704D3F88010DB4B4FEA90189D
:10179000C1F3031600F00F0153F8283001EB4101AB
:1017A00003EB81112FB3D1F80431F61C74439BB2C3
:1017B000A2EB4404D1F8006124F0010462F30F06A7
:1017C000C1F80061D1F800216CF31F42C1F800217B
:1017D000D1F8042163F30F02C1F80421D1F81821D4
:1017E00064F30F02C1F8182101F090F82846BDE813
:1017F000F081F61CACF10E037443A3EB4404D9E76B
:101800008109BD4A00F00F0000EB400052F82110A2
:101810004FF4807202EB80100858000C7047830967
:1018200010F00F02B44850F8230002EB420300EB23
:101830008313D3F800C161F31F4CC3F800C118BF74
:101840007047D0F8802002F00703D0F88020C2F360
:101850000312D21C5A430E39A1EB4202D0F80431D4
:1018600022F0010261F30F03C0F80431D0F818111F
:1018700062F30F01C0F8181170479F4A810952F8AE
:10188000212000F00F0101EB410102EB8111C0F3B7
:1018900001104FF4A27202EB80100858C0F3080048
:1018A0007047F0B4944B840900F00F0C53F82430C7
:1018B0000CEB4C0503EB8516C0F30112D6F81C5156
:1018C00006EB82164D1BD6F8447161F30807C6F883
:1018D00044714CEA021141EA841101F00F02C1F394
:1018E000011101EB4201864A03F5C07352F8211041
:1018F0004A08C90753F822C0C90E40F2FF148C40B1
:101900002CEA040CAD1EC5F3080404FA01F14CEAFC
:10191000010143F82210F0BC00F0F8BF830900F089
:101920000F01C0F30112744850F82300C36901EBA2
:10193000410100EB811013F0100FD0F8281100EBDB
:101940008210C9B2D0F84401C0F3080008BF0021DA
:10195000401A0004000C08BF0120704703091B0255
:1019600003EB810101F1405101F500310007C00E88
:101970000B6802FA00F0184308607047020912026F
:1019800002EB810101F1405101F5003100070968C6
:10199000C00E21FA00F000F00300704770B4DFF8C9
:1019A00058C1820900F00F035CF8225003EB430397
:1019B000C0F301104FF4A87605EB831506EB8016F3
:1019C0000C68AC515CF82220496802EB83124FF49A
:1019D000AA7303EB8010115070BC704730B4DFF86D
:1019E00018C1820900F00F035CF8224003EB4303A7
:1019F000C0F301104FF4A87504EB831405EB8015B8
:101A000064590C605CF8222002EB83124FF4AA7335
:101A100003EB80101058486030BC7047364910B452
:101A2000820983B051F8222000F00F0101EB41013F
:101A300002EB8111C0F301104FF4A87202EB801287
:101A40008A5800924FF4AA7202EB80100858019055
:101A5000002001466A4601234FEA511C01F01F0491
:101A600052F82CC003FA04F41CEA040F18BF401CFF
:101A7000491C2629F0D303B010BC704730B40022B3
:101A800010F00F0F06D000F00F02C0F3011303EBAC
:101A90004202521E184B80094FF4866553F82040CD
:101AA00005EBC205D1F800C044F805C053F820008A
:101AB00040F2344303EBC2024968815030BC7047A6
:101AC00010B4002210F00F0F06D000F00F02C0F388
:101AD000011303EB4202521E074B80094FF4866448
:101AE00053F820C004EBC2045CF804C00AE0000014
:101AF0000008AF2F0050004088410200A08601007E
:101B000090410200C1F800C053F8200040F2344375
:101B100003EBC2028058486010BC7047FE48C068A2
:101B200070470022FD49830951F82310CB6913F057
:101B3000080F0ED000F00F0202EB420201EB8211FF
:101B4000C0F301104FF4A27202EB80100858C0F3EA
:101B5000023210467047DFF8C4C310B482095CF843
:101B60002230DC6944F00804DC615CF8223000F0CB
:101B70000F0202EB420203EB8212C0F301134FF497
:101B8000A27000EB8310135861F30E33135010BC96
:101B900070470022E149830951F82310CB6913F003
:101BA000080F0ED000F00F0202EB420201EB82118F
:101BB000C0F301104FF4A47202EB80100858C0F378
:101BC000024210467047D54A830952F8233000F08C
:101BD0000F0202EB420203EB8212C0F301134FF437
:101BE000A47000EB8310135861F312431350704735
:101BF000042988BF70472DE9F0030027DFF81C8314
:101C0000840958F82430DA69C0F3011C12F0080F77
:101C10004FF4A27202EB8C1C00F00F0202EB4202A6
:101C200005D003EB821555F80C50C5F30237DD697A
:101C3000002615F0080F4FF4A475C0F3011005EB52
:101C4000801504D003EB82104059C0F30246C91B33
:101C50007018042803DD081A011D042003E0002881
:101C6000BCBF014400207E18D96941F00801D96148
:101C700058F8241001EB821151F80C3066F30E3342
:101C800041F80C3058F8241001EB82114A5960F3E6
:101C900012424A51BDE8F0037047A04A800900296A
:101CA00052F82000816914BF41F0080121F00801B9
:101CB000816170479949800951F820008069C0F31B
:101CC000C0007047954A8009002952F820008169B8
:101CD00014BF41F0020121F00201816170478F4978
:101CE000800951F820008069C0F3400070478B4B99
:101CF000820953F8223000F00F0202EB420203EB9C
:101D00008212C0F301104FF4A67303EB8010115040
:101D10007047824A810952F8212000F00F0101EB3F
:101D2000410102EB8111C0F301104FF4A67202EBE6
:101D3000801008587047784A10B4D2F8400110F06B
:101D4000010F0BD0D2F84C01D2F844110028C1F396
:101D500002311EBF0029C043C2F84C0101230020FC
:101D600003EB43018C0104EB801101F1804101F58B
:101D7000A041D1F8402112F0010F0CD0D1F84C2134
:101D8000D1F844C1002ACCF3023C1EBFBCF1000FC5
:101D9000D243C1F84C21401C0228E4D35B1C032B26
:101DA000DDD310BC704700225C49830951F8231031
:101DB000CB6913F0080F0ED000F00F0202EB4202C5
:101DC00001EB8211C0F301104FF4A47202EB8010FA
:101DD0000858C0F3005210467047012070472DE9A3
:101DE000F04F82B0022ADDE90B49DDF8348026BFCE
:101DF000921E4FEA520C4FF0000C022B26BF9A1E87
:101E000053080023464AA2FB04421709B8F1000F09
:101E100014BF012200220192B9F1020F16BF5FEA3E
:101E200009024FF0010B4FF0000B82093B4C00F010
:101E30000F0606EB460554F822404FF4B27E04EB41
:101E4000851AC0F301140EEB841ECDF800A05AF8D9
:101E50000EA061F35C6A6BF3186A05D167F3174A49
:101E600063F3CA1A6CF3C60A019969F3420A61F373
:101E7000000A0099DFF8A49041F80EA059F822203A
:101E80004FF4B471C0F3011A01EB8A1102EB851211
:101E9000B8F1000F555814BF45F0800525F08005B6
:101EA00055500125B5EB901F1CBF02B0BDE8F08F67
:101EB00004EB46001B4951F82020183111F820800E
:101EC00006EB4600800100EB841000F1804000F535
:101ED000A040D0F850491449FF26A1FB02914908BF
:101EE000A1EB81094A44D2009640FFB297404FEAE5
:101EF0008802002003F00F0393400CF00F0C4FF00A
:101F00000F090CFA02FC09FA02F24FEA810805FAFD
:101F100000F121422DD009E000500040884102002C
:101F2000CDCCCCCCA8410200ABAAAAAA08EBC00138
:101F300001F1804101F5A041D1F8809C29EA060910
:101F400049EA0709C1F8809C810001F1804101F54F
:101F5000A041D1F8A89C29EA020949EA0309C1F87D
:101F6000A89CD1F8BC9C29EA020949EA0C09C1F8ED
:101F7000BC9C401C0528CAD302B0BDE8F08F2DE9F7
:101F8000F04F84B0DDE90EA8DDF834C0B8F1000FE1
:101F900014BF012400240294BAF1020F16BF5FEAB5
:101FA0000A044FF0010B4FF0000B8409FA4D00F0CA
:101FB0000F0707EB470655F824504FF4B27E05EBA8
:101FC0008619C0F301150EEB851ECDE9009E59F868
:101FD0000E9061F35C696BF318697CD002996AF327
:101FE000420961F30009DDE9001BDFF8ACA341F809
:101FF0000B904FF4B4715AF82440C0F3011901EB6F
:10200000891104EB8614B8F1000F665814BF46F02E
:10201000800626F0800666500126B6EB901F1CBF96
:1020200004B0BDE8F08F05EB4700DC49DC4C51F80B
:10203000201054F8204007EB4700800100EB85108A
:1020400000F1804000F5A040D0F85009D54DFF26A2
:10205000A5FB01756D08A5EB850739444FEAC10959
:10206000009006FA09FE00200F21A400A1404FEACB
:10207000850B012505FA00F6009D2E4241D015681A
:10208000022D26BFAD1E6D080025121D1E68022EF2
:1020900026BFB61E760800265CF8048BC24FA7FB4D
:1020A00008874FEA07580BEBC00707F1804707F591
:1020B000A047D7F880AC4FEA18682AEA0E0A08FA57
:1020C00009F84AEA0808C7F8808C870007F18047BA
:1020D00007F5A04700E01AE0D7F8A88C06F00F0635
:1020E00028EA0108A64048EA0606C7F8A86CD7F80F
:1020F000BC6C05F00F058E43A5403543C7F8BC5CAA
:102100001B1D401C0528B4D304B0BDE8F08F116836
:10211000022926BF891E49080021D3F800B0BBF16F
:10212000020F26BFABF1020B4FEA5B0B4FF0000B27
:10213000CDF80CB0DFF870B2DCF800E0ABFB0EEBD2
:102140004FEA1B1B6BF31749DDF80CB06BF3CA1990
:1021500061F3C60942E72DE9F00F8F4D84094FF472
:10216000B27955F8244000F00F0505EB450604EB65
:102170008614C0F3011609EB8619DDE9098754F8C6
:102180000940DDF820C0C4F3436BC4F3410904F0F7
:10219000010A002918BFC1F800B0B8F1000F18BF3C
:1021A000C8F80090002F18BFC7F800A081094FF0B1
:1021B00001085BD0B8EB901F1CBFBDE8F00F704763
:1021C00006EB45007549764C51F8201054F820B0C4
:1021D00005EB4500800100EB861000F1804000F522
:1021E000A040D0F850A96F4C0020A4FB0154640813
:1021F0004FEA8409A4EB84042144CF004FEA8B0505
:1022000008FA00F111EA0A0F2AD009EBC00101F126
:10221000804101F5A041D1F8801CF940840004F10F
:10222000804404F5A044C9B2D4F8A86CD4F8BC4CDE
:10223000EE4006F00F06EC4004F00F041AB1640003
:10224000A41C42F8044B1BB17400A41C43F8044BBB
:10225000BCF1000F04D001EB810189004CF8041B94
:10226000401C0528CCD3BDE8F00F7047C4F30740ED
:10227000C4F3C311C4F3C30412B16400A41C1460FA
:1022800013B14900891C1960BCF1000F04BFBDE8FF
:10229000F00F704700EB80008000CCF80000BDE834
:1022A000F00F70473C4A8009002952F82000C169AC
:1022B00014BF41F0200121F02001C161704736496F
:1022C000800951F82000C069C0F34010704730B455
:1022D00090B000224FF48045EC466C1001E0082AD3
:1022E00005D2531C03EB8303B5FBF3F304E0D31FC8
:1022F00003EB8303B4FBF3F35B1A48BF5B424CF878
:102300002230521C102AEAD30023009C01215CF8E1
:102310002120A242BCBF14460B46491C1029F6D30B
:1023200000F00F0202EB42014FEA8111C0F3011CE1
:1023300001EB8C1101F18041840901F5A04135D0F8
:102340000124B4EB901F1EBF10B030BC70470CEBE3
:102350004200D1F850C9124A12F820200F259100EE
:1023600000208D4003F00F028A4004FA00F111EAC8
:102370000C0F0AD0810001F1804101F5A041D1F894
:10238000D03CAB431343C1F8D03C401C0528ECD3F0
:1023900010B030BC7047000088410200A841020024
:1023A000C0410200ABAAAAAACDCCCCCCD1F868011E
:1023B00063F30300C1F86801EAE781091CBF00204C
:1023C000704700F00F0101EB41018901C0F30110DA
:1023D00001EB801000F1804000F5A040D0F86801CA
:1023E00000F00F00082834BF401CC01F00EB800025
:1023F00034BF4FF480414FF40051B1FBF0F070470F
:102400002DE9F0074FF0010991B0B9EB901F1EBF05
:1024100011B0BDE8F007704700F00F02C0F30110E3
:1024200000EB420302EB4202920102EB8010DFF864
:102430003CC500F1804000F5A0405CF82330D0F8A6
:1024400050A90F204FEA83084FF0000C4FF480464C
:102450006C4600FA08F709FA0CF010EA0A0F36D0B9
:1024600051F8043B00204FF4005501E0082805D244
:10247000421C02EB8202B6FBF2F204E0C21F02EB46
:102480008202B5FBF2F2D21A48BF524244F8202031
:10249000401C1028EAD30025009B012054F820207E
:1024A0009A42BCBF13460546401C1028F6D34FEA9B
:1024B0008C0000F1804000F5A040D0F8D02C05F051
:1024C0000F03BA4303FA08F31A43C0F8D02C0CF1F7
:1024D000010CBCF1050FBED311B0BDE8F007704789
:1024E00070B40124B4EB901F1CBF70BC704700F0A7
:1024F0000F02C0F3011000EB420302EB4202920113
:10250000DFF868C402EB801000F1804000F5A040C5
:102510005CF82330D0F850C900209B004FF4804570
:102520006E1004FA00F212EA0C0F16D0820002F1CB
:10253000804202F5A042D2F8D02CDA4002F00F021D
:10254000082A34BF521CD21F02EB820234BFB5FBF3
:10255000F2F2B6FBF2F241F8042B401C0528E0D35E
:1025600070BC704700F00F02C0F3011303EB42028E
:10257000FE4B8009A3F1380C53F822205CF82000B0
:1025800001230029D0F8101403FA02F214BF1143FA
:102590009143C0F81014704700F00F01C0F301130D
:1025A00003EB4101F14B0022800913F82110383B65
:1025B00053F82000D0F81004012303FA01F1084277
:1025C00018BF01221046704770B410F0300F14BFCE
:1025D000012300238609DFF898C300F00F024FEAB9
:1025E00090104FF49A7502EB42025CF820004FF015
:1025F000010405EB821214D085584FEA430C5B426C
:102600000CEB43039B1C04FA03F35B1E03FA0CF46C
:10261000194025EA040401FA0CF12143815070BCF1
:1026200070470029815804FA03F31ABF19438150F7
:102630009943F3D070BC704730B410F0300118BF2C
:10264000012184094FEA9013C94D00F00F0000EBFF
:1026500040004FF49A7202EB801255F823004FF0BD
:10266000010C0CD082584800C240494200EB4100A6
:10267000801C0CFA00F0401E30BC1040704780589F
:102680000CFA01F1084018BF012030BC7047B84B6C
:10269000800953F820C0CCF8741053F820C011689A
:1026A000CCF8781053F820005168C1677047B149E1
:1026B0000028D1F8AC0014BF40F0020020F0020066
:1026C000C1F8AC007047AB490028D1F8AC0014BF8A
:1026D00040F0010020F00100C1F8AC007047A548AF
:1026E000D0F8E000A449096808437047A149C1F83F
:1026F000E400A249086070479E48D0F89800A049BD
:10270000096840EA4100704770B44FEA00758609D5
:1027100000F00F044FEAD565C0F30110A5F10205E2
:1027200002F0010C05444FEA8C334FEA520012D0FC
:1027300001EB41017CB305EB4502D20002EB8C3288
:1027400002EB810101EB800000F1405000F5C03048
:10275000406A70BC704701EB410202EB01117CB191
:1027600098226A4302EB8C3202EB810101EB80007C
:1027700000F1405000F58030D0F88C0E70BC7047EE
:1027800003EB810101EB800000F1405000F5803047
:10279000006870BC7047FFE703EB810101EB80002C
:1027A00000F1405000F5C030006870BC7047F0B4D4
:1027B0004FEA0076870900F00F044FEAD666C0F3AF
:1027C0000110A6F1020602F0010C06444FEA8C3516
:1027D0004FEA520012D001EB41017CB306EB4602F6
:1027E000D20002EB8C3202EB810101EB800000F1A0
:1027F000405000F5C0304362F0BC704701EB41022D
:1028000002EB01117CB19822724302EB8C3202EB95
:10281000810101EB800000F1405000F58030C0F8EC
:102820008C3EF0BC704705EB810101EB800000F1AC
:10283000405000F580300360F0BC7047FFE705EBC7
:10284000810101EB800000F1405000F5C0300360D1
:10285000F0BC7047830900F00F02C0F301100CD0E8
:10286000002A08BF474805D0012A17D000280CBF0E
:102870004548464800EB81307047002A08BF4FF0BA
:102880004050F7D0012A04D000280CBF40484148EE
:10289000F0E7002814BF40484048EBE7002814BF89
:1028A0003F484048E6E710B44FEA007C840900F056
:1028B0000F034FEADC6CC0F30110ACF1020C604472
:1028C00010D0002B08BF38481CD000EB4000C000DF
:1028D00000EB813002EB420100EB8100334910BC78
:1028E00008447047002B08BF31480BD09823584349
:1028F00000EB813002EB420101EB021100EB8100A1
:102900002C49ECE710BC00EB813070472DE9F00753
:102910004FEA901C00F00F04154804EB440150F8F6
:102920002C0000F5C07300EB8110D0F800014FF4CB
:102930007A7280B2B2FBF0F100FB1120002818BFC0
:1029400001200D181C4F002040F2FF1644EA001130
:1029500041EA8C1101F00F02C1F3011101EB4201B8
:1029600057F821104A08C907C90E27E0C0410200E4
:102970008841020000500040E0580040E458004008
:102980009858004000800030E481003024830030FB
:102990004C1800304C1D0030CC0E0030CC090030FB
:1029A00064810030248000300080013024800130B8
:1029B000000001308C0E01309041020053F822805B
:1029C00003EB820228FA01F8D2F80CA0A8EB050963
:1029D00006FA01F8C9F308092AEA080A09FA01F116
:1029E0004AEA0109C2F80C90D2F8189029EA0808BE
:1029F00048EA01019161401C0228A7D3BDE8F00715
:102A000070470000FEF716B810B5FEF713F801285E
:102A100018BF10BD0020FDF7C8FF21210020FEF7E0
:102A20000FF82121BDE810400120FEF709B810B5CC
:102A3000FDF7B4FFFDF7FEFF01280AD10020FDF7E6
:102A4000B4FF21210020FDF7FBFF21210120FDF72C
:102A5000F7FF0121052001F0E8FE0121052001F02A
:102A6000E4FEFB490020887110BD10B54FF40660EC
:102A700001F031FFBDE810404FF4066001F01CBFCB
:102A8000F34A01461079002818BF0120002918BF19
:102A900001211171002151717047ED4A916A9062D4
:102AA00008467047EA490020C8708870487070472F
:102AB000E7490020C87088704870704710B5044618
:102AC00001468422E3481BF0DDFF04F18401BDE8E8
:102AD00010408422E0481BF0D5BF70B50007C00E3F
:102AE0000D46801E00EB400101EB0014DB484FF463
:102AF000987200EBC40029461BF0C4FFD84805F5C6
:102B0000987100EBC400BDE870404FF498721BF060
:102B1000B9BF2DE9F04105460020FDF7CFFF06467D
:102B20000CF045FF04464FF48061CE481BF0AFFF28
:102B30000021AB1902274FF0010C6856002810DB6A
:102B40000209120202EB810202F1405202F5003248
:102B50000007C00ED2F800800CFA00F048EA00002E
:102B60001060012C06D0022C0CD0032C12D0042CA7
:102B700017D02DE024292BD2681890F902000028E4
:102B800026DB14E0252923D2681890F901000028DB
:102B90001EDB0CE025291BD213F9010C002817DBE2
:102BA00005E0242914D213F9020C002810DB0209D5
:102BB000120202EB810202F1405202F500320007DC
:102BC000C00ED2F8008007FA00F048EA000010605A
:102BD000491C2629B1D30021012C38D0022C4FD01A
:102BE000032C5CD0042C18BFBDE8F081B00000F1CC
:102BF000405202F5F83202F58050C2F8FC1FC0F8CE
:102C0000FC10C0F8FC11C0F8FC12C2F8F81FC0F8A4
:102C1000F810C0F8F811C0F8F812B11E6856002874
:102C20000EDB0209120202EB810101F1405101F5B4
:102C300000310007C00E0A680CFA00F0104308606B
:102C4000711E68560028B8BFBDE8F0813AE0B000B8
:102C500000F1405202F5F83202F58050C2F8FC1F34
:102C6000C0F8FC10C0F8FC11C0F8FC12C2F8F81F44
:102C7000C0F8F810C0F8F811C0F8F812BDE8F081FB
:102C8000794AB000115000F1405000F50030C0F812
:102C9000FC10C0F8FC11C0F8FC12BDE8F081724ACB
:102CA000B000115000F1405000F50030C0F8FC10A9
:102CB000C0F8FC11C0F8FC12711E68560028B8BF9D
:102CC000BDE8F0810209120202EB810101F14051DD
:102CD00001F500310007C00E0A680CFA00F010433D
:102CE0000860BDE8F081DFF87CC148B14A424FF48A
:102CF000806300EB810103EB820260461BF0C2BEE1
:102D00004FF4806160461BF0C2BE2DE9F0410546DC
:102D10000020FDF7D3FE554FDFF854810446EDB196
:102D20004C2004FB00F21646294638461BF0AAFE4A
:102D3000324605F5E46140461BF0A4FE04EB440076
:102D400000EB041407EB84004C211BF0A0FE08EB01
:102D50008400BDE8F0414C211BF099BE4C21401C81
:102D600041430C4638461BF092FE21464046BDE8E2
:102D7000F0411BF08CBE10B5354C2062FEF74EF9C9
:102D8000FEF723F9A169A269C1F307216FF30F02CE
:102D9000A261A369C2B243EA0222A261022803D15E
:102DA000A26942F00102A26181421ABFE269002ACF
:102DB00010BD012918BF0021012818BF0020814241
:102DC00008BF10BDBDE8104010474FF0402081699A
:102DD00041F002018161016941F00301016100F0EC
:102DE000B2BF2DE9F0414FF04022054690690C46F4
:102DF00040F002009061106940F00301116100F0A1
:102E0000A2FF2E460025002C7ED00020FDF7CDFD30
:102E100000202168FDF7BEFF40206168FDF7BAFF82
:102E20003046FFF7A8FF0020FDF779FE68B3A068E1
:102E3000FFF76BFF6169E9B1E0694FF480634242DB
:102E400001EB800103EB820206481BF01BFE15E03C
:102E5000308000100080013000C001308C0E013045
:102E60008C4E013000000230FCFF013000000130C8
:102E7000004001300021FE48FFF74BFEFD48A169EC
:102E800069B14FF400721BF0FDFDE068A0B30120B2
:102E9000FDF745FEDFF8E083F84F28B108E04FF476
:102EA00000711BF0F4FDF0E71120FDF738FE68B16A
:102EB000E66840464FF4987231461BF0E3FD384611
:102EC0004FF4987206F598711BF0DCFD0220FDF7B7
:102ED00026FE18B91220FDF722FE68B1E668E84820
:102EE0004FF4987231461BF0CDFDE6484FF49872CE
:102EF00006F598711BF0C6FD4120FDF710FE28B9BC
:102F00005120FDF70CFE00E00DE060B1246954B1E2
:102F100084222146DC481BF0B5FD842204F18401A3
:102F2000DA481BF0AFFDDA48C570857045708562E0
:102F300001790021017145714FF4066001F0CBFC6D
:102F4000BDE8F0414FF4066001F0B6BC10B50020BA
:102F5000FDF72BFD00F0E7FECD48406B002808BFD1
:102F600010BD4FF04020016921F00301016181692A
:102F700021F00201816110BD4FF4066001F0A1BC97
:102F800010B54FF4066001F09CFCFDF753FD0128DD
:102F90000AD10020FDF709FD21210020FDF750FD99
:102FA00021210120FDF74CFDBA48D0F8401321F44F
:102FB0008031C0F840130020FDF7F7FC00F0B3FEAD
:102FC000B348406B002808BF10BD4FF04020016996
:102FD00021F003010161816921F00201816110BDCD
:102FE00010B501F073FC10F0600018BF012010BD97
:102FF000A74AD169D06108467047A548006A704762
:10300000A3488069704772B6A1498A6922EA000024
:10301000886162B670479E480078002818BF01207A
:10302000704770B5FDF706FD002818BF70BD00247D
:10303000974DEC70AC706C7021212046FDF700FDBF
:1030400021210120FDF7FCFC2C70BDE8704001201F
:10305000FDF7ABBC70B50446FDF7ECFC002818BFCB
:1030600070BD00218A4DE970A9706970212100208E
:10307000FDF7E6FC21210120FDF7E2FC022C3CBF1C
:103080000120FDF7EDFC012028706C62BDE8704066
:10309000FDF78BBC10B5FDF7CDFC002818BF10BDA7
:1030A00000207B4CE070A07060702121FDF7C8FC0F
:1030B00021210120FDF7C4FC0120FDF7D1FC0120F6
:1030C00020706062BDE81040FDF76FBC0020FDF786
:1030D0006CBC10B56E4C0020A07060702121FDF713
:1030E000AFFC21210120FDF7ABFC207800281CBF9C
:1030F0000120FDF7B5FC0120BDE81040FDF755BCEF
:103100006349C86270476248C06A70476049086393
:1031100070475F48006B70475D4A00F00F00116B0D
:1031200021F00F01084310637047594890F83000B0
:1031300000F00F00704770B5554C0546E06A421C20
:10314000E262216B11F0800F14BFC1F3021101F094
:103150000F0139B1B2FBF1F001FB1020002808BFCC
:10316000FEF7E9FD207850B1606A10B1606A401E38
:103170006062606A002804BF0020FDF716FC202171
:103180002846FDF75DFCA16A00291CBF2846884738
:10319000FDF71BFF022815D13E48D0F8481311F067
:1031A000010F0FD0D0F8481341F00101C0F84813C7
:1031B000D0F8481321F00101C0F84813A06940F08D
:1031C0000200A0613448016841F02001016070BD37
:1031D0000020B0E70120AEE710B5FFF780FA044603
:1031E000FFF784FA2D48044208BF10BD28488169C2
:1031F00041F0040181610E2101EAD43104F00102A1
:103200000A43816962F31F4181612348016841F0EB
:103210002001016010BD002818BF01201C4948632F
:103220007047134870471E4870471948806B7047B5
:103230001748C179427A914214BFC06B006C704745
:103240001348006C70472DE9F04F0025DFF82090FF
:103250008DB009F14C04AC466F1E09F8057004F8F6
:1032600005C06D1C262DF8DB0025002820DD19E0A7
:1032700078860010004002308C0E01308C4E0130F8
:10328000BC0F0130BC4F01300080013000C0013064
:1032900030800010005000408480001001000700C2
:1032A0009E860010565D09F805606D1CA842DEDCA4
:1032B00000220126CDF804C06D46CDF800C00028DC
:1032C00021DD19F902B0BBF1000F19DBBBF1140FBE
:1032D000A8BFABF1140B04DABBF10A0FA8BF0BF1C6
:1032E000120BBBF1260F0BD24FEA5B180BF01F0B32
:1032F00055F828A006FA0BFB4AEA0B0A45F828A065
:10330000521C8242DDDB002292460DF108084FEA92
:10331000521B02F01F0E55F82BB006FA0EFE1BEAE8
:103320000E0F1ABF08F802A00AF1010A08F802708D
:10333000521C262AEBDB4FF0000A002816DD19F993
:103340000A20002A0EDB142AA8BF143A02DA0A2A3D
:10335000A8BF1232262A3ABF18F8022004F80A2021
:1033600004F80A700AF1010A8245E8DBDFF81894D4
:1033700000220028C9F838C009DD14F902A09245DE
:1033800002D0C9F8384002E0521C8242F5DBFF4A05
:103390000020A2F17204A2F1260A27540AF800C004
:1033A00002F800C0401C2628F7DB0020002906DDBB
:1033B00013F800B004F800B0401C8142F8DC002093
:1033C000CDF804C0CDF800C0002913DD2356002B32
:1033D0000DDB262B0BD24FEA531B03F01F0355F8CE
:1033E0002BE006FA03F34EEA030345F82B30401CAA
:1033F0008842EBDB002003464FEA501B00F01F0E13
:1034000055F82BB006FA0EFE1BEA0E0F1ABF08F88D
:1034100000305B1C08F80070401C2628ECDB002004
:1034200000290ADD2356002B04DB262B3CBF18F8AD
:1034300003301354401C8842F4DB0020C9F840C01C
:10344000002908DD1356834202D0C9F8402002E06B
:10345000401C8842F6DB11F0010F18BF252015D063
:10346000420900F01F0355F8222006FA03F31A421E
:103470000AD1420900F01F0055F8223006FA00F088
:10348000184345F8220001E0401EE9D5002002461D
:10349000430900F01F0B55F8233006FA0BFB13EA23
:1034A0000B0F1ABF08F80020521C08F80070401CCF
:1034B0002628EDDB002000290BDD2256002A05DB43
:1034C000262A3CBF18F802200AF80020401C884237
:1034D000F3DB0020C9F83CC00029DCBF0DB0BDE81B
:1034E000F08F1AF90020824204D0C9F83CA00DB038
:1034F000BDE8F08F401C8842F3DB0DB0BDE8F08FD3
:10350000A3487047A048406C70472DE9F001A04CDB
:10351000002282B0551E04F1050CA5540CF802508F
:10352000521C052AF9DB00228B5CA354521C052A8D
:10353000FADB00230127194600280AD96256002A1F
:1035400004DB052A3CBF07FA02F21343491C8142FF
:10355000F4D300210A466E4607FA01F818EA030F71
:103560001ABF7254521C7554491C0529F4DB002102
:1035700000280AD96256002A04DB052A3CBFB25C47
:103580000CF80120491C8142F4D37F4B0021002814
:1035900059649EBF02B0BDE8F00170471CF90120DC
:1035A0008A4205D0C3F844C002B0BDE8F0017047BC
:1035B000491C8142F2D302B0BDE8F001704740F2ED
:1035C000DB114843734901EB800070477249C0EB3F
:1035D000001001EBC0007047DFF8ACC1012B8CF884
:1035E00007008CF8081003D9401C20F00100114698
:1035F0008CF809008CF80A1000FB01F24FF6FF71FD
:1036000001EA4202ACF8122001EA4000ACF81400D2
:1036100070475D48807A70475B48407A70475A4AE5
:10362000D072117370475848007B70475648C07A73
:1036300070475A4A1070517070475849085C70477B
:103640002DE9F047DFF84091044699F8040000287E
:1036500004BF99F801001BF01FFA0AF092FA58B95A
:1036600004F030F8022818BF052805D100230122F4
:103670007F2107200EF07AF899F80300002808BF90
:10368000BDE8F0874FF00008D9F8200047464646CD
:10369000454610F0070F1CBFDFF8F88010F0020F4E
:1036A00005D0B9F812103B4A21F001018F1810F033
:1036B000F00F18BF384E10F4774F18BF384DD9F8B7
:1036C0002C002060FDF784FC10F0010F06D0FEF7FF
:1036D00022F8022828BF99F8020000D20020E760F3
:1036E000C4E90108C4E904650120BDE8F087264863
:1036F0000021C1704171704770B505460020FDF78B
:10370000DDF94C2100FB01F21446264928461BF046
:10371000B9F9224605F5E460BDE8704022491BF086
:10372000B1B9F0B583B00020FDF7C8F90446694689
:103730000020FEF753F90022002C3DD96E464FF0D1
:10374000010C4FF6F07502EB4200002100EB021075
:103750004B0901F01F0756F823300CFA07F73B42DC
:1037600024D0CB075B0C03EB80034F0803EB8703EC
:1037700003F1405303F580331B889BB2AB4215D94C
:10378000002003B0F0BD0000308000101087001052
:1037900078800010B01901101C2101103D8000102C
:1037A0000C2201100000013000400130491C262984
:1037B000CED3521CA242C6D30120E2E770B5000767
:1037C000C00E0D46801E00EB400101EB0014FD48C9
:1037D0004FF4987200EBC40128461BF053F9FA48E5
:1037E0004FF4987200EBC40105F59870BDE8704085
:1037F0001BF048B92DE9F04F07460007C00E83B013
:10380000801E002527F03F0BE9464FF001084FF6D8
:10381000F0760290384665F31F1040EA0B0000F086
:10382000FF0A5046FDF77BF900283DD05046FEF7D1
:1038300078F908FA00F4022C88BF02246946504641
:10384000FEF7CCF80022002C2ED9029898212844AB
:1038500000FB01FA02EB4200002100EB021C4809C8
:1038600001F01F0359F8200008FA03F3184215D09D
:1038700001F001000AEB803000EB8C004B0800EBFC
:10388000830000F1405000F58030B0F88C0E80B21B
:10389000B04203D903B00020BDE8F08F491C2629AF
:1038A000DDD3521CA242D5D36D1C022DB2D303B07E
:1038B0000120BDE8F08F10B504468422C3491BF0F7
:1038C000E1F804F18400BDE810408422C0491BF0F7
:1038D000D9B82DE9F04F83B0002002904020FDF7C9
:1038E0001EF9E9464FF001084FF6F07758B3402033
:1038F000FDF7E4F8044669464020FEF76FF8002221
:10390000002C20D9002102EB420C480959F8203044
:1039100001F01F0008FA00F003420ED0C807400C67
:1039200000EB8C004B0800EB830000F1405000F5E9
:10393000C030008880B2B84254D8491C0529E4D36D
:10394000521CA242DED301267000A0F1020B00251A
:1039500046EA0510C0B240F0400A5046FDF7DFF8D5
:10396000B8B35046FEF7DDF808FA00F4022C88BF21
:10397000022469465046FEF731F80021002C28D970
:103980000BEB050000EB40004FEAC00A002001EB02
:10399000410C420900F01F0359F8222008FA03F3F2
:1039A0001A4210D000F001020AEB823202EB8C02C4
:1039B000430802EB830202F1405202F5C032928CBE
:1039C00092B2BA420ED8401C0528E2D3491CA1424B
:1039D000DCD36D1C022DBBD3701CC6B2022EB3D932
:1039E00001200290029803B0BDE8F08F2DE9F0416C
:1039F0000026784D00280C4645D000F00F01C0F39A
:103A0000011001290EBF00210229BDE8F081022822
:103A100028BFBDE8F0810F18FDF70CF85FEA000839
:103A20001CBF0020FCF7C1FF00239820474303EB95
:103A30004300002200EB031C02F0010007EB803082
:103A4000510800EB8C0000EB810000F1405000F5C4
:103A50008030521CC0F88C4E262AEDD35B1C022B02
:103A6000E5D3B8F1000F08BFBDE8F081AE706E700D
:103A700021210020FCF7E4FF21210120FCF7E0FFD9
:103A80002878A0B330E0FCF7D5FF07001CBF00206A
:103A9000FCF78BFF002303EB4300002200EB031035
:103AA000D107490C4FEA520C01EB800101EB8C0C61
:103AB0000CF1405C0CF5803C521CCCF80040262AEE
:103AC000EED35B1C312BE6D3002F08BFBDE8F0819D
:103AD000AE706E7021210020FCF7B2FF2121012081
:103AE000FCF7AEFF287810B10120FCF7B9FFBDE864
:103AF000F0410120FCF759BF10B5FDF70FFF354924
:103B0000088210BD334B10B4E02101EA102C1B8A4F
:103B1000C1B2C0F30422994288BF194664246143AC
:103B2000B1FBF3F102EBC20303EB021201EB8201E2
:103B30004FF47A72284B0CFB02F2A3FB023292087C
:103B4000521C520810F4803F08BF494210F4003F55
:103B500014BF8818881A00B210BC704700211F4893
:103B6000FEF7D7BF01211D48FEF7D3BF10B50121D5
:103B70001A48FEF7CEFF41F2EC0119481AF087FF10
:103B8000BDE8104041F2EC0116481AF080BF114820
:103B900010B5006A14490840FFF7EDF84FF4806152
:103BA00012481AF074FF40F68C610D481AF06FFF4E
:103BB00040F68C610B481AF06AFFBDE81040002007
:103BC000FDF7BCBC8C0E01308C4E01300080013002
:103BD00000C0013030800010ABAAAAAA788600107D
:103BE00000000130004001300100FF000000023001
:103BF00082B04FF4FA62009013E000BF00BF00BF34
:103C000000BF00BF00BF00BF00BF00BF00BF00BFBC
:103C100000BF00BF00BF00BF00BF0198411E01915F
:103C2000EBD20098411E009128BF0192F5D202B05C
:103C300070472DE9F0410027634D0126002808BF99
:103C40002E701FD001282F7018BF6F701AD04FF040
:103C50004028D8F8100040F00400C8F81000297877
:103C60005A4C002914BF49F608305948E06014BF87
:103C700058484FF0BB70A0605748006830F0FF0212
:103C800006D101E06E70E2E7E26860F30302E260F1
:103C900089B1A06840F01800A0600120FFF7A8FFDC
:103CA000A06840F48050A0600120FFF7A1FFA06849
:103CB00040F40070A0600120FFF79AFF687870B1AF
:103CC000E06840F02000E060A06820F40070A06090
:103CD0000120FFF78DFFE06840F01000E060D4F8AD
:103CE000B00040F00100C4F8B0000120FFF780FFF1
:103CF000E6674FF4E0602061C4F8887028780028F7
:103D000018BFC4F89460E06820F03000E060A0685C
:103D100020F49050A060D8F8100020F00400C8F8FB
:103D20001000BDE8F0812948C16821F03001C16070
:103D3000816821F4905181604FF04020016921F0A9
:103D40000401016170474FF04020016941F0040116
:103D500001611D491D480A783AB1826842F0180293
:103D60008260826842F490528260497819B1C168D9
:103D700041F03001C160D0F8B01041F00101C0F84D
:103D8000B0107047B0F5007F28BF40F2FF10C0F3BD
:103D90000800124941EA00200C49086470470B49A9
:103DA0004FF0204008647047084A116C4FF02040E3
:103DB0001064506C11F0FF0FC0F308201CBF41F0DD
:103DC00020411164704700008280001000600040B4
:103DD00005F4010020009B00D0FE0400130000A0A9
:103DE0004FF040200021016302224263826B02F007
:103DF0003C0242F001028263026922F00302026186
:103E0000026A22F001020262424A136843F001038F
:103E100013603C2282612822C2613F4801603F4812
:103E200001603F4850F88C2F42F4805202603D4AB6
:103E3000481E10603C480160704710B501F0F9FA67
:103E400039480468002C08BF30BFFAD00021016057
:103E500001F0F3FA204610BD10B501F0EAFA324B3A
:103E600000204FF0402101221C6824B1186001F0AD
:103E7000E4FA204610BD72B6D1F838C00CF03C0C04
:103E8000C1F838C00A6320BF0863D1F838C00CF00D
:103E90003C0C4CF0010CC1F838C062B6BFF36F8F18
:103EA000BFF34F8FE0E710B504460F2000F0F8FC99
:103EB0000F2000F0DDFC1D490A6842EA040008609A
:103EC00010BD1A490A6822EA000008607047164AC5
:103ED000516850600846704770B51448006814492E
:103EE0000968114D00EA0104696800291CBF2046D9
:103EF000884714F0100F05D0094850F88C1F41F482
:103F00008051016007480460286840F40040286040
:103F100070BD0000004800402448004010480040A8
:103F20000030004014480040848000101C480040CD
:103F300018480040704770470022B2EBD10F26D2DC
:103F40000368B3F1FF3F04BF4368B3F1FF3F17D1EC
:103F50008368B3F1FF3F04BFC368B3F1FF3F0FD1E4
:103F60000369B3F1FF3F04BF4369B3F1FF3F07D1DA
:103F70008369B3F1FF3F04BFC369B3F1FF3F01D0D1
:103F8000002070472030521CB2EBD10FD8D3012053
:103F9000704710B40023B3EBD20F30D2D0F800C07A
:103FA0000C68A44522D1D0F804C04C68A4451DD1AA
:103FB000D0F808C08C68A44518D1D0F80CC0CC68E3
:103FC000A44513D1D0F810C00C69A4450ED1D0F887
:103FD00014C04C69A44509D1D0F818C08C69A44517
:103FE00004D1D0F81CC0CC69A44502D010BC00207C
:103FF0007047203020315B1CB3EBD20FCED310BC06
:10400000012070472DE9F041054601F01AFA002021
:1040100021264FF4825784464FF4E0221660C5F8FB
:1040200000C0116841F004011160116811F0040F23
:10403000FBD1176080232C460021D4F80080B8F112
:10404000FF3F04BFD4F80480B8F1FF3F1DD1D4F87E
:104050000880B8F1FF3F04BFD4F80C80B8F1FF3FEF
:1040600013D1D4F81080B8F1FF3F04BFD4F8148006
:10407000B8F1FF3F09D1D4F81880B8F1FF3F04BF71
:10408000D4F81C80B8F1FF3F08D0C2F800C0401C33
:10409000C0B20828C2D30220BDE8F081491C2034F8
:1040A000B1EBD30FC9D3C2F800C00120BDE8F08145
:1040B0002DE9F041054601F0C4F9002009268446A7
:1040C0004FF4E0231E60C5F800C0196841F00401F8
:1040D0001960196811F0040FFBD12C464FF480626F
:1040E00000212768B7F1FF3F04BF6768B7F1FF3FC2
:1040F00017D1A768B7F1FF3F04BFE768B7F1FF3FEB
:104100000FD12769B7F1FF3F04BF6769B7F1FF3FE0
:1041100007D1A769B7F1FF3F04BFE769B7F1FF3FD8
:1041200008D0C3F800C0401CC0B20328CAD3022084
:10413000BDE8F081491C2034B1EBD20FD1D3C3F8D4
:1041400000C00120BDE8F0812DE9F05F884681467E
:1041500004274FF07F0A4FF0020B4FF4E02601F0E6
:1041600070F94946424653464FF0060CC6F800B077
:1041700052F8040B41F8040BC6F800C0306810F088
:10418000040FFBD15B1EF1D2002030604C46454647
:104190001F20D4E900C3D4E90221D5F800E0E645A8
:1041A00004BFD5F804C09C4505D1AB68934204BF59
:1041B000EA688A4208D07F1E03D34846FFF722FFF1
:1041C000CDE70220BDE8F09F10341035401EE0D24C
:1041D0000120BDE8F09F70B50D46044601F031F9AD
:1041E0004FF40072214628461AF04CFC012070BDA5
:1041F0002DE9F0410546C005ADF5007D14460E469B
:10420000C00D25D0A8466FF308086F4601F019F9D4
:104210004FF40072414638461AF034FCC5F30800EA
:10422000C0F50077A74288BF274668443A46314622
:104230001AF037FC4046FFF7E5FE022844D06946F5
:104240004046FFF781FF022843D03D443E44E41B33
:10425000B4F5007F19D34FF40072314668461AF066
:1042600020FC2846FFF7CEFE02282DD069462846BE
:10427000FFF76AFF02282CD0A4F5007405F500753D
:1042800006F50076B4F5007FE5D2C4B16F4601F0C3
:10429000D8F84FF40072294638461AF0F3FB22464C
:1042A000314668461AF0FDFB2846FFF7ABFE0228B0
:1042B0000AD069462846FFF747FF022809D00DF5C6
:1042C000007D0120BDE8F0810DF5007D0A20BDE8EC
:1042D000F0810DF5007D0B20BDE8F08130B4354D47
:1042E0002A68002101244FF0030C04FA01F3034271
:1042F00004D04B000CFA03F39A431A43491C0C29CF
:10430000F3DB2A6030BC7047F0B42A4D2A680021E4
:1043100001244FF0030C022604FA01F3034206D0F5
:104320004B000CFA03F7BA4306FA03F31A43491C8D
:104330000C29F1DB2A60F0BC70472DE9F001002266
:1043400001251D4C0F2605FA02F3034217D0D3179F
:1043500002EB537C4FEAEC0304EB83031F682CF061
:10436000070CA2EB0C0C4FEA8C0C06FA0CF827EAAF
:10437000080701FA0CFC47EA0C0CC3F800C0521CF9
:104380000C2AE0DB0B498A6A22EA00008862BDE859
:10439000F001704707498A6A1043886270470548F0
:1043A000416821F080014160416821F40071416061
:1043B000704700000010004020100040704772B6A7
:1043C0004FF04020816941F040018161C16941F0B5
:1043D0004001C16162B6016A41F0010101627047AA
:1043E0004FF04020016A21F00101016272B6C169FB
:1043F00021F04001C161816921F04001816162B613
:10440000704710B572B64FF04024A06940F04000EC
:10441000A061E06940F04000E06162B6206A40F0CF
:1044200001002062D94843F63F71C16000218163D9
:104430008164C0F8D01003210A2000F0F6F90A20A8
:1044400000F016FA206A20F00100206272B6E069DE
:1044500020F04000E061A06920F04000A06162B659
:1044600010BDCA4A10605160484390607047C74A07
:1044700010605160484310F0010F18BF401C90605D
:104480007047C249C1F8D0007047C049002818BF22
:10449000012088647047BD498863C86840F0020005
:1044A000C8607047DFF8E4C2CCF82000CCF82410D4
:1044B000CCF82820CCF82C300120CCF83000DCF8E7
:1044C000340010F0010F05D020BFDCF8340010F0EC
:1044D000010FF9D110F0020018BF4FF0FF30704704
:1044E000AA48C16821F00201C1607047A748C168AD
:1044F00041F00101C1607047A44B186259629A6291
:1045000001201864586C10F0010F04D020BF586CC3
:1045100010F0010FFAD110F0060018BF4FF0FF3075
:1045200070479A48C16821F00101C16070479748FF
:10453000C16841F00401C1607047944A81891167E4
:1045400001685162416891628168D16201211165FF
:10455000516D11F0010F04D020BF516D11F0010F0A
:10456000FAD1536F0361936F1B148382936FC3F36C
:104570000523C382936F03F03F030383D36F1B14A0
:104580004383D36FC3F305238383D36F03F03F03C8
:10459000C383D2F88030C3F309430384D2F8802068
:1045A000C2F30902428411F0020018BF4FF0FF303D
:1045B00070477648C16821F00401C16070477348B4
:1045C000C16841F00401C1607047027C017B02F0C8
:1045D0003F0241EA02416D4A9165016851624168BA
:1045E00091628168D16201211165516D11F0010F55
:1045F00004D020BF516D11F0010FFAD1D36D838229
:10460000D36D1B0CC382136E0383136E1B0C438389
:10461000536E8383526EC2F30E42C28311F00200C6
:1046200018BF4FF0FF3070475848C16821F00401AF
:10463000C16070475548C16841F00801C1607047CA
:10464000DFF848C1CCF89820CCF82000CCF8243012
:10465000CCF828100120CCF89000DCF8940010F081
:10466000010F05D020BFDCF8940010F0010FF9D144
:1046700010F0060018BF4FF0FF3070474348C16884
:1046800021F00801C160704701684FEA31423F499B
:10469000C1F8BC204068C1F8C000C86840F02000E4
:1046A000C860704701684FEA31423849C1F8BC2000
:1046B0004268C1F8C020027A407A02F0010262F337
:1046C0005F00C1F8C400C86840F02000C8607047AF
:1046D0002E4B18625A6299620120C3F8B400D3F8D5
:1046E000B80010F0010F05D020BFD3F8B80010F0CB
:1046F000010FF9D110F0060018BF4FF0FF307047DE
:10470000224A106251620120C2F8B000D2F8B8000B
:1047100010F0010F05D020BFD2F8B80010F0010F43
:10472000F9D110F0060018BF4FF0FF30704717485E
:10473000C16821F02001C16070471448C16841F090
:104740001001C1607047A3F1050C104BC3F8A8C05D
:1047500018625A6299620120C3F8A000D3F8A4003D
:1047600010F0010F05D020BFD3F8A40010F0010F06
:10477000F9D110F0060018BF4FF0FF307047034822
:10478000C16821F01001C160704700000090004036
:10479000234810B5022140F8501F0121016110216A
:1047A000416241F20601416100218161042181637E
:1047B00090214163416B41F001014163C16B21F4E0
:1047C0000021C163C16B41F40051C163C16B21F091
:1047D0000101C163C16B41F00101C1634FF48171FB
:1047E00001610161032000F043F80021032000F083
:1047F0001CF8002010BD10B5032000F045F8084853
:104800004FF4807101660021016610218167022149
:104810004165002010BD034900200870704700006A
:10482000003000408C800010704700F00303DA0075
:104830004FF0FF0C0CFA02F24FF0050C0CEBC30327
:1048400001FA03F300F00C0101F1E021002807DA7E
:10485000D1F8140D90431A401043C1F8140D70475D
:10486000D1F8000490431A401043C1F80004704787
:1048700000F01F01012202FA01F14009800000F15D
:10488000E020C0F80011704700F01F01012202FA79
:1048900001F14009800000F1E020C0F8801170476C
:1048A00000F01F01012202FA01F14009800000F12D
:1048B000E020C0F8801270474FF0E021C1F80001FD
:1048C00070474FF0E021C1F8800170474FF0E020C1
:1048D000D0F8000170474FF0E021C1F88002704726
:1048E000084800687047074A11681060084670471A
:1048F000044A126800F1100352F8230042F8231012
:104900007047000008ED00E002210C20FFF78DBF8A
:1049100072B64FF04020816941F480518161C169D4
:1049200041F48051C16162B6704772B64FF04020C9
:10493000816921F480518161C16921F48051C16193
:1049400062B67047AA4881B0016F11F4007FFBD1B5
:10495000816E11F0010F1CBFD0F88410009104D0BB
:10496000D0F88410009A9142FAD0016F11F4007FC0
:1049700004BF4CF27101016642F24131816601B01F
:1049800070479B4981B04FF40D528A660A6FCA6620
:10499000012898BF012005D9401EB0F5803F28BFEF
:1049A0004FF6FF7082B24FF05C5040EA022048663A
:1049B0004FF01140C1F88000086F10F4007FFBD168
:1049C000886E10F0010F1CBFD1F88400009004D055
:1049D000D1F88400009A9042FAD0086F10F4007F5A
:1049E00004BF4CF27100086642F24130886601B0A3
:1049F00070477F4881B0016F11F4007FFBD1816E59
:104A000011F0010F1CBFD0F88410009104D0D0F831
:104A10008410009A9142FAD04FF40D51816601B092
:104A200070474FF04020806910F4805008BF7047F5
:104A30006F48806E00F0010070476D48406EC0F313
:104A40000F2070476A48D0F88400704710B50C20DA
:104A5000FFF726FF0C20FFF70BFF65490220486790
:104A600010BD634910B5032088670C20FFF70CFFC9
:104A7000BDE810400C20FFF713BF5E4A11681060BC
:104A8000084670475A4810B5016FC166594800681A
:104A9000002818BF80475848016841F480510160E0
:104AA00010BD54484068704710B572B64FF04020B2
:104AB000816941F480518161C16941F48051C161D2
:104AC00062B603204A4988670C20FFF7DDFE0C2000
:104AD000FFF7E6FE00F03CF9484B0420C3F88800DD
:104AE0004FF6FF70C3F88C0072B66033FFF749FFD2
:104AF0004FF40070186062B610BDF8B572B63C484D
:104B0000016F11F4007FFBD1816E11F0010F1CBF0A
:104B1000D0F88410009104D0D0F88410009A91420B
:104B2000FAD04FF40D51816634494FF400320A66D1
:104B300062B6D1F804124FF04025002946D02D4C22
:104B40004FF6FF73591AA1602A6BD5F834C002F0F2
:104B50000F020CF00F0C6244121D01FA02F2A2F5D2
:104B60004341DFF89CC0513961452FD2D0F8840011
:104B7000191AE160B1F5803F28D2224B4FF0000CAA
:104B8000A1FB03070CFB037301FB0C31634619F017
:104B90008DFF401C40082061B0F57A7F38BF4FF48C
:104BA0007A70194B9968002908BF98605A681A6092
:104BB0009968C3E901108A4215D9824205D9814218
:104BC00001D9616002E0606000E0626000F0D0F84E
:104BD00072B6A86920F48050A861E86920F480507A
:104BE000E86162B6F8BD8242EFD88142EBD8E8E7CF
:104BF00000C00040908000108480001000A00040A1
:104C00004F62250000E1F505388700104FF0402085
:104C1000816941F0040181610C48016841F404712B
:104C20000160001F016821F004010160016841F08A
:104C3000100101607047064908607047BFF34F8F4D
:104C4000054904480860BFF34F8FFEE714ED00E00C
:104C500008ED00E00400FA050CED00E04FF0402004
:104C6000816941F0040181610B48016841F0010153
:104C700001600B490948C1F8C40070470948006841
:104C800042F270010840704708480749016008492E
:104C900081600021C1607047144C004001005FA09A
:104CA0000060004000440040A0C00E000010004022
:104CB000508A5900022824BF00207047DC4B53F86B
:104CC000202043F820101046704770B5D94C206F53
:104CD000D74D10F0010F05D00120E06628680028AC
:104CE00018BF8047206F10F0020F08BF70BD022070
:104CF000E0666868002808BF70BDBDE870400047E6
:104D000010B572B64FF04020816941F08001816199
:104D1000C16941F08001C16162B60222C5490A65DC
:104D200001230B660323CB664A6572B6816921F0C5
:104D300080018161C16921F08001C16162B60920F1
:104D4000FFF796FD0221BDE810400920FFF76DBD79
:104D500072B64FF04020816941F080018161C169E4
:104D600041F08001C16162B60220B2490865704716
:104D7000B0490220486572B64FF04020816921F0A9
:104D800080018161C16921F08001C16162B6704713
:104D90004FF040208069C0F3C0107047A548016FF4
:104DA00011F4007F14BF4FF440714FF4807101661D
:104DB000704710B59F4CE06F10F0020F4FF00100EC
:104DC00018BF0320606700F06DF94FF040210A6BB7
:104DD000496B02F00F02D04001F00F01C8400521DD
:104DE000B0FBF1F04FF405710009C4F8801092494E
:104DF000A1FB00104009C4F88400206F10F4007F6C
:104E000014BF4FF440704FF48070206610BD894885
:104E1000016F11F4807F14BF4FF440714FF40071A3
:104E200001667047834B30B4DA6F12F0010F14BF84
:104E3000032202225A6700EB4005C5EBC010C1EB0C
:104E4000C0004FF4FA744C43C0EB001000EB40007C
:104E50007A4904EBC000A1FB00104FF04021002272
:104E60000C6B4FF0020CC008496B04F00F0401F00A
:104E70000F012144C8400521B0FBF1F0B0F5803F9F
:104E800005D3511C4008CAB2B0F5803FF9D242EABE
:104E90000C2141F01001C3F88810C3F88C00186F82
:104EA00010F4807F14BF4FF440704FF40070186608
:104EB00030BC70475F48016F11F4003F14BF4FF4DE
:104EC00040314FF48031016670475A48016F11F448
:104ED000803F14BF4FF440314FF4003101667047FA
:104EE0005448006FC0F3002070475248006FC0F371
:104EF000402070474FF040218969C1F3C01100295B
:104F000004BF002070474B4900280CBFD1F80002B5
:104F1000D1F8040270474FF040239A69C2F3C012DF
:104F2000002A04BF00207047424A00280CBFD2F874
:104F30008000D2F88800C0F30A200CBFD2F880208D
:104F4000D2F8882002F00F02D3F830C05B6B0CF06F
:104F50000F0C03F00F0363441A449140012202EB4B
:104F6000400048433449A1FB001000097047344910
:104F700001200870704770B432224FF04023514333
:104F80001A6BD3F834C002F00F020CF00F0C62441D
:104F9000121DD14008BF012104D0B1F5803F28BFC8
:104FA0004FF6FF719A69C2F3C012002A1CBF70BC91
:104FB000704772B69A6942F080029A61DA6942F0EB
:104FC0008002DA6162B602241A4A14652504156665
:104FD0004FF0040CC2F888C0C2F88C10DFF864C02F
:104FE000C2F86CC05467184902283CBF104E46F8FE
:104FF00020100021124801704FF4007111660178F1
:1050000019B920BF01780029FBD01566C2F878C015
:10501000C2F86CC0546572B6986920F0800098613F
:10502000D86920F08000D86162B670BC704700007B
:10503000A880001000A000401F85EB51CDCCCCCC47
:10504000A4800010020002021F6F00004FF0E02158
:1050500000208861086127494860704710B54FF00B
:10506000E02460610020A0610221401EFFF7DDFB0B
:1050700007202061BDE8104008F0A0BC10B508F082
:10508000A1FC4FF0E0210020086110BD10B508F030
:1050900099FC4FF0E0210020086116480188491C66
:1050A000018010BD1348806870472DE9F041114C14
:1050B000002705462780A0684FF47A71B0FBF1F015
:1050C0004FF0E026401E7061B7610221C81EFFF755
:1050D000ACFB0720306108F071FC2188A942FCD3A9
:1050E00008F070FC3761BDE8F0810349484301498D
:1050F00088607047B080001040420F004FF04020A1
:10510000816921F400518161C16921F40051C161BB
:105110007047A8490A78824218BF062828BF7047FE
:10512000A54AA64B52F830C0C3F808C002EBC00233
:105130005268DA60087070474FF04020816941F48E
:1051400000518161C16941F40051C161704710B5DE
:1051500001210720FFF769FB4FF04020816941F4EE
:1051600000518161C16941F40051C161934A00213C
:10517000116093495160DFF83CC200219CF8003077
:105180003BB10CF110031C6894605B68D3608CF831
:1051900000108C491161816921F400518161C1695C
:1051A00021F40051C16110BD8248406870478348B6
:1051B000806970474FF04020806910F4005008BFAC
:1051C00070477E48006900F0010070474FF04020B2
:1051D000806910F4005F04D0784B186910F0010F5B
:1051E00001D10020704710B472494FF6FE700024C0
:1051F0008A684AB19A69D1F808C0624504D08C60C7
:105200004C6010BC0120704700BF00BF00BF00BF52
:1052100000BF00BF00BF00BF00BF00BF00BF00BF96
:1052200000BF00BF00BF00BF00BF00BF00BF00BF86
:1052300000BF00BF00BF00BF401E0028D8DC8C604C
:105240004C6010BC002070475A498860704759482C
:10525000806870475948016941F001010161554971
:105260000120486070475548016921F00101016142
:1052700050490020486070470021002808BF4FF0C7
:10528000006103D0022808BF4FF080614B480269DB
:1052900022F04062114301617047484901200969C9
:1052A00001F04061B1F1806F04BF02207047B1F19D
:1052B000006F08BF002070474048406970473D4874
:1052C000007870474FF04020806910F4005F38D0BC
:1052D0003A4A106910F0010F33D03648406801286F
:1052E0002FD090696FF07F43984238BF00EB400C9D
:1052F00027D25169B1EB9C0F01D30120704700BF49
:1053000000BF00BF00BF00BF00BF00BF00BF00BFA5
:1053100000BF00BF00BF00BF00BF00BF00BF00BF95
:1053200000BF00BF00BF00BF00BF00BF00BF00BF85
:1053300000BF00BF00BF00BF00BF00BF00BF98425A
:10534000D7D30020704710B50720FFF7A9FA072030
:10535000FFF78EFA1948016941F01001016110BD93
:10536000164810B5016921F0100101610720FFF70F
:105370008BFABDE810400720FFF792BA0D4AD168BA
:10538000D0600846704738B50C4CE069E0610949C7
:1053900010F0020F1CBFA2698A60C96800291CBFF7
:1053A00000018847E06900900748016841F08001EA
:1053B000016038BDBC800010CC80001000D00040DF
:1053C000D0121300660F001584800010704770B56E
:1053D00005464FF40D500406A0660320E0662648FB
:1053E00060664CF2710020662448C4F8800042F2E6
:1053F0004630A06602210020FFF717FA0020FFF7D1
:1054000037FA002D08BF70BDA06E42F2413108434B
:10541000A06670BD012110B5880781674FF40D515A
:1054200081660020FFF730FABDE810400020FFF74A
:1054300037BA0120810748677047012081078867D4
:1054400070474CF271008107086670470C4A11687A
:105450001060084670470A4808B5006818B18047D0
:10546000002818BF08BD4CF2710188070166016F62
:10547000C166006F009008BD075E5F3700AF2F91D7
:10548000FC800010FE49002088717047FC4880793C
:10549000704770B5FA4C00254FF4E4612570E57053
:1054A000F84819F0F4FA4FF4E461F74819F0EFFA0C
:1054B000A56025714C21F54819F0E9FA4C21F44812
:1054C00019F0E5FA65717421F24819F0E0FA7421D7
:1054D000F14819F0DCFAE56070BDE9480079002870
:1054E00018BF01207047E6484079002818BF012006
:1054F0007047E348C078002818BF01207047E5488E
:10550000704770B5E54DE64E044601462A7830787E
:10551000E04B10444200184619F0C3FA2A7830785C
:10552000DD4B104442002146184619F0BAFAD4481F
:1055300001214171817941F00401817170BDD04830
:10554000C0687047CF4870472DE9F041CC4F804686
:105550003878002819BFD3480578D348058819BF83
:10556000D2480478D248048805FB04F6FEF727FFEA
:1055700021462846FEF775FFC2494346C24A0846FF
:10558000FEF790FFFEF72CFF72004146BE4819F06F
:1055900088FA0120F870B87940F00100B871012054
:1055A000BDE8F0812DE9F047B54D04460146287865
:1055B000DFF8D0C2DFF8EC82DFF8EC92BB4EBC4FD4
:1055C000002815BF98F80020B9F8002033783B88F0
:1055D00002FB03F04FEA4002604619F062FA2878B5
:1055E000DFF8A4C22146002815BF98F80020B9F8BA
:1055F000002033783B8802FB03F04FEA400260460C
:1056000019F04FFA0120E870A87940F00100A87164
:10561000BDE8F0879A488068704770B5A54C05468C
:10562000014622789948520019F03BFA227829461F
:105630005200974819F035FA91480121017181799A
:1056400041F00201817170BD2DE9F04FADF25C7D3A
:10565000DFF82C820120CDF8400798F80300CDF840
:105660003C0798F80400CDF8380798F805B002F028
:1056700029F80446FDF7C6F9CDF85407FDF7CBFC31
:10568000CDF85007FBF755FFCDF84C07FBF7A0FC12
:105690000646FBF79AFC0746FDF7B6F9FBF7EFFF66
:1056A0000830050998F80100002804BF0420C8F854
:1056B000140011D002F01EF88146022C1CBF0920F4
:1056C000C8F8140012D0B9F1060F04BF0220C8F8C0
:1056D0001400002088F80100FBF77AFC10F0010F9D
:1056E00015D002F081F93C280BD010E013F097FCA4
:1056F00048F20211084214BF3C201E20C8F81400D2
:10570000E1E7FFF757FD002818BFFFF7DBFD4FF07B
:105710000109022F14D102F0F8F888B9022C04D044
:10572000052C08BF052007D00AE04FF47A706843C3
:105730004FF47A7190FBF1F0C8F8140088F80190EA
:10574000D8F814000428BCBF0420C8F8140098F846
:105750000100B8F81410000240EA014040F00102D4
:105760000023912107200CF001F816F0010F25D13C
:10577000022C23D00020FBF7E1FEFDF78BFC002676
:10578000B24606F0F9FF01281ED00DF5E460FDF7E2
:1057900057FF002800F016820DF5E46007F02EFF99
:1057A000D8F81400C01EB042ACBF01250025DDF8BA
:1057B0002C0748B3DDF8380750B144E0FDF731FC61
:1057C0000020CDF84007DAE74FF0010A00F0E4B915
:1057D0006846DDF82C1719F06EF90746ADB1354C67
:1057E000394620784200294819F05BF9207839467B
:1057F0004200274819F055F988F8049098F80600F7
:1058000040F0020088F806001DE0FEF7D8FD294CA4
:1058100001212078FEF725FE1D4A3B46A2F14C01EE
:105820000846FEF73FFEFEF7DBFD207839464200D2
:10583000174819F036F988F8049098F8060040F0F7
:10584000020088F80600DDF82807002800F00F8124
:10585000DDF83C07002840F00A8198F80000DDF8E8
:10586000284700287ED1D8F8087047B10D48007845
:10587000CDF848070D480078CDF844071CE038E023
:10588000008100104422011044870010A49C0010E5
:10589000F09C0010642901103C9D00105381001001
:1058A000548100104F81001056810010508100106B
:1058B0005881001055810010FEF781FDDDF8441776
:1058C000DDF84807FEF7D3FD21463A460846FEF7C5
:1058D00013FEFEF785FDFA480078022804BF38461B
:1058E00007F0F6FAF6480078092804BF204607F0CA
:1058F000EFFAF4480078012811D9F14F38780428DC
:1059000004BF204607F0E4FA2146684619F0D8F8AB
:1059100004463878052804BF204607F0D9FA01F07C
:10592000F4FFF8B101F0CEFE022820D10DF05EF8B0
:1059300018B113F0E6FB082819D1E34800220378D8
:10594000E2480778002F12D90020002B0CD902FB67
:105950000301401C34F911C083424FEAEC0C24F8D7
:1059600011C000E003E0F2D8521CBA42ECD3D84890
:10597000007868B9D5480278D3480178204619F0F4
:10598000A4F8CF480078332804BF204607F0A0FAD7
:105990009DB3D04898F800202146002A07BFCE4A80
:1059A0001288CE4A127819BFCD4B1B78CD4B1B887D
:1059B00002FB03F24FEA420219F073F898F8000074
:1059C000C94B2146002819BFC4480078C248008846
:1059D00019BFC34A1278C34A128800FB02F04FEA8B
:1059E0004002184619F05DF888F8039098F8060010
:1059F00040F0010088F8060032E0FFE7CDF84447A8
:105A000098F80000002819BFB4480778B248078802
:105A100019BFB3480478B348048807FB04F0CDF8F5
:105A20004807FEF7CCFC21463846FEF71AFDA94987
:105A3000AD4A0846DDF84437FEF734FDFEF7D0FCEA
:105A4000DDF84807DDF844174200A74819F029F8A7
:105A500088F8039098F8060040F0010088F80600E6
:105A600097480078032804BF9A4807F031FADDF818
:105A7000300700287ED0BBF1000F7BD1044698F898
:105A8000000038BBD8F80C7027B3984801789848C4
:105A900000780844401C4008019002200090FEF766
:105AA0008EFCDDE90010FEF7E2FC21463A4608468E
:105AB000FEF722FDFEF794FC8E480078022804BF12
:105AC000384607F027FC8B480078092804BF204699
:105AD00007F020FC7E48007868B97B4801787B4855
:105AE0000278204618F0F6FF82480078332804BF79
:105AF000204607F00FFCD5B17F48804D804F2146EE
:105B00002B783A781A44520018F0CBFF2A783B7869
:105B10007C481A442146520018F0C3FF88F80590CB
:105B200098F8060040F0040088F8060021E0734869
:105B300025460178724800780C18FEF740FC601C7E
:105B400040080221FEF78DFC6B492B466D4A084642
:105B5000FEF7A8FCFEF744FC62002946694818F0ED
:105B6000A0FF88F8059098F8060040F0040088F837
:105B7000060000E006E05F480078032804BF5E48A6
:105B800007F0C8FBFDF7B3FDD8F81400761CB0424F
:105B900011DCD8F8100070B1FCF736FFDDF84C07C7
:105BA000FBF7CCFCDDF8540788B1DDF8500760B195
:105BB000FDF770FA0BE0DDF84007002818BFFDF78D
:105BC00069FADEE501F0D5FDDBE5FDF72AFABAF169
:105BD000000F04BF0420C8F8140009D0DDF83C070A
:105BE00088F80300DDF8380788F8040088F805B065
:105BF000B8F814104FEA0A2040EA0142002391212C
:105C000007200BF0B3FD0DF25C7D5046BDE8F08F30
:105C100010B50024FDF7F1F93B4910F0070F0AD049
:105C2000CA78002A08BF012410F0020F03D00A79B5
:105C3000002A08BF012410F0F00F03D04879002893
:105C400008BF01240020002C08BF10BD00200870F0
:105C5000BDE81040F8E408B540F20F3101F0F1FE64
:105C6000012804D1FFF7D4FF009002F088F82648FD
:105C7000C17800291CBF4179002904D0007900288F
:105C80001CBF012008BD002008BD08B540F20F313F
:105C900001F0D7FE012804D1FFF7BAFF009002F00F
:105CA0006EF81948C17800291CBF4179002904D039
:105CB000007900281CBF012008BD002008BD00009D
:105CC000E58100104E8100104C8100104D810010C4
:105CD000C4ED001044220110568100104F810010C5
:105CE000508100105881001044870010518100102D
:105CF00052810010EA8100106429011053810010C4
:105D0000548100103C9D0010008100107047FE4936
:105D100010B50022CA700A714A7100281CBF012008
:105D200048700CF076FDBDE81040FAF75CBB10B58A
:105D30004FF4E461F54818F0AAFEBDE810404FF4B6
:105D4000E461F34818F0A3BEF2487047F2480188B6
:105D5000F248008848434100EE4818F098BE70B5FC
:105D60000646ED480488ED480588FEF728FB2946DD
:105D70002046FEF77CFBE54A3146E648FEF7BCFBD1
:105D8000FEF72EFBE6480078152818BF70BDE148E5
:105D9000BDE8704007F09CB870B50446DE48058841
:105DA000DE480688FEF70BFB31462846FEF75FFB10
:105DB0002246D6491046FEF79FFBFEF711FBD84856
:105DC0000078162804BF204607F082F8204670BDF0
:105DD000002818BF0120CC49C870704710B5CA4CC4
:105DE000002804BFA06010BDDFF838C3CE490B788F
:105DF000CE490A7801465A435200604618F051FED7
:105E0000C848A06010BD10B54C21C94818F03FFE2D
:105E1000BDE810404C21C74818F039BEC44870474F
:105E2000002818BF0120B8490871704710B57421C7
:105E3000C14818F02CFEBDE810407421BF4818F08E
:105E400026BE002818BF0120AF494871704710B521
:105E5000AD4C002804BFE06010BD74220146B84874
:105E600018F01FFEB648E06010BD70B5A64D0021C9
:105E70000446E970297169710CF0CBFCFAF7B3FAAA
:105E8000002C14BF012000202870BDE87040FFF7EF
:105E9000DBBB2DE9F04F89B04FF4E461A14818F065
:105EA000F6FD7421A64818F0F2FDFDF7A6F80446A9
:105EB000FCF7A8FD0890FDF7AEF80790FBF739FB5B
:105EC0000690FCF7A1FDFBF783F810F0010F0BD053
:105ED00001F08AFD3C2807D1FFF76CF920B10420BE
:105EE000FFF717F9FFF7EEF90020FBF727FBFDF7A7
:105EF000D1F800252E4606F03FFC012853D0684615
:105F0000FDF79EFB00285ED0684607F077FB14F093
:105F1000070F1CD08448DFF80CB2DDF8089090F829
:105F200000808248DA460778FEF749FA0120FEF73A
:105F3000ACFA39464046FEF79AFA52464946584668
:105F4000FEF7DAFA0020FEF7A0FAFEF749FA14F09D
:105F5000F00F20D07B48DFF8E8B1022701787A48BB
:105F6000DA46DDF8109000780844401C4FEA5008EB
:105F7000FEF725FA0120FEF788FA39464046FEF77B
:105F800076FA524649465846FEF7B6FA0020FEF722
:105F90007CFAFEF725FAFDF7AAFB6D1C102D03D243
:105FA000FDF778F8A7E701260520FFF7B2F8FCF720
:105FB0002BFD0698FBF7C2FA089848B1079828B15C
:105FC000FDF768F804E001F0D4FB94E7FDF729F849
:105FD000DEBB4D4F14F0070F1BD05348DFF844C110
:105FE00001785248E046007801FB00F210200021C1
:105FF000002A88BF03460AD938F9115005EB50052D
:10600000B5FBF3F52CF81150491C8A42F4D84548E9
:10601000B86014F0F00F18D04A48494B01784A484C
:106020001C4600780A184FF010014FF000000AD00B
:1060300034F9105005EB5105B5FBF1FC23F810C005
:10604000401C8242F4D83E48F86009B03046BDE8B2
:10605000F08F012070474FF47B3070474FF47B3056
:1060600000687047034600209A682C2A88BF2C22BB
:106070000021B1EB920F28BF704753F821C0491C93
:106080006044B1EB920FF8D37047304A01689142F7
:1060900014D14168B1F5807F10D9836800222C2B80
:1060A00088BF2C230021B1EB930F09D250F821C0F7
:1060B000491C6244B1EB930FF8D30AB1002070473A
:1060C000012070474FF47B31204B0A689A4263D11C
:1060D00091F827300022012B08BF0122052804BFB8
:1060E00091F82300704738DC012804BF087F70470F
:1060F000022804BF91F820007047032804BF91F8DC
:1061000021007047042823E0008100104422011080
:1061100044870010648E00105681001058810010D2
:10612000E5810010849500104F810010508100100F
:10613000A49C0010F09C0010642901103C9D0010EC
:10614000B09D001051810010528100104353494D01
:1061500004BF91F82200704731E0142808D01528B8
:106160000CD0162811D0172804BF1846704726E017
:10617000002A1CBF91F82400704704E0002A1CBFCD
:1061800091F8250070472D207047002A1CBF91F818
:106190002600704728207047052812D007DC012808
:1061A0000DD002281CBF032804280AD007E01428B9
:1061B00018BF1528E7D01628ECD0172801D0FF20EB
:1061C0007047002070472DE9F047ADF5007D0024B1
:1061D0004FF40071684618F05AFCFF20A04660F3A7
:1061E00007082D20254660F3070560F30F252820BA
:1061F00060F317454FF47B37F74E64F31F654FF498
:1062000081794FF02C0AFF224FF40071684618F094
:1062100066FCCDE902A4CDE9064805940A94CDE9CF
:1062200000690494CDE908453846FDF7EBFE694660
:106230003846FDF789FF012818BF00200DF5007DC5
:10624000BDE8F0872DE9F047ADF50C7D89460546A0
:106250001F4690464FF0000A4FF400716846949E26
:1062600018F015FC4FF0000CCDF800C24FF47B3451
:10627000CDF804C2CDF808C2CDF80CC2CDF810C2DA
:10628000CDF814C2CDF818C2CDF81CC2CDF820C28A
:10629000CDF824C2CDF828C2CF492068884206D064
:1062A000FFF791FF0DF50C7D5046BDE8F087D4E96E
:1062B00001120DF5007AE3688AE80F0004F110017D
:1062C0000DF5047A0FC98AE80F00D4E90801A26A23
:1062D0008A92CDE9880184988DF820928DF82182E8
:1062E000401C8DF822728DF81C528DF82362849028
:1062F000002D14BF8698859800F1010014BF869088
:10630000859080AB82980021CDF80CC22C2894BFD8
:1063100002462C220020B0EB920F06D253F820C088
:10632000401C6144B0EB920FF8D348428390FF22A7
:106330004FF40071684618F0D2FB80AC94E80F006F
:106340008DE80F0084AC94E80F0004AC84E80F00E3
:10635000DDE988018A9A4FF47B34CDE908010A927D
:106360002046FDF74FFE69462046FDF7EDFE012869
:1063700018BF00200DF50C7DBDE8F0872DE9F04138
:10638000ADF50C7D0F46804616464FF40071684609
:1063900018F07DFB002580954FF47B348195829524
:1063A00083958495859586958795889589958A9511
:1063B00089492068884218D16068B0F5807F14D977
:1063C000A06821464FF0000C2C2888BF2C20002309
:1063D000B3EB900F11D251F823205B1C9444B3EB24
:1063E000900FF8D3BCF1000F07D0FFF7ECFE0028A8
:1063F00004BF0DF50C7DBDE8F0810FCC0DF5007CE0
:106400008CE80F000FCC0DF5047C8CE80F00D4E96C
:106410000001A2688A92CDE988018DF824828DF866
:1064200025728DF8266201208DF8270282980021BE
:1064300080AB83952C2894BF02462C220020B0EB21
:10644000920F06D253F820C0401C6144B0EB920F6B
:10645000F8D348428390FF224FF40071684618F049
:106460003EFB80AC94E80F008DE80F0084AC94E80C
:106470000F0004AC84E80F00DDE988018A9A4FF42C
:106480007B34CDE908010A922046FDF7BBFD694641
:106490002046FDF759FE012818BF00200DF50C7DA0
:1064A000BDE8F0812DE9F04F4C4D4FF0000885B06C
:1064B0006C42474646461720FFF704FE4FF47B32F6
:1064C000844645491068884217D15068B0F5807FEE
:1064D00013D9936800212C2B88BF2C230020B0EB0C
:1064E000930F80F0FF8052F82090401C4944B0EB9D
:1064F000930FF8D3002900F0F580FFF764FE002821
:1065000004BF05B0BDE8F08F1420FFF7DBFD02905B
:106510001520FFF7D7FD00901620FFF7D3FD40B2FE
:1065200001901620FFF7CEFD404240B20390FCF7E9
:1065300064FDDFF8AC908246002089F8030089F8FA
:10654000040089F805000CF064F9F9F74CFF00200D
:1065500089F80000FFF778F81AF0F00F05D018F06E
:10656000C3FA012808BF48F001081AF0070F7DD0D0
:106570001C481E4A0026B0F800E01B48038899F822
:106580000200A3EB000984468145C4BFAEEB0C01B9
:10659000A1F1010B1CDD61468B4516DD01F1010AFD
:1065A00001FB03070AFB030A32F8177032F81AA03E
:1065B000A7EB0A073FB2002FB8BF7F423FB2B742F6
:1065C000C8BFBEB2491C8B45E8DC401C8145E2DCFB
:1065D000009800280CE000004353494DF1D8FFFF1C
:1065E00000810010588100105681001044220110D3
:1065F00018BF864288BF48F002080027E246AEEB8B
:106600000A0000905045C8BFA9F1010B1BDD604690
:10661000834513DD0AFB030132F811E002EB41016F
:106620004988AEEB010109B20029B8BF494209B25D
:10663000B942C8BF8FB2401C8345EBDC00980AF119
:10664000010A5045E3DC0298002818BF874288BF42
:1066500048F00408E2460098504516DD6146894539
:106660000EDD0AFB031032F9100000E017E0A8422B
:10667000C8BF0546A042B8BF0446491C8945F0DCA6
:1066800000980AF1010A5045E8DC0198002806DD6F
:10669000854202DC0398844201DA48F00808FF2FA3
:1066A00088BFFF27FF2E88BFFF267F2DC8BF7F250D
:1066B00004DC15F1800FB8BF6FF07F057F2CC8BFD9
:1066C0007F2404DC14F1800FB8BF6FF07F04E0B2C8
:1066D0000090EBB2F2B2F9B24046FFF7B3FD05B05D
:1066E000BDE8F08FBCF1000F18BFBCF1010F3FF403
:1066F0000BAF02E7FE49002008627047FC49887032
:106700007047FB4890F902007047F94800787047DD
:10671000F74840787047F6480021C17141714172D5
:106720008172C1727047F24920F07E40C8617047A3
:10673000EF48C0697047EE48408A7047EC48808A4D
:106740007047EB48B0F916007047E948B0F91800F7
:106750007047E748B0F91A007047E548007B70477A
:10676000E348C078002818BF0120704710B54FF4E7
:10677000E461E04818F08BF9DD490020C87010BDD5
:106780002DE9F74F90B000250C46DB4901950295A5
:10679000039504950595069507950895099508684C
:1067A0001746052A08BFB0F97A6005D0062F0CBF3E
:1067B000B0F97860B0F97660B0F97400B0420ADAE6
:1067C00012F02DFC48F20211084203D0CA480068BA
:1067D000B0F8746036B20023324601A9109818F060
:1067E00088F9059800B22080BDF826106182BDF8B6
:1067F0001E106181BDF82010A181BDF82210E18139
:10680000BDF824102182BDF81810A180BDF81A101F
:10681000E180BDF81C1021810028B8BF25808DF8CB
:106820002850B648B64900888DF82A008DF82950BE
:1068300009788DF82B107142ADF82E10ADF83000AC
:1068400080B2ADF82C60ADF80000DDE90A232146E6
:10685000109800F0B0FC052F11D0E582A5822583A9
:10686000A088002804BF4FF40040A0806089002861
:1068700004BF47F6FF70608113B0BDE8F08FFEF7EC
:1068800061FE002118F03AF9002800F0F180DDF8EF
:1068900028C0DDE90B0ACCF3072310994FEA1C62EC
:1068A000ADF80050ADF8345099469A4269D91FFAB4
:1068B0008AF50CF0FF0603FB056E1FFA8EF80E95A5
:1068C00031F91880BDF80060BDF834500FFA80FB34
:1068D000D845C4BF761CB6B24FEA204BD845BCBFE2
:1068E0006D1CADB2ADF800600EF101081FFA88F81A
:1068F000ADF8345031F918800FFA80FBD845C4BF89
:10690000761CB6B24FEA204BD845BCBF6D1CADB269
:10691000ADF80060DDF83880CCF3074B03FB08BE10
:10692000AEF102081FFA88F8ADF8345031F918803A
:106930000FFA80FBD845C4BF761CB6B24FEA204B95
:10694000D845BCBF6D1CADB2ADF80060AEF101081A
:106950001FFA88F8ADF8345031F918800FFA80FB2F
:10696000D845C4BF761CB6B24FEA204BD845BCBF51
:106970006D1CADB2ADF800605B1CADF834509A42AE
:1069800095D80CF0FF03CCF3074E9E456CD91FFA47
:106990008AF609FB063C1FFA8CF8BDF800C031F9F5
:1069A00018800FFA80FBADB2D845C4BF0CF1010CC2
:1069B0001FFA8CFC4FEA204BD845BCBF6D1CADB212
:1069C000ADF800C009F1010808FB06381FFA88F885
:1069D000ADF8345031F918800FFA80FBD845C4BFA8
:1069E0000CF1010C1FFA8CFC4FEA204BD845BCBFC0
:1069F0006D1CADB2ADF800C0A2F1020808FB06386C
:106A00001FFA88F8ADF8345031F918800FFA80FB7E
:106A1000D845C4BF0CF1010C1FFA8CFC4FEA204B87
:106A2000D845BCBF6D1CADB2ADF800C0A2F10108E5
:106A300008FB0636B6B2ADF8345031F916600FFADD
:106A400080F84645C4BF0CF1010C1FFA8CFC4FEADC
:106A500020484645BCBF6D1CADB2ADF800C05B1C04
:106A6000ADF834509E4592D8E582BDF80000A08272
:106A7000DDF830900A9E109D4FF0000C052F4DD090
:106A80001D48062F006803BFB0F87810022738466B
:106A9000B0F876101CBF01270020B4F90230B4F919
:106AA0000020934241D18A423FDDC6F307210144D1
:106AB000C0EB166A8A452ED9C6F30742F0B2D21B44
:106AC0003844A2F10108804522D91FFA89F201FB5E
:106AD000020292B235F9123005EB4202B2F90220FD
:106AE000B3EB020B48BFA2EB030B0FFA8BF209E0EA
:106AF00018810010249E00102C8300105881001073
:106B0000568100106245C8BF9446401C8045DCD8C1
:106B1000491C8A45D0D8A4F818C0A1E6FE4802272F
:106B20000068B0F87A103846B7E7228398E6084341
:106B300018BF7047F948C16911F0807F08BF7047DE
:106B4000F5490968096F11F4003F08BF704700213B
:106B50001170182101827047F048406A70472DE992
:106B6000FF5FEF480027DDF83CA005880E98119ED6
:106B70008B46B9463C4650452CD006FB050E109876
:106B80003BF91EC006FB05093BF91900BCEB0001EF
:106B900048BFA0EB0C0106FB05A83BF91840B4EB7D
:106BA000000C48BFA0EB040C01EB0C0004B232F95E
:106BB0001EC032F91900BCEB000148BFA0EB0C016C
:106BC00032F918C0BCEB000248BFA0EB0C028818D9
:106BD0000FFA80F9012B37D04FF0010817F093FF1F
:106BE000D049002C0A7807DD109906FB05113BF906
:106BF00011101431282909D80099B1F914103C2931
:106C000004DC0099B1F916103C2926DD0E9902EB3F
:106C10000A0C11448C4520D9129B139D13442A441D
:106C20008B421CBF8D1A15F1020F30F9115000EB89
:106C30004106B6F90260A5EB060508D01E353C2DCD
:106C400008D94FF0000808E0A1450CDD0AE00A353C
:106C5000142DF6D8491C8C45E2D8A14503DDB8F1C6
:106C6000000F00D0012704B03846BDE8F09F704700
:106C7000AA48B0F90E007047A8490020C8817047A3
:106C80000021018041804FF400428280C180018157
:106C9000521E42818181C181018241828182C182F1
:106CA000018370479D4902281CBF80208870002006
:106CB0000862704770B5994E04460D46706A84426A
:106CC00006D044EA052200236B2107200AF04EFD7E
:106CD0000CB1746270BD022D1CBF8020B07000200A
:106CE0003062F6E72DE9F0418846054612F07FF95B
:106CF000044612F078F904FB00F1884E22180024B3
:106D000096F9020009B210F1800F274618BF0A2831
:106D10001BDAB6F91A003239814211DA0124B8F1CE
:106D2000000F12D10021002A0FD935F91100B0F55A
:106D3000487F01DA002403E0491C9142F5D324B9CD
:106D400010F02EFE012808BF0124706A012808BF38
:106D5000002C16D1306A4EF6C42188420BD200F0C6
:106D6000B7FC0021022819D0042808BF4FF4FA719B
:106D7000306A084430624EF66021814228BF012407
:106D800000D23762706A844206D044F480720023D5
:106D90006B2107200AF0EAFC54B906E00BF036FD3F
:106DA000002814BF11210821E2E78020B07037626B
:106DB0007462BDE8F0812DE9FF4F8BB0574DDDE9DE
:106DC00018A704460020287068700BF033FD0028D7
:106DD00040F0448100F076FC052871D0287B0190BA
:106DE00051494D48DDF8309091F800B000684D49A8
:106DF00090F8866009780091B0F98480B5F91800A0
:106E00003228688A05DA002804BF7006060E04D10D
:106E100000E010B9287901282BD10BF04DFD40BBC3
:106E2000012F26D0BAF1010F02D1A88AC82820D894
:106E3000A88A002804BF688A00281AD00BF0E6FC54
:106E4000012819D0B9F80000E881009900201BEB57
:106E500001030AD039F91010B5F90E209142C8BFCC
:106E6000E981401C80B28342F4D8B5F90E00404558
:106E70000EDD0020A87223E02748006890F88760A4
:106E80000198012814BF4FF03C084FF04108D9E7A2
:106E9000E86910F4803F13D01F480068006F10F4B9
:106EA000803F0DD0A87A401CC0B2A872B04207D96A
:106EB000102028820120287200204FF0FF34A87291
:106EC00010F06EFDA0B100F003FC042810D1287F63
:106ED00010F0800F0CD01048006890F8700010F08F
:106EE000800F05D00720288201204FF0FF34287240
:106EF0000BF08CFC01287CD10748BAF1000F006828
:106F00000A9090F8881076DC012F74D0E86910F4AC
:106F1000003F1DD00A9809E02C8300101881001052
:106F2000568100105481001053810010006F10F43E
:106F3000003F0DD0687A401CC0B26872884207D901
:106F4000112028820120287200204FF0FF3468723F
:106F50000C980090FE484FF0000B012F0078039032
:106F6000FC48007801900A9890F88700069045D078
:106F70000198400807900398400809900020049069
:106F800082460590DDE9001001EB400002900023ED
:106F90001A461946BAF1000F0CBFDDE90076DDE9AB
:106FA00002760020002E88BFA6F1010E29D937F9FC
:106FB0001080B8F1640FD8BF002214DD70450DD2E7
:106FC00007EB400CBCF902C0B8EB0C0948BFACEBB6
:106FD00008090FFA89FCDC45A8BFE346491C002AD2
:106FE00004BF01225B1C401C8642E0D8012B05D85F
:106FF00007E033E0FFE700206872A9E70020E872AD
:107000002CE0BAF1000F0CBF049105910AF1010ABE
:10701000BAF1020FBBD3079904988842EED90999B7
:1070200005988842EAD9BBF1320FE7DCE87A401CC8
:10703000C0B2E872E96911F4801F0FD00A99096F94
:1070400011F4801F1CBF0699884207D9142028829A
:107050000120287200204FF0FF34E87211F0DFFFAA
:1070600010F4014F28D000F02DFB022824D14FF05E
:10707000010817F04DFD074611F0B9FF064611F063
:10708000B2FF024600210020002E08D900FB0213A7
:1070900037F913300F2B0FDB401CB042F6D3B8F199
:1070A000000F09D0491C0129EDD9B8F1000F03D018
:1070B00001204FF0FF3428720EF0D7FC032823D1B3
:1070C000002000900190287C8DF80000BDF80000A1
:1070D000022264F30F20ADF80000E979BDF8020048
:1070E00061F30300697961F30710297A61F30820DD
:1070F000A97961F34920ADF80200E889ADF80400F0
:10710000062168460EF0B4FCB4F1FF3F26D0002CF7
:1071100007BFA87901280FB0BDE8F08FFEF716FE73
:107120000024AC71012028704FF4E4618A4817F004
:10713000AEFCEC7000F0CCFA04280D982CD000289E
:1071400018BFFEF72FFA0E98002804BF0FB0BDE855
:10715000F08F0FB0BDE8F04FFEF7D3B9287A0128C1
:107160001CBF0FB0BDE8F08F0D98FEF7F8FD0024AE
:107170002C72012068704FF4E461774817F087FCA7
:10718000EC700D98002818BFFEF70CFA0E98002836
:10719000DFD10FB0BDE8F08F002818BFFEF7D4F99B
:1071A0000E98002804BF0FB0BDE8F08F0FB0BDE807
:1071B000F04F17F0B2BC2DE9F8070023DDF820C02E
:1071C000C2F30724ADF80030160E2546D3B21FFADD
:1071D0008CFCC2F30747A64259D904FB0C381FFAAE
:1071E00088F230F9129000EB4202B2F902A0B9EB3A
:1071F0000A0248BFAAEB090212B2BDF900909145FC
:10720000B8BFADF8002008F1010292B230F9129037
:1072100000EB4202B2F90280B9EB080248BFA8EBCA
:10722000090212B2BDF900809045B8BFADF8002048
:1072300004FB0C78A8F1030292B230F9129000EB33
:107240004202B2F902A0B9EB0A0248BFAAEB090256
:1072500012B2BDF900909145B8BFADF80020A8F179
:10726000020292B230F9128000EB4202B2F90290AF
:10727000B8EB090248BFA9EB080212B2BDF90080C1
:107280009045B8BFADF80020641CA642A5D8A7F170
:107290000108984559D96F1CB41E761E05FB0C32A7
:1072A00092B230F9129000EB4202B2F902A0B9EBAF
:1072B0000A0248BFAAEB090212B2BDF9009091453B
:1072C000B8BFADF8002007FB0C3292B230F9129033
:1072D00000EB4202B2F902A0B9EB0A0248BFAAEBE6
:1072E000090212B2BDF900909145B8BFADF8002077
:1072F00004FB0C3292B230F9129000EB4202B2F968
:1073000002A0B9EB0A0248BFAAEB090212B2BDF90A
:1073100000909145B8BFADF8002006FB0C3292B248
:1073200030F9129000EB4202B2F902A0B9EB0A0266
:1073300048BFAAEB090212B2BDF900909145B8BF4F
:10734000ADF800205B1C9845A8D8BDF8000005E00A
:107350005381001054810010249E00104880BDE825
:10736000F80770472DE9FF4FDFF81483074689B00F
:10737000D8F800009946B0F878A011F00EFA01286C
:1073800004BF4FF6FF7000EA4A0ABE4CBE4D3846B5
:107390002288298817F0C6FB11F041FE48F2021638
:1073A000304207D0B9F9141001233846169A17F065
:1073B000BEFB04E0012238461699FFF7E1F9B24816
:1073C0000288B0480188384617F0ACFBAF4F002464
:1073D00025463C71FEF7B6F800940194029403949C
:1073E00004940594069407940894A54C01232168FD
:1073F000B1F87620694617F07CFB2168BDF91A00C8
:10740000B1F9761049428842B8BF0125BDF8200085
:10741000B0F5FA7F88BF01259C48057111F0FFFD8A
:1074200048F2021108420DD11698B0F91200002856
:1074300008DC0BF0EBF9012804D09448007901280E
:1074400040F0DA808F4802888F4801880B9817F047
:1074500069FB11F0E4FD48F2021B10EA0B0F00F08B
:10746000BC8047F6FF70039086480B9E4FF00009E2
:1074700007888548179C4D460088019011F0CFFD84
:1074800010EA0B0F0FBF50467D480068B0F874003B
:107490000FFA80F811F0C3FD10EA0B0F1FBF7848F8
:1074A0000068B0F87400404208BFCAF1000000B2A2
:1074B000029011F0B4FD10F4807F4FF0000B14BF68
:1074C0004FF0210CBC46002000900398804568DAFC
:1074D000DDE9002000287CD9ACF10100059001987D
:1074E000401E0490ACF1020003905846E34538BFBB
:1074F00013B251D202FB070A1FFA8AF136F91110B2
:107500000029B4BFC1F1000E8E46C6451ADD4145C3
:107510000BDDB4F904E0714502DDA180E380208138
:1075200009F101010FFA81F90CE0DDF808E08E4560
:1075300008DDB4F90AE08E4502DD6181A381E081B6
:10754000691C0DB20599884223D206EB4A0136F92F
:107550001AE0B1F902A0BEEB0A0148BFAAEB0E0186
:1075600009B2DDF800A052451CBFDDF810A052455D
:1075700005D058451CBFDDF80CA0504504D1B4F926
:1075800002A08A45B8BF6180B4F900A08A45B8BF9F
:107590002180401C6045ADD30198521C8242A4D387
:1075A00017E0DDE90001002913D95B46E3450CD261
:1075B00000FB073189B236F9112002998A42BCBF1B
:1075C000691C0DB25B1C6345F2D30199401C8842D3
:1075D000EBD3A4F81090658204E0062217990B986B
:1075E000FFF7CEF828480288264801880B9817F044
:1075F00099FA1999012008701798B0F9100000281D
:1076000008DC1798B0F91200002803DC1F48007945
:10761000012821D11B4C1C4D0A982288298817F07B
:1076200081FA11F0FCFC48F20211084207D0052350
:1076300047F6FF71189A0A9817F079FA04E00522C4
:1076400018990A98FFF79CF82A8821880A9817F059
:1076500069FA1A99012008701698418A0B484182EC
:107660001699098A818216994989C1821699898851
:1076700001831899098A41830DB0BDE8F08F00009D
:107680002C830010588100105681001018810010C2
:1076900010B50AF0AFFE0AF09AFF002010BD0000FE
:1076A000FE49C8707047FD48C0787047FB490871B3
:1076B0007047FA4800797047401E022894BF0120A5
:1076C00000207047F54800787047F448807870478C
:1076D000F2480078022805D005281CBF002070471A
:1076E00006F0EBBA0BF075B8EC4908707047EB493F
:1076F00048707047E9484078704770B5E74E0446D7
:107700000D463078A04212D002281ED0052814BFA2
:10771000002006F0D2FA44EA05213278002341EA3B
:10772000024141EA0062612107200AF01FF8307827
:10773000844218BF7070B570072C28BF70BDDFE899
:1077400004F016070B13160F16000BF042F8E2E7D1
:10775000284600F027FB0AE028460BF0E5F806E093
:10776000284606F09FFA02E028460AF0F1F8347045
:1077700070BDCB4900200968B1F8B01011F4807FCA
:1077800008BF7047FCF759BBC54900200968B1F82C
:10779000B01011F4807F08BF7047FCF75DBBC04993
:1077A00000200968B1F8B01011F4007F08BF7047DD
:1077B00017F0C2B9B949487900281CBF401E48716A
:1077C000704770B5B7480068B44C10F0130F0FD075
:1077D00010F0100F05D0B44951F88C2F42F48052AC
:1077E0000A60B24908606079002804BF0120607116
:1077F0004FF040208069AA4D10F0020F296806D191
:10780000AB48006810F0010F01D0607940B1B1F8C9
:10781000B010002011F4807F18BFFCF71DFB07E0BB
:10782000B1F8B010002011F4806F18BF17F089F97B
:10783000A049084208BF70BD2968D1F8B010090CF2
:10784000617170BD10B572B6FDF7E4FDBDE8104082
:10785000FDF7F4B910B5012802D0022805D007E0E1
:107860004FF47F30FCF7CEFB02E094499248086069
:1078700072B6FDF7CFFDBDE81040FDF7DFB98749CF
:1078800000288A7918BF01208871C0B2824208BFDF
:1078900070470022002818BF012200230121022086
:1078A00009F064BF7D488079002818BF0120704727
:1078B0007A4AD179814208BF704710720120507214
:1078C00070477648007A7047744948727047734829
:1078D000407A704770B5714C0028E57918BF0120D7
:1078E000E071C0B2F8F75EFDE079854214BF002870
:1078F00070BD247817F02AF9022C1CBF052C70BD2E
:1079000002212046BDE87040F7E610B511F087FB74
:1079100048F2021108421CBF002010BD5F48C07928
:10792000002818BF012010BD00285C4918BF0120A5
:107930008872704710B511F072FB48F202110842CC
:107940001CBF002010BD5548807A002818BF0120B8
:1079500010BD5248C07A70472DE9F0414F4D0028C4
:107960001CBF0020E87204D1E87A002818BFBDE8E7
:10797000F081534E37683020FCF7C6FC06213020DA
:10798000FCF7DBFCF06A40F03000F0624D4C4FF049
:107990007F0811E0FDF755FDF06A10F0100F03D0DD
:1079A000E87A40F07E00E872F06A10F0200F03D011
:1079B000E87A40F00100E872201EA4F1010403DD22
:1079C000E87A38EA0000E5D13020FCF7E3FC3760C4
:1079D000BDE8F081314AD082118370472F48006A98
:1079E00070472E48C06970472C48C069002818BFEE
:1079F000C07A70472949486270472848406A7047F2
:107A00002649886270472548806A70472448026882
:107A100002F5C873118A508A02F5A872FBF713BCED
:107A200010B506F06EFE002818BFC07A10BD10B564
:107A300006F067FE00280CBF4FF0FF3090F92400DD
:107A400010BD2DE9F04FDFF854A099B00E46CAF8EA
:107A5000200006F056FECAF81C00002800F0E48062
:107A600005788AF80C5041788AF80D10837804461E
:107A7000681C8AF80E3000F0FE008AF80F00E278E9
:107A80008AF8102094F804C08AF811C060798AF846
:107A9000120040008AF8130016E000004081001038
:107AA0002C8300101848004000300040144800406B
:107AB000144C004008001300AD2007B0304C0040CB
:107AC00000100040803801004FEA5C008AF8140082
:107AD0000AF11A004FF0000B80F800B080F801B0F6
:107AE00020788AF815002846FBF776FD9AF81210E0
:107AF0009AF81100FBF793FD6946204606F01FFE39
:107B0000E089DAF8245000281CBF6843050BB4F85C
:107B10001280DAF82890B8F1000F08BF4FF48058AF
:107B2000E78A002F08BF4FF480574FF48050189019
:107B3000002016F0040F18BF052016F0080F18BF1C
:107B400040F0020016F0020F18BF40F0F00016F0EF
:107B5000010F18BF40F4774016F4807F18BF40F43F
:107B6000803016F4007F18BF40F47E00E16901EA1E
:107B7000000600981090059812900798CDF844B030
:107B8000CDE9130B01981590A07A179003981690E1
:107B900010A93046FBF725F916F0070F74D0002026
:107BA000F8F78CFF9AF8101088421AD00020F8F7E6
:107BB0007AFF9AF8100000EB400101EB00107549C4
:107BC00001EB80004C2116F062FF9AF8100000EBE8
:107BD000400101EB0010704901EB80004C2116F0D0
:107BE00056FF06F06EFA18B101460020F9F7ADFD18
:107BF00006F07EFA6843050B06F09AFA09FB00F0DE
:107C0000000B4030C1090A20012202FA00F30B42A6
:107C100001D1401EF9D5A0F10509207B002818BF2D
:107C2000A0F1010B11D10CE05C480068B0F8B00085
:107C300010F4807F18BFFCF70FF9002019B0BDE8E1
:107C4000F08F0020F9F76DFF8346607B002814BF9A
:107C5000401EF9F79EFF0BEB0901052905DDA9EB95
:107C6000010101F10509052104E00029BCBFA9EBD0
:107C7000010900218144B9F1050F06DDA9F10500D4
:107C8000C5404FF0050908E00EE0B9F1000F04DA35
:107C9000C9F1000085404FF000090020F9F75BFFB3
:107CA00049460020F9F78FFF16F0F00F43D0207CF3
:107CB00070B116F0100F03D0411E0120F9F74BFFF1
:107CC00016F0400F04D0207C411E0220F9F743FF3C
:107CD000207D70B116F0200F03D0411E1120F9F75E
:107CE0003AFF16F0800F04D0207D411E1220F9F7D4
:107CF00032FF607C70B116F0100F03D0411E0120DE
:107D0000F9F761FF16F0400F04D0607C411E02209D
:107D1000F9F759FF607D70B116F0200F03D0411EB6
:107D20001120F9F750FF16F0800F04D0607D411E3E
:107D30001220F9F748FFE07A00281CBF0001F9F78C
:107D40003DFC029806F099F9049830B12B469AF858
:107D50000D209AF80C1016F0FEFE3A4641462846D1
:107D6000189B16F0FDFE0698FEF738F80898FEF707
:107D70006EF80AF07BFE19B00120BDE8F08F10B557
:107D8000FBF7FEF806F081F905490020C8610120E3
:107D900010BD000000000130004001302C830010B5
:107DA00040810010FE4908707047FD480078704718
:107DB000FC4810B4FC4A016891421CD14168B1F5FD
:107DC000987F18D8D0F808C00146BCF5007F12D8BB
:107DD00000220B461146B2EB9C0F24BF10BC70472B
:107DE00053F82140491C2244B1EB9C0FF8D3002AE0
:107DF00004BF10BC7047002010BC7047E948FCF776
:107E000001B9E7490120087070472DE9F041174694
:107E10000E4605461024FFF7E4FD15F0070F18BFC6
:107E2000062403D115F0F00F18BF08243246102C99
:107E300028BFBDE8F081002A08BFBDE8F0812044DA
:107E40003B4690F920102046BDE8F04106F09FBC6B
:107E50002DE9F04FADF6446D0C468046FFF7C1FDAD
:107E6000814618F0070F7DD06F4605263846FBF790
:107E700043FC09F1050599F925104FF464633A466E
:107E8000304606F084FC95F8200003286FD1C748DF
:107E90000578C7480778512004F030FF824600215A
:107EA000084604F0B9FE0646C2480078512804BFCF
:107EB000002005F00DF80020BF4A530C04EB8001B0
:107EC000401CCA87A1F840300428F7D30023002FB4
:107ED00020D90020002D88BF03F0070C17D9BCF172
:107EE000040F34BF0121022103FB050204EB8101D1
:107EF00036F91220B1F93AB09345B8BF4A87B1F9C3
:107F00003CB09345C8BF8A87401CA842E7D35B1C9E
:107F1000BB42DED30020A94B84F83C0003F10805E6
:107F2000012204EB800133F91060B1F93EC0B44581
:107F300007DB94F83CC002FA00F64CEA060C84F821
:107F40003CC0B1F9401035F910C0614507DC94F828
:107F50003C1002FA00FC41EA0C0184F83C10401C81
:107F6000042800E003E0DCD3504604F0C7FE18F01C
:107F7000F00F04BF0DF6446DBDE8F08F07246D4689
:107F8000FBF73BF810F0300F0CBF022001206946D0
:107F9000FBF714FC99F927104FF418732A46204672
:107FA00006F0F5FB0DF6446DBDE8F08F2DE9F34FBB
:107FB00089B000200690087803904868049088688B
:107FC00005900D7B487B0190887B8A8AD1E9088BDC
:107FD000C0F5807602EA00070998B1F91090B1F96E
:107FE00012A0896910F0010F07914FF0000044D0F2
:107FF00000900198002840F2E8800098012101FAE1
:1080000000F20798104018BF012000240290610977
:1080100004A804F01F0250F82110012090400142F2
:1080200000F0B7803BF9020B0299A0EB0A0000298F
:108030000CBFA9EB000509EB000538F9020BA0EB1A
:108040000A0014BF4844A9EB0000002DB4BF6942E8
:1080500029460028B8BF4042884278D92246009974
:108060000398FAF751FB0246C0F30420D1B212F490
:10807000803F6FD0002D6FDB70E0F9F7AEFE00900F
:1080800001980321684301EB400020F003024146C0
:10809000584616F006FD0098F9F79FFE01984FF03C
:1080A000000B002852D90121079801FA0BF2104069
:1080B00018BF012000250290690904A805F01F02DD
:1080C00050F8211001209040014237D038F9020BBE
:1080D0000299A0EB0A0000290CBFA9EB000409EBF0
:1080E00000042A4659460398FAF70EFBC0F3042110
:1080F000C2B210F4803F02D0002C02DB03E0002C5F
:1081000001DD941B00E09419BC4205DD1F293ABF34
:108110000024491C3C4606E0002C04DA0029C6BFB6
:108120003C46491E002400F4783040EA012040EA31
:1081300004032A4659460398FAF739FB6D1C262D8D
:10814000BAD301980BF1010B8345ACD33DE020E09D
:1081500000E001E0002D01DD8D1900E08D1BBD4226
:1081600005DD1F283ABF0025401C3D4606E0002DD6
:1081700004DA0028C6BF3D46401E002502F47831CF
:1081800041EA002040EA0503224600990398FAF7E5
:108190000EFB641C262CFFF43AAF0098401C0FE045
:1081A0006C81001000EE0300544352464C810010D5
:1081B0004D810010E58100100080FFFF84810010D8
:1081C000019900908842FFF418AF0998032826BF50
:1081D0000120069006980BB0BDE8F08F2DE9F04F16
:1081E0008BB0002205920A7800924A6802928A684F
:1081F00003924D7B8A7B0492B1F91080B1F9122071
:1082000007920C6A8A690892898A049AC0F1080A5E
:1082100001EA020600283BD0BAF1000F7ADB4FF0EA
:10822000000B002D77D9012000FA0AF00690AAF180
:108230000100012101FA00F009900121089801FADA
:108240000BF2104018BF012000270190790902A805
:1082500007F01F0250F821100120904001427DD00C
:1082600034F9021B0798081A019900290CBFA8EBE2
:10827000000908EB00093A4659460098FAF744FA13
:10828000034610F4803F72D0B9F1000F74DA71E048
:108290004FF0000B002D3ED90121089801FA0BF296
:1082A000104018BF012000270190790902A807F0AB
:1082B0001F0250F821100120904001424BD034F9A8
:1082C000021B0798081A019900290CBFA8EB0009A6
:1082D00008EB00093A4659460098FAF715FAFE49A4
:1082E000014011F4803F17D0B9F1000F29DA11F4E1
:1082F000F8511CBFA1F5807141F4803121D110F4F7
:10830000604F1ED0A0F500504FF4D05110F4003F44
:1083100017D014E04AE042E0B9F1000F11DD11F48A
:10832000F85118BFA1F580710BD110F4604F08D03F
:10833000A0F500504FF4D05110F4003F01D04FF49D
:108340008D3100F43830084340F080033A465946F6
:108350000098FAF72CFA7F1C262F02E016E006E0C0
:108360000AE0A2D30BF1010BAB4595D317E0B9F1AD
:10837000000F01DD06988343BAF1000FC4BF0998CE
:1083800003433A4659460098FAF711FA7F1C262F04
:10839000FFF45CAF0BF1010BAB45FFF44EAFBAF14C
:1083A000000FC2BF05980BB0BDE8F08F0027002D6D
:1083B0002ED904980DF1080A4FF0010BC0F5807911
:1083C00040F480780024600904F01F015AF820006E
:1083D0000BFA01F1084215D0224639460098FAF707
:1083E00093F9C1B201EB590101EA0801B14288BF1A
:1083F000314620F0FF0040EA01032246394600984A
:10840000FAF7D5F9641C262CDDD37F1CAF42D9D3F3
:10841000012005900BB0BDE8F08F2DE9F04F89B039
:10842000002204920A7800924A6802928A680392B3
:108430004A7B0192B1F91060B1F912B00C6A8969F6
:10844000C0F105080591002837D0B8F1000F70DBA6
:108450004FF00009002A6BD908F10800012101FA48
:1084600000FA401E01FA00F006900121059801FA79
:1084700009F2104018BF012000250790690902A8E1
:1084800005F01F0250F821100120904001425FD0FA
:1084900034F9020B0799A0EB0B0000290CBF371A27
:1084A00037182A4649460098FAF72EF9034610F481
:1084B000803F3FD0002F41DA3EE00027002A4FD90D
:1084C0000120059900FA07F20A4214BF4FF0010A91
:1084D0004FF0000A0025690902A805F01F0250F8B4
:1084E00021100120904001421BD034F9020BBAF157
:1084F000000FA0EB0B000CBFA6EB000906EB000978
:108500002A4639460098FAF7FFF8B9F1000FC8BFBC
:1085100040F4803040F480532A4639460098FAF7F8
:1085200046F96D1C262DD6D301987F1C8742C7D3F0
:1085300016E01AE0002F01DD23EA0A03B8F1000F6C
:10854000C4BF069803432A4649460098FAF72FF914
:108550006D1C262D92D3019809F10109814584D320
:10856000B8F1000F04BF01200490049809B0BDE8E1
:10857000F08F2DE9F04F89B0002204920A78009222
:108580004A6802928A6803924A7B0192B1F91060AC
:10859000B1F912B00C6A8969059150490969421A0A
:1085A000C2F10308814277D83DD101984FF000070E
:1085B000002871D90120059900FA07F20A4214BF78
:1085C0004FF0010A4FF0000A0025690902A805F0E2
:1085D0001F0250F821100120904001421BD034F9B5
:1085E000020BBAF1000FA0EB0B000CBFA6EB0009C9
:1085F00006EB00092A4639460098FAF785F8B9F1E2
:10860000000FC8BF40F4003040F400432A4639460A
:108610000098FAF7CCF86D1C262DD6D301987F1C54
:108620008742C7D34FE0B8F1000F51DB01984FF0FC
:108630000009002847D908F10D00012101FA00FACC
:10864000401E01FA00F006900121059801FA09F296
:10865000104018BF012000250790690902A805F005
:108660001F0250F8211001209040014223D034F91C
:10867000020B0799A0EB0B0000290CBF371A371823
:108680002A4649460098FAF73FF8034610F4003F9F
:1086900003D0002F05DA02E015E0002F01DD23EA08
:1086A0000A03B8F1000FC4BF069803432A4649469F
:1086B0000098FAF77CF86D1C262DCED3019809F1AD
:1086C00001098145C0D3B8F1000F04BF0120049017
:1086D000049809B0BDE8F08F001F01006C81001004
:1086E0002DE9F14FADF54E7D0020C090BF9072B6E0
:1086F000FAF783FC0746FCF74BFB48B1FCF7F0FBAD
:10870000C090FCF7D7FBFCF7F0FBBF90FCF7DDFB5C
:10871000FAF75BFBFAF776F9C590FAF77CFCC490A0
:10872000FAF772F9FAF701FDBC900020FAF7F4FCB1
:108730000120F9F7EEFAC8901120F9F7EAFAC9908A
:108740000220F9F7E6FACA901220F9F7E2FACB9084
:10875000FCF767F9C390FCF74CF94FF49350FCF722
:10876000BAF862B60020F9F7A5FAC29001210020FC
:10877000F9F793FA0020F9F7B2FA0021C190084600
:10878000F9F7A0FA0120F9F728FBCC900020FAF7BE
:1087900084F9C7900020FAF773F9C690F8F7C9FE7C
:1087A000CD900020F8F7CAFE002006469EAD45F8A1
:1087B0002060401C0C28FAD317F0070F4FF001047B
:1087C0000AD040F68C61FE489E9416F060F940F69F
:1087D0008C61FC4816F05BF917F0F00F47D00120D0
:1087E000F8F79DF938B19821F74816F050F998211B
:1087F000F64816F04CF91120F8F791F938B19821A4
:10880000F34816F044F99821F24816F040F9022096
:10881000F8F785F938B19821EF4816F038F9982122
:10882000EE4816F034F91220F8F779F938B19821AA
:10883000EB4816F02CF99821EA4816F028F90120A7
:10884000F8F76DF9002818BFA0941120F8F767F920
:10885000002818BFA1940220F8F761F9002818BF7A
:10886000A2941220F8F75BF9002818BFA3944FF0E8
:10887000405ADFF874B3DFF874939E984FF0FF0806
:1088800058B330468DF8006001A9F9F7A7F89DF8B4
:108890000000F9F7C3F88DF80C009DF80000F8F718
:1088A0000DF98DF80D009DF80000F9F77CFA00280D
:1088B0000CBF4FF0FF31002106918DF80E80B9F802
:1088C0000200ADF81000ADF812609DF80000F9F755
:1088D00025F8ADF81400CDE908AB9F986F4640B37A
:1088E0008DF8286007F12C013046F9F777F89DF8EC
:1088F0002800F9F793F88DF834008DF8354010967C
:108900008DF83680B9F80200ADF83800ADF83A605D
:108910009DF82800F9F702F8ADF83C009DF80C002E
:108920009DF80D1048430AEB40010BEB4000CDE9E8
:108930001210A0984FF4806A02264FF0AA3BE0B3D1
:108940008DF8504007F154012046F9F747F89DF89B
:108950005000F9F763F88DF85C009DF85000F9F7C6
:10896000E0F804FA00F08DF85D009DF85000F9F78A
:10897000D0F91A908DF85E80B9F80400ADF8600067
:10898000ADF862A09DF85000F8F7C8FFADF864009C
:1089900097481C9097481D909DF85D00022809D9C2
:1089A0009DF85C10801E48431C9901EB40001C9010
:1089B0008DF85D601A9800B100E007E09DF8500066
:1089C0004FF0AA31F9F793F9CDF868B0A198E0B368
:1089D000112007F17C018DF87800F8F7FFFF9DF872
:1089E0007800F9F71BF88DF884009DF87800F9F706
:1089F00098F804FA00F08DF885009DF87800F9F7F2
:108A000088F924908DF88680B9F80600ADF88800C2
:108A1000ADF88AA09DF87800F8F780FFADF88C00DB
:108A200075482690754827909DF88500022809D939
:108A30009DF88410801E4843269901EB4000269043
:108A40008DF88560249800B100E007E09DF878007B
:108A50004FF0AA31F9F74BF9CDF890B0A298E0B3F6
:108A600007F1A40130468DF8A060F8F7B7FF9DF834
:108A7000A000F8F7D3FF8DF8AC009DF8A000F9F73F
:108A800050F804FA00F08DF8AD009DF8A000F9F759
:108A900040F92E908DF8AE80B9F80800ADF8B0001E
:108AA000ADF8B2A09DF8A000F8F738FFADF8B4001B
:108AB00053483090534831909DF8AD00022809D9B1
:108AC0009DF8AC10801E4843309901EB4000309077
:108AD0008DF8AD602E9800B100E007E09DF8A00091
:108AE0004FF0AA31F9F703F9CDF8B8B0A398E0B385
:108AF000122007F1CC018DF8C800F8F76FFF9DF840
:108B0000C800F8F78BFF8DF8D4009DF8C800F9F77E
:108B100008F804FA00F08DF8D5009DF8C800F9F7C0
:108B2000F8F838908DF8D680B9F80A00ADF8D8007A
:108B3000ADF8DAA09DF8C800F8F7F0FEADF8DC005B
:108B400031483A9031483B909DF8D500022809D928
:108B50009DF8D410801E48433A9901EB40003A90AA
:108B60008DF8D560389800B100E007E09DF8C800A6
:108B70004FF0AA31F9F7BBF8CDF8E0B0F8F728FAD2
:108B800010F0010F0BD0FEF72FFF3C2807D1FCF7A8
:108B900011FB20B10420FCF7BCFAFCF793FBFAF7B9
:108BA00079FA4FF00008C346C2464646C14603F074
:108BB000E3FD01287DD0BBF1800F7AD8AAA827E079
:108BC00000000130004001308C0E01308C4E01302D
:108BD000240F0130244F0130BC0F0130BC4F013055
:108BE0005410013054500130004000306C810010AE
:108BF000CC090030CC490030CC0E0030CC4E0030D7
:108C00004C1800304C5800304C1D00304C5D00308A
:108C1000FAF716FD00286ED0AAA804F0EFFCBC9865
:108C2000002818BF00273BD09EA850F82700A0B30B
:108C300007EB8701684600EBC104207810F00F0FA6
:108C40002BD0F9F766F810F0010F26D0216A257BAA
:108C500001F0030000EB8502D21C22F0030221F098
:108C60000301CDE9BD1278A90C1878A8BD9915F0BB
:108C700018FF0020002D0BD9411934F8102034F8CA
:108C8000113024F81030401C24F811208542F3D80C
:108C900078A9BE9ABD9815F004FF7F1C0C2FC3D392
:108CA0001AF1010A7DD04FF0000A5046B0AD0127FD
:108CB00000E077E00BF1010B45F82070401C0C2818
:108CC000FAD3052E6ED2DFE806F003172A3D5000D6
:108CD00000249EA850F8240048B104EB84016846A3
:108CE00000EBC1014846FFF744FC45F82400641C32
:108CF0000C2CEED33BE068E000249EA850F8240042
:108D000048B104EB8401684600EBC1014846FFF717
:108D100084FB45F82400641C0C2CEED327E00024CF
:108D20009EA850F8240048B104EB8401684600EB8B
:108D3000C1014846FFF752FA45F82400641C0C2C88
:108D4000EED314E000249EA850F8240048B104EBB0
:108D50008401684600EBC1014846FFF727F945F852
:108D60002400641C0C2CEED301E04FF0010801211B
:108D7000002055F82020CAB1401C0C28F9D3A9B115
:108D80001F2E0DD2761CCE9807FA06F1014207D1AC
:108D9000761C042E04D8CE9807FA06F10142F7D0CB
:108DA00001E005E017E04FF0000901E009F10109D9
:108DB000FAF79DFCB8F1000F0DD1BC98002818BF40
:108DC000F8F7B9FFFAF766F9F1E6FEF7DDFCB8F15E
:108DD000000F3FF4ECAEFAF78AFCF9F715FE052018
:108DE000FCF797F90120C899F8F781FF1120C9997C
:108DF000F8F77DFF0220CA99F8F779FF1220CB9986
:108E0000F8F775FFBC98FAF787F90020C199F8F7D1
:108E100059FF0020C299F8F740FFCC98F8F7DDFF22
:108E2000C798F9F73AFEC698F9F72AFECD98F8F7F1
:108E300085FBC59830B1C49810B1FAF72BF901E061
:108E4000FAF7EFF8FBF7A4FF48B1C098002818BF65
:108E5000FBF7A4FFBF98002818BFFBF7D8FFC39803
:108E6000002818BFFBF76EFDB8F1000F0CBF012002
:108E700000200DF54F7DBDE8F08F70B5FE4D164614
:108E8000D5F844231205120D1DD000281CBFC1F3D4
:108E90000800FAF777FFD5F8480340F00100C5F85D
:108EA0004803D5F8480320F00100C5F84803002224
:108EB000341E23DDD5F8481340F2AF2011F0010F26
:108EC00008D1401E01D2002070BDD5F8481311F022
:108ED000010FF6D0D5F84403C0F30B000244D5F8D7
:108EE000480340F00100C5F84803D5F8480320F0D6
:108EF0000100C5F84803641E002CDBDC1001B0FB48
:108F0000F6F080B270BD2DE9F84F040016D0DB48B2
:108F1000006CC0F30829FAF747FF49EA0042002332
:108F20009621072008F022FCD348D0F8401341F4E2
:108F30008031C0F84013322000900AE0FAF72FFF8A
:108F40000120BDE8F88F00BF00BF00BF00BF00BF19
:108F50000846411E0091F6D24FF0000840F2FF177C
:108F6000C246464608EB070000EBD0704510A9B298
:108F700064220120FFF781FFF0B1A04288BF6F1E7D
:108F800038BF05F101081ED1AA461FFA8AF14FF039
:108F900064024FF00100FFF770FF044600235246C1
:108FA0009721072008F0E2FBA4F5A8502C38A02850
:108FB0009CBF0120BDE8F88FB9F1000F10D04846E2
:108FC000FAF7E0FE0EE0011B48BF211A321B48BF32
:108FD000A21B9142BCBFAA460646B845C2DDD4E7F3
:108FE000FAF7DDFE49F4803200239721072008F0CC
:108FF000BDFB0020BDE8F88F2DE9F04FA04CADF58A
:10900000157D01262778FEF75DFB012840F06B8176
:1090100004F0E7FC9B480068B0F91E10B0F91C0092
:1090200015F0A3FD17F0020F00F0548180ADFEF79C
:10903000BFFE4FF0000828B101465022284615F027
:1090400021FD21E0FF225021284615F048FD8E48E1
:1090500080904FF4987081905020CDE98208CDE93E
:1090600084084FF0FF308B908A90CDF81882899059
:10907000CDE98780ADF838828DF83A82CDF830821C
:10908000CDF834828DF83B828048FAF7BBFF859893
:10909000401C8590F9F799FE41F27C50FFF733FFB1
:1090A0007749C860F9F752FF80A8CDE9008040F207
:1090B0003339002577E0284605F023FB002871D0DE
:1090C000008900EA090434F0CC006BD040F20F3183
:1090D0002846FEF7B6FC002864D0F9F78EFF009909
:1090E00000295DD1F9F747FE24F0EE0030F47E4010
:1090F00017D01F20FFF7F4FA0090F9F785FC0098CD
:1091000000284DD17EB114F0010F03D00720019942
:10911000FEF79EFE14F0100F03D0F0200199FEF729
:1091200097FE0098E0BB14F0220F06D0FCF7B1FECA
:109130000090F9F769FC009890BB8EB314F0020F11
:1091400016D0FCF767FA83465148017851480078F9
:1091500048434FEA400AFEF744FC4FF0060C5FEA32
:109160000B0205D090F926105346604605F00FFB20
:1091700014F0200F14D0FCF7E2F9044646480178B9
:109180004648007808444FEA400AFEF72AFC0146A8
:109190000820220004D091F92810534605F0F7FA70
:1091A000FEF7EDFD6D1C05F0A8FAA842009802D963
:1091B000002880D003E0002808BF012000D0002054
:1091C00018B1FCF746FF01281FD087980023401CE8
:1091D0008790502084901A462121072008F0C6FA73
:1091E00000231A461946FE20CDF80080FDF72AF824
:1091F00080AD05F05AFA50B381698891C1698991AF
:1092000041698A91C0688B9027E017F0080F14BF5E
:10921000A220A12084901A48C16859B11749096C4D
:10922000C1F30821ADF838129DF83A12491C8DF8A7
:109230003A1206E0ADF838829DF83B12491C8DF8D1
:109240003B12C0F80C808698401C8690D0E74FF007
:10925000FF308B908A90899088900B4880904FF4D3
:10926000987081905020CDE982080021AA682C4690
:10927000084654F8203013E00050004000600040E1
:109280006C8100102C8300105443524600EE030002
:109290004F81001050810010518100105281001048
:1092A000401C1944B0EB920FE3D34842E860FF2220
:1092B0004FF40071684615F012FC502229466846AA
:1092C00015F0E0FB984C2046FAF79CFE69462046D4
:1092D000FAF73AFF0020FCF71AFD00233A46402136
:1092E000072008F043FA0DF5157DBDE8F04F03F0B7
:1092F000A3B98E4A022804BF1181704707DC0028F9
:1093000004BF51807047012808BF91807047112821
:1093100004BFD1807047122808BF518170470146B1
:1093200000200229814A04BFB2F90800704709DC15
:10933000002904BFB2F902007047012908BFB2F941
:1093400004007047112904BFB2F9060070471229C2
:1093500008BFB2F90A00704770B50126FEF728FD74
:1093600020B10069A12818BFA22801D0002070BD3B
:10937000002405F0C2F9002834D9204605F0C1F9CF
:1093800000281EBF058925F0CC0030F47C4024D095
:1093900040F20F312046FEF754FBF0B115F0010FFB
:1093A0000AD0FAF7BEF938B944F4807200232021BC
:1093B000072008F0DBF9002615F0100F0BD0012074
:1093C000FAF718FA38B944F4805200232021072014
:1093D00008F0CCF90026FEF7D2FC641C05F08DF9EC
:1093E000A042CAD8304670BD0020704700207047A8
:1093F0004E48407870474D4900204870704770B51E
:10940000002105220846FFF738FD0023474A0028BF
:109410002BD05178002908BF5361A0F5A85CACF1AE
:10942000750CBCF10E0F20D9491CC9B25170D2F88D
:1094300014C00A296044506121D93D495370096C18
:10944000C1F308249CB14EF65441884294BF651C78
:10945000651E2846FAF796FC44EA0542002395214A
:10946000072008F083F9012070BD537007E041F236
:109470007C50FFF748FD00281CBF012070BD002074
:1094800070BD10B5FEF794FC38B32A4A01689142CA
:1094900023D14168B1F5987F1FD8D0F808C00146A4
:1094A000BCF5007F19D800220B461146B2EB9C0F89
:1094B00007D253F82140491C2244B1EB9C0FF8D34A
:1094C0005AB9188F00281CBFA0F57F41B1F1FF01E8
:1094D00003D0FAF757FC012010BD002010BD10B5D5
:1094E000FEF766FCD8B1134A0168914217D1416872
:1094F000B1F5987F13D8D0F808C00146BCF5007FBD
:109500000DD800220B461146B2EB9C0F09D253F83E
:109510002140491C2244B1EB9C0FF8D30AB1002032
:1095200010BD188F10BD000000EE03006C8100100C
:10953000006000405443524670470020704710B509
:1095400003F00700042808BFFEF77CF9002010BDD7
:1095500010B403F007020024FE4BDFF8FCC3012A1D
:1095600002D0022A17D013E005208CF80000FB4837
:10957000CCF80C4000681A68532111701A68452114
:1095800051701A68010A91701968C87018680471DE
:1095900010BC002070479CF80020052A14D1DCF88C
:1095A0000C20052A28BF104605D21B689B5C03705F
:1095B000501CCCF80C00052806D10120CCF80C403A
:1095C000087003208CF8000010BC0120704770B5B3
:1095D00003F007020125DF4CDF4B4FF0000C012A9E
:1095E00002D0022A25D022E005201870DB48C3F8FB
:1095F0000CC000682268AC2111702268010A517009
:10960000216888702068C570206880F804C004F064
:10961000EDFF48B1D24D286805F0F1F820B1286877
:109620002168007E487102E02168FF204871002017
:1096300070BD1A78052A10D1DA68062A28BF1046AC
:1096400004D22468A45C0470501CD860062804D19D
:10965000C3F80CC00D7003201870012070BD03F01A
:109660000702022A1CBF002070472022027001203E
:10967000087070472DE9F041B74F0D46064613F0CC
:10968000070F04D003F00700022808D004E012F00E
:10969000040F1CBF0020B8700020BDE8F08102F06C
:1096A000C5FF002814BF0124002402F0C2FF0028D7
:1096B00014BF0222002242EA0403B878002814BF33
:1096C0000422002242EA0300307001202870BDE825
:1096D000F08170B503F0070C00269F4C9D4DBCF146
:1096E000010F0AD0204613F0070F00780DD0BCF10F
:1096F000040F08BF062818D029E0E6602868067025
:10970000286846700520207021E005281FD1E068F8
:10971000022803D22B681A54401CE060022816D19C
:109720000120E6600870062010E0286800785528BF
:109730000BD128684078AC2818BFBC2805D1286810
:109740000122411C062002F057FF03202070002058
:1097500070BD70B503F0070200257E4C7E4B012AD8
:1097600002D0022A24D021E005201870DD6002F02A
:109770000CFF41F6E8710144B0F5783F10D8CA7883
:10978000086862F31F60774A904208BF002007D143
:109790000A18236812791A54401C1428F8D305E0DB
:1097A000002021680D54401C1428FAD3002070BDFD
:1097B0001A78052A13D1DA68142A28BF104607D26E
:1097C000D4F800C01CF802C080F800C0501CD8605B
:1097D000142804D10120DD600870032018700120D6
:1097E00070BD70B503F0070200255A4C5A4B012A90
:1097F00002D0022A3FD03CE005201870DD6002F064
:10980000C4FE41F6E8710144B0F5783F2BD8CA7820
:10981000086862F31F60534A904224D12268087C92
:1098200010702268487C50702268887C9070206894
:10983000CA7CC27020680A7A02712268487A507124
:109840002268887A90712268C87AD0712268087D6F
:1098500010722268487D50722268887D9072C87D9F
:109860002168C87205E0002021680D54401C0C28B6
:10987000FAD3002070BD1A78052A13D1DA680C2AB1
:1098800028BF104607D2D4F800C01CF802C080F8E8
:1098900000C0501CD8600C2804D10120DD60087085
:1098A00003201870012070BD70B503F00702002579
:1098B000284C294E012A02D0022A36D033E004F087
:1098C000F4FE40B3D0E906212368C0681A70D4F8CA
:1098D00000C0130A8CF80130D4F800C0130C120E2B
:1098E0008CF802302368DA702268117123680A0A42
:1098F0005A7123680A0C090E9A712268D171216885
:1099000008722268010A51722268010C9172010EDC
:109910002068C17204E021680D54401C0C28FAD361
:1099200005203070F560002070BD3278052A10D116
:10993000F2680C2A28BF104604D223689B5C03708F
:10994000501CF0600C2804D10120F5600870032041
:10995000307009E0D84102009C810010044C0040A6
:109960002C83001034CD12AB012070BD70B503F014
:1099700007020024F94DFA4B012A02D0022A3ED0F8
:109980003BE0052018700026DC6002F0FEFD00F5CB
:109990000051B0F5783F98BF11F0030F27D1F14A7D
:1099A0000868904204BF0022104620D151F82030B0
:1099B000401C1A440728F9D302B1C6B128680A7CB2
:1099C00002702A68487C50702A68887C90702A68E7
:1099D000C87CD0702A68087D10712A68487D507153
:1099E0002A68887D9071C87D2968C87105E00020CB
:1099F00029680C54401C0828FAD3002070BD1A783E
:109A0000052A13D1DA68082A28BF104607D2D5F8EC
:109A100000C01CF802C080F800C0501CD8600828A4
:109A200004D10120DC60087003201870012070BD93
:109A30002DE9F04103F0070C0027C94E4FF005084F
:109A4000BCF1010F0DD013F0070F0FD03246BCF15F
:109A5000020F127810D0BCF1040F08BF062A26D0DE
:109A600058E086F800807770F76053E07270BE4867
:109A7000F062062030704DE0052A15D1F268042A04
:109A800028BF104609D2C2F10303D6F82CC0DB0070
:109A90002CFA03F30370501CF060042804D1012059
:109AA000F7600870032030700120BDE8F081707805
:109AB0000125002410F0010F11D002F066FDB0F571
:109AC000783F23D86A030021B1EB900F07D252F8F8
:109AD000043B491C1C44B1EB900FF8D3B5B170782E
:109AE00010F0020F0ED004F0E0FD78B18268002182
:109AF000B1EB920F06D250F8043B491C1C44B1EB69
:109B0000920FF8D3002D18BFF46200D1F76277707E
:109B100086F800800020BDE8F081F0B503F0070C66
:109B200000268E4D8E4C83B0BCF1010F0ED013F089
:109B3000070F1DD0224603271278BCF1020F26D052
:109B4000BCF1040F08BF062A36D03CE002AA01A9E6
:109B5000684603F0A6F8052020702968019808706F
:109B6000296800984870296802988870E6602AE0A1
:109B7000E068032803D229680A54401CE0600228E8
:109B800021D306212170032808BFE6601BE0052AC7
:109B90000FD1E268032A28BF104604D22B689B5CD1
:109BA0000370501CE060032803D10120E6600870B8
:109BB000277003B00120F0BD2868827801784078D2
:109BC00003F062F8277003B00020F0BD08B503F081
:109BD000070001280AD104F009FD38B101208DF8F1
:109BE0000000024669460D2002F006FD002008BD77
:109BF00008B503F0070001280AD104F0F7FC38B1DA
:109C000000208DF80000012269460D2002F0F4FCCE
:109C1000002008BD08B503F00700012809D104F0B1
:109C2000E5FC30B103208DF800000122694602F006
:109C3000E3FC002008BD0020704708B503F00700D2
:109C400001280AD104F0D2FC38B10B208DF80000B5
:109C500001226946032002F0CFFC002008BD1FB599
:109C600013F0070F0ED104F0C1FC58B19DF80800A5
:109C7000F0280AD004F0BAFC20B1012202A9092080
:109C800002F0BAFC04B0002010BDFEF7B7F8F9E707
:109C90000020704770B503F00700304C304D0128AC
:109CA00008D013F0070F12D0042804BF2878062824
:109CB00016D01FE00020E860216808702168487015
:109CC000216888702168C8700520287012E0E86853
:109CD00004280FD221680A54401CE860062008E0DE
:109CE00004F084FC30B104221046216802F084FCA8
:109CF00003202870002070BD10B503F00700012874
:109D000004D103F06EFE164900200871002010BD3A
:109D100010B503F0070C124CBCF1010F06D013F084
:109D2000070F09D0BCF1020F20D015E00020E06041
:109D300007F013FDE0610FE0E068002804BF1002A7
:109D4000E06106D0012804D1E0691043E06107F02A
:109D500003FDE068401CE060002010BDD841020017
:109D60009C81001054464953EFBEADDEE26812B14B
:109D7000012A04D007E0A18B090A017003E0237FC8
:109D8000037001200870501CE0600120E5E710B569
:109D900003F0070CFE4CBCF1010F06D013F0070FC7
:109DA00009D0BCF1020F18D015E00020E06007F0E8
:109DB000D7FCE0610FE0E068002804BF1002E0611A
:109DC00006D0012804D1E0691043E06107F0CBFC24
:109DD000E068401CE060002010BDE26812B1012A7A
:109DE00004D007E0A18B090A017003E0237F037010
:109DF00001200870501CE060012010BD70B503F018
:109E0000070CE34D0E460446BCF1010F06D013F0DB
:109E1000070F07D0BCF1020F18D015E00020E86052
:109E2000286111E0E868002804BF1002E86108D04A
:109E3000012806D1E869104381B2E861E8880FF093
:109E400006F9E868401CE860002070BD2869022817
:109E50000ED2E8880FF001F92B6982B2002B04BF03
:109E6000100A207004D0012B02D122700120307022
:109E70002869401C2861012070BD10B403F0070C54
:109E8000C34CBCF1010F08BF00200BD013F0070F2B
:109E900003D0BCF1020F09D005E0E068002808BF3C
:109EA000E280401CE06010BC00207047E2681AB9F4
:109EB000A379037001200870501CE06010BC0120E1
:109EC00070472DE9F047064603F00700B04F89467A
:109ED000012808BF002037D0DFF8B882AE4D13F05C
:109EE000070F02D0022833D02FE0F868002808BFFF
:109EF0007A7027D0012804BF1002F86122D002280E
:109F000020D1F8691043F8617E7884B204F06EFBCA
:109F1000C0B1062E16D2DFE806F00306090C1013B6
:109F2000A8F80E400EE0A8F80C400BE028688483E7
:109F300008E02868A0F8144104E02868048601E0DD
:109F400028684486F868401CF8600020BDE8F08767
:109F5000386902282AD297F801A0002404F046FBB1
:109F6000C8B1BAF1060F16D2DFE80AF00306090CF1
:109F70001013B8F80E400EE0B8F80C400BE028685B
:109F8000848B08E02868B0F8144104E02868048E47
:109F900001E02868448E3869002804BF200A307028
:109FA00004D0012802D1347089F800003869401CBF
:109FB00038610120BDE8F0872DE9F0411C461546C7
:109FC0000E46074604F012FB88B1724814F0070FE2
:109FD00004D004F0070102290CD008E0002D1ABFBC
:109FE00090F8F800C0084FF0FF300CF0A9F80020FE
:109FF000BDE8F08190F8F800C0083870012030709A
:10A00000BDE8F0812DE9F0411C4615460F46064695
:10A0100013F0070F08D104F0E9FA28B1022D3CBF74
:10A02000284609F044FC03E004F00700022802D0AF
:10A030000020BDE8F08109F033FC30700120387059
:10A04000BDE8F08170B503F007020026534C504D77
:10A05000012A02D0022A15D012E008F085FC2168FE
:10A060000870FDF72FFB2168487004F027F821687D
:10A070008870FDF72DFB2168C87005202870EE6000
:10A08000002070BD2A78052A10D1EA68042A28BF6A
:10A09000104604D223689B5C0370501CE8600428BF
:10A0A00004D10120EE60087003202870012070BDEB
:10A0B0002DE9F04103F0070C384E0025344CBCF17B
:10A0C000010F08D013F0070F08BF627168D0BCF110
:10A0D000020F66D095E0FDF76BFE617901293AD059
:10A0E0000A216161002875D04169FF292CBFFF2139
:10A0F000C9B2326811708169FF2934BFC9B2FF212A
:10A1000032685170C169FF2934BFC9B2FF2132687A
:10A1100091703268017CD170326890F82010117112
:10A12000018C3268090A5171016A3268090C917117
:10A13000016A3268090ED171016BFF2934BFC9B2BF
:10A14000FF2132681172406BFF2834BFC0B2FF207C
:10A150003168487254E01121616198B3326890F817
:10A160003C1001231170002100EB81023768B2F826
:10A170003EC04FEA1C2C07F803C037685B1C92F8FE
:10A180003EC007F803C0B2F840C04FEA1C2C09E0FB
:10A190009C810010B83101102C830010D8410200BE
:10A1A0002FE031E037685B1C491C07F803C0D6F884
:10A1B00000C05B1C92F840200CF803205B1C0429B3
:10A1C000D2D31DE000E005E0FF221121306814F039
:10A1D00086FC15E030680570306845703068857021
:10A1E00031685020C8703168FF20087131684871AB
:10A1F000316888713168C87130680572306845729D
:10A20000E5600020BDE8F0816369E2689A4228BFFA
:10A21000104607D2D6F800C01CF802C080F800C073
:10A22000501CE060984206D10120E560087060791A
:10A23000002818BF65710120BDE8F08103F0070216
:10A24000FF4B4FF0000C012A08BFC3F80CC001D02F
:10A25000022A01D000207047DA68022A3DBF80F848
:10A2600000C0501CD8601046022803D10120C3F85A
:10A270000CC00870012070472DE9F047064603F036
:10A280000700EF4F8A464FF00008012808BFC7F8C3
:10A290000C8001D0022802D00020BDE8F087F868C9
:10A2A000A0BB0024254602F070F9014600F50050DD
:10A2B00018384FF400524FF04009B1F5783F20D8DC
:10A2C00090F803C003686CF31F63DFF878C363453D
:10A2D00017D1091FB4EB910F06D252F8043B641C4E
:10A2E0005D40B4EB910FF8D3C17D406961F31F600D
:10A2F000A84206D104F07AF9012804BF802030700A
:10A3000001D086F80090F868401CF860012803D15D
:10A31000C7F80C808AF800000120BDE8F0872DE91D
:10A32000F04103F007020026C74CC54D012A02D0B8
:10A33000022A5ED05AE0C54800680520287004F063
:10A3400055F9002851D0C24F386804F058FA002857
:10A350004BD00EF05CFE80460EF05DFE39680A7E42
:10A3600012F0040F11D0C98A2268090A11703968E5
:10A370002268897D517039682268898A090A91703A
:10A3800039682268097DD17010E0898A2268090A3B
:10A39000117039682268097D517039682268C98A4C
:10A3A000090A917039682268897DD17022684FEA64
:10A3B00018211171216881F805802268010A9171C4
:10A3C0002168C8713868226890F8421111722268B9
:10A3D00090F840115172018B2268090A917222682B
:10A3E000817CD1722168007C0873EE600020BDE89A
:10A3F000F0812A78052A10D1EA680D2A28BF104674
:10A4000004D223689B5C0370501CE8600D2804D1C3
:10A410000120EE600870032028700120BDE8F08163
:10A420002DE9F04703F007020025874C844B012AF1
:10A4300002D0022A5CD058E0052018700026DD60AA
:10A4400002F0A3F800F50053B0F5783F98BF13F081
:10A45000030F44D17F4A1968914204BF002211467C
:10A4600008D153F821C0491C62440729F9D3002AB6
:10A4700008BF01269F7C93F813807EB3002241F62B
:10A48000E8710144B0F5783F07D8CB78086863F3EA
:10A490001F606C4B984208BF01228E7C91F813908C
:10A4A000002A08BF002013D004F0FFF8216880695B
:10A4B0000E70216881F801902268010C000E9170E5
:10A4C0002168C87020680771206880F805800CE05A
:10A4D00021680D54401C0628FAD306E0FFE700204F
:10A4E00021680D54401C0628FAD30020BDE8F087EF
:10A4F0001A78052A13D1DA68072A28BF104607D22E
:10A50000D4F800C01CF802C080F800C0501CD8600D
:10A51000072804D10120DD60087003201870012095
:10A52000BDE8F08770B5054603F007000C46022829
:10A5300029D104F05BF830B3454800220068037E5F
:10A54000C3F380008000C3F3400100EB410003F03F
:10A5500001010844082812D2DFE800F00406080AC6
:10A560000C0E111004220AE0052208E0062206E083
:10A57000072204E0022202E0032200E001222A7006
:10A580000120207070BD002070BD10B503F0070CD5
:10A590002B4CBCF1010F06D013F0070F0AD0BCF111
:10A5A000020F1AD017E00020E06020610EF0AFFD2E
:10A5B000E06110E0E068002804BF1002E06107D00D
:10A5C000012805D1E0691043E06180B20EF09CFDE6
:10A5D000E068401CE060002010BD2269022A0BD216
:10A5E00012B1012A04D007E0A18B090A017003E02F
:10A5F000237F037001200870501C2061012010BDD2
:10A6000070B503F0070100260D4D0446012908BF6F
:10A610002E6301D0022901D0002070BD286B0028D4
:10A6200004BF0D4814F0A6FA296B102928BF267024
:10A6300002D20948405C2070481C2863012070BD8C
:10A640009C81001034CD12ABD8410200044C004074
:10A650002C8300105446495344A500102DE9F041C5
:10A6600003F007010026FD4D0746012908BF2E63B0
:10A6700001D0022902D00020BDE8F08195F8300019
:10A6800000F00F042879204304D1F54814F072FA41
:10A6900001202871052C28BF2E71F148005D38700B
:10A6A000286B401C28630120BDE8F08170B504468A
:10A6B00003F007000D4602281CBF002070BD14F0F7
:10A6C0005EFA20700120287070BD2DE9F04103F082
:10A6D00007020026E34DE14C012A02D0022A1AD0DB
:10A6E00016E005202070002211461046E66002F0B8
:10A6F000D8FA4FF6FF7101EA40006061FCF7E2FF13
:10A70000032803BF28782028D74802F0DDFAA0628A
:10A710000020BDE8F0812278052A1DD1D4F814C0AC
:10A72000E268624528BF104607D212F0010F1CBF35
:10A730006378037013D0501CE06060450CD1012099
:10A74000E660087003202070FCF7BCFF032806BFFA
:10A750002878202802F0C5FA0120BDE8F081A76A18
:10A7600022F00103FB5A1F0A07706370E3E770B51C
:10A7700003F007020025B94C012A02D0022A11D0A9
:10A780000EE0BA4805220068B0F94211B0F9400164
:10A79000227008444000E560606102F086FDA0621E
:10A7A000002070BD2278052A17D1D4F814C0E268C1
:10A7B000624528BF104607D212F0010F1CBF637814
:10A7C00003700CD0501CE060604506D10120E560AC
:10A7D00008700320207002F076FD012070BDA66A8B
:10A7E00022F00103F35A1E0A06706370EAE70020A4
:10A7F000704770B50D46044613F0070F04D003F000
:10A800000700022805D002E01046FCF74FFF0020A9
:10A8100070BDFCF74EFF20700120287070BD70B530
:10A8200003F0070203258D4C012A02D0022A17D01B
:10A8300014E004F00CF80646FCF73BFF01463046F6
:10A8400004F07EFA206200281ABF052020702570CF
:10A85000304604F05CFA60620020E060002070BDC9
:10A860002278052A0BD1236AE2689B5C0370501C96
:10A87000E060626A904202D30120087025700120D6
:10A8800070BD00207047002070477FB51C460E4603
:10A89000054613F0070F08D103F0A8FE28B10122E6
:10A8A00002A9262001F0A8FE03E004F00700022818
:10A8B00002D004B0002070BD02F0CEFA2870012052
:10A8C000307004B070BD2DE9F04103F0070200279D
:10A8D000624E88460546012A02D0022A0BD007E0C4
:10A8E000052030701220F760706102F0EDF9B0625F
:10A8F0000020BDE8F0813078052819D1F268706930
:10A90000824228BF104608D212F0010F1CBF707897
:10A91000287010D0F068401CF0607169884207D13F
:10A920000120F76088F800000320307002F0D9F9A8
:10A930000120BDE8F081002402F08EFA012804D144
:10A94000F068B16A20F001000C5A200A2870747077
:10A95000E0E770B50D46044613F0070F04D003F08E
:10A960000700022805D002E0104603F06DFF00202A
:10A9700070BD03F06CFF20700120287070BD7FB5A2
:10A980001C460E46054613F0070F08D103F02EFEB5
:10A9900028B1012202A9202001F02EFE03E004F0DC
:10A9A0000700022802D004B0002070BD08F029F989
:10A9B00028700120307004B070BD7FB51C460E4673
:10A9C000054613F0070F08D103F010FE28B101224D
:10A9D00002A9212001F010FE03E004F00700022884
:10A9E00002D004B0002070BD08F011F928700120D9
:10A9F000307004B070BD7FB51C460D46064613F09E
:10AA0000070F08D103F0F2FD28B1012202A91C2092
:10AA100001F0F2FD03E004F00700022802D004B0C8
:10AA2000002070BDFCF786FF0446FCF76EFF44EA89
:10AA3000400030700120287004B070BD7FB51C4606
:10AA40000E46054613F0070F12D103F0CFFD78B183
:10AA5000012202A90C2001F0CFFD0DE09C81001025
:10AA600044A50010E5810010D82901102C830010A6
:10AA700004F00700022802D004B0002070BD07F0E7
:10AA800073FF28700120307004B070BD7FB51C4684
:10AA90000E46054613F0070F08D103F0A7FD28B1B5
:10AAA000012202A90F2001F0A7FD03E004F0070036
:10AAB000022802D004B0002070BD0DF06EFE00F040
:10AAC0000F0040F0100028700120307004B070BDFD
:10AAD0002DE9F04103F0070CFB4D0E460746BCF193
:10AAE000010F07D0F94C13F0070F07D0BCF1020F8C
:10AAF0001BD017E00020E860286113E0E868042814
:10AB00003CBF21680A54032809D1206821680068E5
:10AB1000C97800BA20F0FF000843FBF704FEE8689C
:10AB2000401CE8600020BDE8F081286970B9FBF79F
:10AB3000FFFD216820F07E42100E08702168100C85
:10AB400048702168100A88702068C2702A69042A37
:10AB500006D22068032A805C387004BF0120307060
:10AB6000501C28610120BDE8F0817FB51C460D46D0
:10AB7000064613F0070F08D103F038FD28B1012273
:10AB800002A9102001F038FD03E004F007000228BC
:10AB900002D004B0002070BD0DF003FE00F00F04E1
:10ABA0000DF0FBFD64F31F1030700120287004B01D
:10ABB00070BD70B5C44D144613F0070F04D003F0F8
:10ABC0000702022A06D003E01046F5F7F5FB6C6396
:10ABD000002070BD95F8342002700120087070BD0F
:10ABE00070B50D46044613F0070F04D003F00700BC
:10ABF000022805D002E01046FBF780FD002070BD62
:10AC0000FBF77FFD20700120287070BD2DE9F04119
:10AC100003F0070CAD4DAC4C4FF00008BCF1010F38
:10AC20000DD013F0070F1AD02246A94E0327127831
:10AC3000BCF1040F1DD0BCF1020F3DD02FE0C4F8D1
:10AC40000C80286880F80080286880F801802868D7
:10AC500080F80280286880F80380052007E0E0681B
:10AC600004281CD229680A54401CE0600620207089
:10AC700015E0062A13D103F0B9FC80B128680078EA
:10AC800010B101280ED009E02868407800287068CB
:10AC900014BF40F0800020F080007060277000201A
:10ACA000BDE8F081286840780028706814BF40F43F
:10ACB000007020F40070F0E7052A0FD17268736805
:10ACC000C2F3C01203F4007342EA53122B681A70E5
:10ACD00002700120C4F80C80087027700120BDE8C4
:10ACE000F08110B503F00702774C012A02D0022A46
:10ACF0000DD00AE004F07AF80021206200281ABF83
:10AD00004FF4056060626162E160002010BD636A1B
:10AD1000E2689A4228BF104607D2D4F820C01CF837
:10AD200002C080F800C0501CE060984204BF0120BF
:10AD30000870012010BD10B4DFF898C113F0070FA0
:10AD400004D003F00702022A13D00FE0012A04BF47
:10AD5000DCF8000040F0010006D0002A04BFDCF857
:10AD6000000020F0010001D1CCF8000010BC002050
:10AD70007047DCF80030002213F0010F18BF0122E9
:10AD8000534BD3F804C0544B1B68B3F8F030C3F3F3
:10AD90000334012303FA04F41CEA040F18BF42F041
:10ADA000020202700B7010BC0120704770B514468F
:10ADB0000E46054613F0070F04D003F007000228E3
:10ADC0000ED00BE0002C14BF0120002002F0E8FDA3
:10ADD00024B13F48016821F440510160002070BD5A
:10ADE00002F0E5FD002814BF012200222A70012094
:10ADF000307070BD2DE9F04103F0070C324C0F4666
:10AE00008046BCF1010F12D0314E13F0070F4FF006
:10AE1000030510D02046BCF1020F027826D0BCF109
:10AE2000040F02BFE0680128062A33D036E005206F
:10AE30002070002018E0E06810B1012804D011E073
:10AE40006270062020700DE07168607800EA0203ED
:10AE500019437160716820EA020291437160F9F749
:10AE60003DFA2570E068401CE06017E0E0680128CA
:10AE700008BF062A03D16078F9F746FA2570706892
:10AE800088F8000001203870E068401CE060012074
:10AE9000BDE8F0816078F9F737FA25700020BDE849
:10AEA000F08170B5044603F007000D4602281CBF70
:10AEB000002070BDFCF7F6FC002814BF0122002220
:10AEC00022700120287070BD9C810010D8410200C2
:10AED00000100040144C00402C83001070B50D464B
:10AEE000044613F0070F04D003F00700022805D032
:10AEF00002E0104607F05FFC002070BD07F05EFC2A
:10AF000020700120287070BD70B50D46044613F006
:10AF1000070F04D003F00700022805D002E0104616
:10AF2000F6F759F8002070BDF6F758F820700120A8
:10AF3000287070BD70B503F00702DFF834C40C460A
:10AF40000546012A08BF05200DD013F0070F08BFE2
:10AF5000062008D0022A09D0042A04BF9CF8000069
:10AF6000062809D00EE08CF800000BE0FCF7F1FC9D
:10AF700028700120207070BD03208CF80000012093
:10AF8000FCF7EAFC002070BD70B503F00702F84D35
:10AF90000E460446012A04BF0020E86001D0022AC0
:10AFA00001D0002070BD0FF014F8EA68002A04BF39
:10AFB000000A207004D0012A02D1207001203070D4
:10AFC000501CE860012070BD03F0070210B4E84B8C
:10AFD000012A04BF0020D86001D0022A02D010BC90
:10AFE00000207047DA68022A0CD24FF0010C002AC8
:10AFF00008BF80F800C005D0012A03D1682404707E
:10B0000081F800C0501CD86010BC0120704770B59A
:10B01000044603F007000D46022807D013F0070F7F
:10B0200004BF1046FCF73CFB002070BDFCF73BFB67
:10B0300020700120287070BD2DE9F04103F0070257
:10B040000027CB4E0C460546012A08BFF76001D009
:10B05000022A02D00020BDE8F08113F095FDF268CD
:10B06000002A04BF000A28700BD00121012A04BF66
:10B070002870217005D0022A03D1F76021700320C7
:10B080003070F068401CF0600120BDE8F0810020C5
:10B09000704710B503F00702B54C012A02D0022A0E
:10B0A00027D024E003F0A2FE0023002804BF23627F
:10B0B00063621BD000F1500121624168B1F5887FC5
:10B0C00090F820100CD390F8212001EB020C01FB2A
:10B0D00002C190F8222090F823001044084404E0B4
:10B0E00090F822000A1801FB00206062E360002053
:10B0F00010BD636AE2689A4228BF104607D2D4F8AE
:10B1000020C01CF802C080F800C0501CE0609842CB
:10B1100004BF01200870012010BD03F00702012ABE
:10B1200002D0022A05D002E091490020C860002028
:10B130007047012202700A701046704710B513F074
:10B14000070F04D003F00702022A05D002E01046E0
:10B1500001F0D4FD002010BD864A12780270012053
:10B16000087010BD10B513F0070F04D003F00702EC
:10B17000022A05D002E0104602F0B2F8002010BD0D
:10B180007D4A127802700120087010BD00207047BF
:10B1900003F00702764B012A04BF0020D86001D0DB
:10B1A000022A01D000207047DA684FF0010C002A13
:10B1B00008BF80F800C0501CD860012808BF81F883
:10B1C00000C0012070471FB513F0070F07D103F02F
:10B1D0000DFA20B1012202A90B2001F00DFA04B0F2
:10B1E000002010BD70B503F00700614C1546012822
:10B1F00004BF0020E06024D013F0070F21D103F03A
:10B20000F5F9F0B1E0685D4E03283CBF31680D549C
:10B21000401CE060032814D1F7F7D7FD3068B0F880
:10B22000010045BAF7F7EEFB040018BFF7F74EFF31
:10B23000306829460078F6F788FA002C18BFF7F72F
:10B2400048FF002070BD70B503F00700484D14465C
:10B25000012804BF0020E86020D013F0070F1DD1A3
:10B2600003F0C4F9D0B1E868444E02283CBF31680D
:10B270000C54401CE860022810D1F7F7A6FDF7F740
:10B28000C1FB040018BFF7F721FF30684178007850
:10B29000F6F707FB002C18BFF7F71BFF002070BD67
:10B2A00070B50D46044613F0070F04D003F00700F5
:10B2B000022805D002E01046F7F728FF002070BDF5
:10B2C000F7F727FF20700120287070BD7FB51C465E
:10B2D0000E46054613F0070F08D103F087F928B191
:10B2E000012202A9172001F087F903E004F007000A
:10B2F000022802D004B0002070BD07F010FB002827
:10B3000014BF012200222A700120307004B070BDE9
:10B310007FB51C460E46054613F0070F08D103F013
:10B3200065F928B1012202A9182001F065F903E0AE
:10B3300004F00700022802D004B0002070BD07F01E
:10B34000DBFA28700120307004B070BD2DE9F041A7
:10B3500003F0070C064C0E460746BCF1010F0FD058
:10B36000064D13F0070F0FD0BCF1020F21D01DE0E6
:10B370009C810010E5810010EA810010D841020094
:10B380000020E060206111E0E06803283CBF2968EC
:10B390000A54401CE060032808D12868B0F8010076
:10B3A00040BA01B228680078FDF7A3FF0020BDE88D
:10B3B000F0812269022A12D242B928680078FDF78A
:10B3C000AEFF2A68010A51702968887028682269CE
:10B3D0001044012A4078387004BF01203070206981
:10B3E000401C20610120BDE8F08110B503F007008A
:10B3F000F949012808BF00200CD013F0070FF74BC4
:10B4000002D0042808D018E0C86804283CBF1B6894
:10B410001A54401CC86010E0C86804280DD318688E
:10B42000196840788978000440EA01201968C978D1
:10B43000014318680078F8F7D9FA002010BD10B55C
:10B4400003F00702E44C012A02D0022A07D004E0EC
:10B450000020E060F9F725FBE061002010BDE26804
:10B46000042A07D2C2F10303D4F81CC0DB002CFA73
:10B4700003F30370501CE060042804BF012008702F
:10B48000012010BD10B503F00700012807D103F01B
:10B49000ADF820B1002211461D2001F0ADF80020CA
:10B4A00010BD2DE9F04103F00705CB4E1746884645
:10B4B0000446012D04BF0020F0601BD013F0070FDD
:10B4C00016D103F093F898B1F068C44B03283CBF41
:10B4D00019680F54401CF06003280BD1186890F9CC
:10B4E000022090F9011090F90000FAF747FF01E0FF
:10B4F000022D02D00020BDE8F081F06830B10128B3
:10B5000009D002280CD003280FD015E01420FAF738
:10B51000D9FD207010E01520FAF7D4FD20700BE063
:10B520001620FAF7CFFD207006E01720FAF7CAFDC3
:10B530002070012088F80000F068401CF0600120B5
:10B54000BDE8F08170B50D46044603F00700002108
:10B55000A14E012814BF13F0070FF16001D002289B
:10B5600001D0002070BDF06840B101280BD0022846
:10B570000ED0032811D0042814D019E00120FAF7C6
:10B58000A1FD207014E00220FAF79CFD20700FE06E
:10B590000320FAF797FD20700AE00420FAF792FDE5
:10B5A000207005E00520FAF78DFD2070012028703D
:10B5B000F068401CF060012070BD70B503F0070C0E
:10B5C0000026864C844DBCF1010F06D013F0070F06
:10B5D0000CD0BCF1020F1FD01CE007F0E7FAEE60C0
:10B5E000216808702168000A487013E0E8680228A2
:10B5F00003D221680A54401CE86002280AD1EE6098
:10B600002068007810F0010F04D002221920216870
:10B6100000F0F2FF002070BDEA68022A28BF104641
:10B6200004D223689B5C0370501CE860022804D19C
:10B630000120EE60087003202870012070BD7FB5E6
:10B640001C460E46054613F0070F08D102F0CEFF48
:10B6500028B1012202A9242000F0CEFF03E004F06B
:10B660000700022802D004B0002070BD0DF03EFD9E
:10B6700028700120307004B070BD7FB51C460E46A6
:10B68000054613F0070F08D102F0B0FF28B10122E0
:10B6900002A91F2000F0B0FF03E004F00700022819
:10B6A00002D004B0002070BD0DF02BFD28700120E9
:10B6B000307004B070BD7FB51C460E46054613F0D1
:10B6C000070F08D102F092FF28B1012202A923201E
:10B6D00000F092FF03E004F00700022802D004B05B
:10B6E000002070BD10F0B2FD28700120307004B051
:10B6F00070BD7FB51C460E46054613F0070F11D1ED
:10B7000002F074FF70B10DF008FD01469DF80800CD
:10B7100081420BD00DF0FEFC012202A91E2000F098
:10B720006BFF03E004F00700022802D004B0002001
:10B7300070BD0DF0F2FC28700120307004B070BDB7
:10B740002DE9FF41244E1C460F46054613F0070F16
:10B750001CD102F04BFFC8B19DF80800002818BFAB
:10B76000012802D0022807D014E0F070012202A9BB
:10B77000082000F041FF0DE0F07004208DF8080073
:10B78000012202A9082000F037FF03E004F00700BF
:10B79000022803D004B00020BDE8F081F0782870C2
:10B7A0000120387004B0BDE8F0817FB51C460D461D
:10B7B000064613F0070F08D102F018FF28B1012246
:10B7C00002A9082000F018FF03E004F00700022897
:10B7D00006D0002004B070BD9C810010D84102004A
:10B7E000FBF770FF801E052813D2DFE800F0030787
:10B7F0000E05100000240DE001240BE0022406F0E9
:10B80000AAF8042808BF052404E0032402E0042465
:10B8100000E0FF24347001202870DBE72DE9F041BF
:10B820001C4617460E46054613F0070F0BD102F0D3
:10B83000DDFE40B1384606F0B8FF00221146012077
:10B8400000F0DAFE03E004F00700022802D0002036
:10B85000BDE8F08106F0ACFF287001203070BDE833
:10B86000F08110B5104613F0070F08BF07F06AF813
:10B87000002010BD10B5104613F0070F08BF07F0E9
:10B8800068F8002010BD70B5044603F007000D46AF
:10B8900002281CBF002070BD07F063F82070012053
:10B8A000287070BD03F0070230B4FD4B4FF0000C60
:10B8B000012A05D0022A04BF1A78022A0BD01EE002
:10B8C00002201870F748C3F80CC06FF07F41006881
:10B8D000081AD86113E0DA68042A28BF104606D295
:10B8E000DD69D40025FA04F40470501CD8600428E3
:10B8F00005D10120C3F80CC008700320187030BCBB
:10B900000120704713F0070F04BFE74802700020C2
:10B91000704710B503F00700E149012804BF00207B
:10B92000C86013D013F0070F10D1C868DF4B04288C
:10B930003CBFD3F800C00CF80020401CC8600428AD
:10B9400004D104221220196800F056FE002010BD18
:10B950002DE9F0478C4603F007010024D04F16462E
:10B96000012904BFFC603C6162D013F0070FD04B8B
:10B97000DFF8408307D0022932D0042904BF387889
:10B9800006284DD055E0FD68002D08BF3E6224D04A
:10B99000012D06D0D7F81490AC1E4C4515D27CB9B9
:10B9A00008E0701C7861396A0844B0F5007F88BFF0
:10B9B0007C6112E04FF400721946BF4813F062F840
:10B9C000BA49386A096820440E54601C484504D1BD
:10B9D000B948C0F8FC8106203870681CF86028E07F
:10B9E000FF2101707B69C3B13A6A39690A44B2F533
:10B9F000007F10D2B14D2D68454518BF047004D1A9
:10BA000002F5783292F8002A0270481C984204BF6E
:10BA100001208CF80000481C38610120BDE8F08747
:10BA20001D461846F8F7EEFAA3492846F8F78CFBAE
:10BA30003C700020BDE8F0872DE9F047164603F082
:10BA400007020024964F012A04BFFC603C6164D0C9
:10BA5000DFF86C8213F0070F07D0022A33D0042AD4
:10BA600004BF387806284FD058E0FD68002D08BF85
:10BA70003E6225D0012D06D0D7F81490AC1E4C455F
:10BA800016D284B908E0701C7861396A0844B0F5B0
:10BA9000007F88BF7C6113E04FF400724FF47A316D
:10BAA000854812F0EFFF8149386A096820440E5436
:10BAB000601C484504D18048C0F8FC8106203870DD
:10BAC000681CF8602AE0FF2202707B69CBB1D7F8CE
:10BAD00020C03A699444BCF5007F10D2794D2D689E
:10BAE000454518BF047005D10CF5783C9CF800C89A
:10BAF00080F800C0501C984204BF01200870501C00
:10BB000038610120BDE8F0874FF47A30F8F77AFA0F
:10BB100069494FF47A30F8F717FB3C700020BDE814
:10BB2000F08770B503F007005D4C1546012804BF8F
:10BB30000020E06014D013F0070F11D102F056FD81
:10BB400070B1E068594902283CBF0A681554401C8E
:10BB5000E060022804D102220968052000F04CFDB3
:10BB6000002070BD2DE9F041054603F007004F4C61
:10BB70004B4E0F4601280AD013F0070F14D00228AD
:10BB80001BD0042804BF3078062834D03FE00020C2
:10BB9000F060216808702168487021688870216809
:10BBA000C8700520307032E0F06804282FD2216878
:10BBB0000A54401CF060062028E0F06860B906F0E6
:10BBC000E9FB216808702268010A51702268010CA3
:10BBD000000E91702168C870F06804283ABF21688F
:10BBE000095CFF21297024BF01213970401CF060DD
:10BBF0000120BDE8F08102F0F9FC40B12068C17875
:10BC0000006861F31F6006F0C0FB03203070002065
:10BC1000BDE8F081002070477FB51C460E46054602
:10BC200013F0070F08D102F0E1FC28B1012202A9AC
:10BC3000272000F0E1FC03E004F00700022802D016
:10BC400004B0002070BD06F0B8FE287001203070EE
:10BC500004B070BD03F007001149012808BF00209F
:10BC600009D013F0070F07D1C86818B9164B1B6825
:10BC70001A448A61401CC860002070472DE9F041D9
:10BC800003F00701064C1646054601291ED00E4F4B
:10BC900013F0070F38681DD0022930D02CE00000C7
:10BCA0009C810010B480001036800010D841020042
:10BCB00000EA0300554E564D54A50010FCEB03005E
:10BCC000324E564DFCE90300508300100020E06026
:10BCD000206111E0A56905F04DFE01280CD1A06995
:10BCE0003968884224BFD031814205D9E0680428F0
:10BCF00038BF2E54401CE0600020BDE8F081A669EA
:10BD000005F038FE50B1A26939688A4224BF01F1BA
:10BD1000D000904284BF2069305C00D8FF2028709A
:10BD20002069401C20610120BDE8F0817FB51C46E0
:10BD30000E46054613F0070F08D102F057FC28B154
:10BD4000012202A91B2000F057FC03E004F00700C9
:10BD5000022802D004B0002070BD06F01CFD28703F
:10BD60000120307004B070BD7FB51C460E460546FC
:10BD700013F0070F08D102F039FC28B1012202A903
:10BD8000112000F039FC03E004F00700022802D083
:10BD900004B0002070BD10F0C6F82870012030708B
:10BDA00004B070BD002070470020704770B50D468C
:10BDB000044613F0070F04D003F00700022805D053
:10BDC00002E0104609F045FE002070BD09F04DFE6E
:10BDD00020700120287070BD10B503F00702FF4CE1
:10BDE000FF4B4FF0000C012A02D0022A34D031E080
:10BDF000C3F80CC002F0FAFB00282BD0F94802F07F
:10BE00000DFD38B3F8480068007E10F0040FF548C7
:10BE100010D0C18C2268090A1170226890F826108F
:10BE20005170818C2268090A9170216890F8240071
:10BE3000C8700FE0818C2268090A1170226890F89E
:10BE400024105170C18C2268090A9170216890F801
:10BE50002600C870002010BDDA68042A28BF1046EA
:10BE600004D22468A45C0470501CD860042803D158
:10BE70000120C3F80CC00870012010BD70B503F09C
:10BE80000701D64DD64C012902D0022914D011E069
:10BE9000012001F08DFC0020E06001F09EFC20817B
:10BEA000296808702A68010A0028517004BF002020
:10BEB00001F07EFC002070BDE168022902D22A68F0
:10BEC000525C0270481CE060012070BD2DE9F04119
:10BED00003F007020026C24D0F460446012A02D095
:10BEE000022A09D005E005202870EE60288940006C
:10BEF00068610020BDE8F0812878052817D1EA683C
:10BF00006869824205D212F0010F1CBF6878207068
:10BF100010D0E868401CE8606969884207D10120B8
:10BF2000EE60387003202870002001F041FC0120F1
:10BF3000BDE8F08101F06AFC010A21706870E8E751
:10BF40001FB513F0070F04D1012202A91A2000F037
:10BF500053FB04B0002010BD002070470020704744
:10BF600003F007009E49012806D013F0070F04BF15
:10BF70000878012806D014E0012008700020C8606D
:10BF800088610DE0C868042805D28B69401C42EA2C
:10BF900003228A61C860042803D1032008708869DD
:10BFA00008620020704703F00700DFF834C2012860
:10BFB00007D013F0070F04BF9CF80000022809D037
:10BFC0001EE002208CF800000020CCF80C00CCF819
:10BFD0001C0015E0DCF80C00022808D2DCF81C106C
:10BFE000401C42EA0121CCF81C10CCF80C000228BD
:10BFF00006D1DCF81C00CCF8240003208CF80000EB
:10C000000020704770B403F007020025744C012A29
:10C0100002D0022A06D002E002202070E56070BC47
:10C02000002070472278022A1CD1D4F824C0E2688C
:10C03000624528BF10460ED212F0030F04D1236AC6
:10C0400053F8046BC4E90763237F0370E069000AB7
:10C05000E061501CE060604504D10120E56008709B
:10C060000320207070BC0120704770B503F00700FA
:10C0700000255B4C0E46012806D013F0070F04BFC5
:10C080002078022805D02BE002202070E560E561D1
:10C0900026E0616AE068884219D2E169090A41EA4A
:10C0A0000262401CE26110F0030FE0600FD1206AD1
:10C0B000B0F5802F28BF026006D2B0F5005F03D331
:10C0C00004224A49F8F794F8206A001D2062616A48
:10C0D000E068884204D10120E560307003202070C0
:10C0E000002070BD70B503F0070C00253C4CBCF17E
:10C0F000010F08BFE56039D013F0070F03D0BCF182
:10C10000020F35D032E0052A08BF39482DD005DCB2
:10C1100016D2DFE802F0171A1D2022003248202A2A
:10C12000006808BFF83020D006DC102A1DD0112A84
:10C1300008BF2C4819D003E0302A11D0312A12D080
:10C14000A56113E04FF400500FE04FF47F300CE096
:10C150004FF4443009E0274807E04FF47C3004E016
:10C1600001F0B4FC01E00FF06BFAA061002070BD9B
:10C17000E268042A07D2C2F10303D4F818C0DB0036
:10C180002CFA03F30370501CE060042824BF012044
:10C190000870012070BD70B403F0070C104DBCF1A5
:10C1A000010F07D00D4C13F0070F07D0BCF1020FA1
:10C1B00031D02DE00020E860286129E0E8680528FA
:10C1C0003CBF21680A54042820D123682268A96949
:10C1D000D3F8013012781BBA0EE00000D8410200FB
:10C1E0009C810010B83101102C830010B881001020
:10C1F00000EA030000EE0300D4F800C023F0FF03C0
:10C200009CF804C043EA0C0341F82230401CE8606B
:10C2100070BC002070472B6973B1042B07D22268D1
:10C22000032B1A445278027004BF01200870581C76
:10C23000286170BC012070472268D5F818C01278B8
:10C240005CF8222026684FEA126C86F801C0266846
:10C250004FEA124C86F802C026684FEA122C86F884
:10C2600003C0D4F800C08CF80420D8E710B503F060
:10C270000700012804D1002211460E2000F0BCF96D
:10C28000002010BD2DE9F04103F00704C74E17460A
:10C2900088460546012C04BF0020F06017D013F03B
:10C2A000070F12D102F0A2F978B1F068C049022854
:10C2B0003CBF0A681754401CF060022807D10222D4
:10C2C0000968072000F098F901E0022C02D0002054
:10C2D000BDE8F081F26812B1012A04D009E0FBF751
:10C2E000F1F9287005E0FBF7F3F92870012088F8D0
:10C2F0000000F068401CF0600120BDE8F08170B5DE
:10C3000003F007000025A94C012808D013F0070FFF
:10C310000BD0042804BF2078062825D02DE0A56185
:10C32000E5616570E560257027E0E068022807D2C6
:10C33000A16942EA0121A16161781144617010E0B4
:10C34000042807D2E16942EA0121E16161781144E0
:10C35000617006E0052804D261788A4204BF062194
:10C360002170401CE06008E0D4E9060101F048FCBF
:10C37000002804BF0120A0702570002070BD10B5FA
:10C380008A4C13F0070F07D003F00700042804BFFE
:10C390002078062822D02BE0E068022807D2A16985
:10C3A00042EA0121A16161781144617013E0814981
:10C3B000091808D27E490968014401F8022C617805
:10C3C0001144617007E07C49091804D261788A42FF
:10C3D00004BF06212170401CE06009E07749A06994
:10C3E00001F030FC002804BF0120A0700020207064
:10C3F000002010BD03F0070CBCF1010F00D0BEE718
:10C400006A49002088614870C8600870704730B47D
:10C4100003F007050024DFF894C1012D07D013F0C5
:10C42000070F0DD0022D3CD0042D54D06FE0CCF876
:10C430001840CCF81C40CCF80C408CF8004066E06A
:10C44000DCF80C0002280BD2DCF8181042EA0121BB
:10C45000CCF818109CF8011011448CF8011019E068
:10C46000042817D2DCF81C10032842EA0121CCF87A
:10C470001C109CF801301A448CF801200AD10622C5
:10C480008CF80020DCF81820114304BF4FF4007131
:10C49000CCF81C104A49401CCCF82C10CCF80C00ED
:10C4A00035E0DCF80C20042A28BF10460AD2C2F17D
:10C4B0000303DCF82C50DB0025FA03F30370501C57
:10C4C000CCF80C00042803D10120CCF80C400870F3
:10C4D00030BC012070479CF80000062815D1DCF81C
:10C4E000180000224102DCF81C0043021046B2EBA7
:10C4F000930F06D251F8045B401C2A44B0EB930F13
:10C50000F8D3CCF82C208CF80040CCF80C4030BC90
:10C51000002070472DE9F04103F0070490460E46D5
:10C520000746012C04D0274D13F0070F05D00BE070
:10C530001E480021C160417008E002F057F8002851
:10C5400018BF85F8008001D1022C02D00020BDE880
:10C55000F0812878387001203070BDE8F08170B526
:10C560000D46044613F0070F04D003F0070002281D
:10C5700005D002E0104609F0E6FC002070BD09F08D
:10C58000DFFC20700120287070BD4FF47F300168FF
:10C59000880A424211EB822218BF401C404201EB44
:10C5A0008000C01C20F00300704700009C81001038
:10C5B000D8410200FEFDFFFFFDFDFFFF54A5001066
:10C5C000EFBEADDEC4ED0010F848002202704270EC
:10C5D000827002714271C270DFF8D4C3114601EB60
:10C5E000410300200CEB43031A54401C0628FBD3E4
:10C5F000491C2029F3D3704712F0CBBA2DE9F04142
:10C6000015460E460746F8F761F900F008040820C1
:10C61000F8F757F92A463146384612F0BAFA054675
:10C620002046F8F749F92846BDE8F081DF488078D0
:10C630007047DE4840787047DC49002048707047FA
:10C64000DA49CA681043C860704710B568B1F8F796
:10C6500073FD7820F4F7D3FCD648F8F78FFEF8F78F
:10C6600072FEBDE81040F8F7F5BDF8F7FCFDF8F7ED
:10C6700077FE0020F8F782FEBDE81040F8F73EBDD7
:10C68000CA4910B508208871FBF71CF8AFF24500C5
:10C69000BDE81040F6F7ACBC2DE9F0474FF00008BC
:10C6A000F6F7AEFCDFF804A30446DAF80C00C14646
:10C6B00040B1DAF80C0010F0400F18BF44F0040449
:10C6C000CAF80C9014F00F0650D00127FAF7FAFFC1
:10C6D00005463046F6F797FC012E1DD0FAF7F8FF15
:10C6E00044EA0064002322460321072005F03EF8B7
:10C6F00014F0050F14BF00200120F3F73DFE14F0E5
:10C70000060F33D04FF0010806F063F80646022DFD
:10C7100018D0052D0AD029E09AF80600854208BFF6
:10C7200000278AF80650002FD8D1E8E714F0020F4E
:10C730000ED1A14C206858B10120F9F7E8FAC4F8ED
:10C74000009005E014F0020F1CBF0120F9F7DFFA9A
:10C7500001F0C8FA002818BF01F0CBFA022E05D06C
:10C76000022D4FF0020004D001F09CFA4046BDE8D3
:10C77000F08706F0D9F8F9E72DE9F84F0027F8F728
:10C7800060FEFAF79FFF022804D101F0EBFE0028BB
:10C7900018BF0127FFF780FF002818BF0127DFF827
:10C7A0000C9299F80200002800F02F82D9F80800B6
:10C7B0006D464FF0FF34002640B1D9F80820002321
:10C7C0000121084604F0D2FFC9F80860F8F77EF8A6
:10C7D00000F0080A0820F8F774F899F80300DFF869
:10C7E000D0B100B399F8050000EB4001401CC0B285
:10C7F0000BEB410189F80500202828BF89F8056066
:10C8000099F80300401E89F803004C7891F80080E5
:10C810000020002C05DD0A1892782A54401C84421E
:10C82000F9DC0E704E705046F8F746F8002CC0F256
:10C83000DC8108F0FF000024282880F09381DFE8E5
:10C8400000F0872914212C3B1848F74D87888EC7A4
:10C85000F6939CA6F587878787DBF8FDF287F1F0D2
:10C8600087EFEEED87ECEB87EAA10020F9F74FFAAE
:10C8700010E09DF80000AC280CBF01200220FAF760
:10C88000E9FF07E09DF800100120FAF736FF0120CC
:10C8900089F80100012400F065B99DF803100098A3
:10C8A00061F31F6001F0CAFF01210320FAF725FFA1
:10C8B000012089F80100EDE7BDF8000040BA05F05D
:10C8C0006CFD02210320FAF718FF012089F801000E
:10C8D000E0E79DF801109DF800008AE04FF0010AA2
:10C8E00089F801A099F8000080BBF6F779FB68B3DE
:10C8F0009DF8005089F800A0FAF7E4FE012808BF6F
:10C90000002515F0040F18BFFCF76EFD15F0020F9F
:10C9100006D01F20FBF7E4FEF9F7BBFA45F001054E
:10C9200015F0010F10D0FAF7CDFE022802D105F064
:10C9300050FF48B1FAF7C6FE052802D101F0BDF953
:10C9400010B10020F9F791FA89F8006089F80160C8
:10C9500008E19DF80000401E01F03AFC9AE79DF8BE
:10C96000000006F004F895E79DF8000010F00F00B5
:10C9700018BF01200BF025FFF4E09DF800000BF03C
:10C9800016FFEFE09DF8000006F00BF8EAE09DF8D6
:10C99000000010B1012811D0E4E000200FF0C0FA2F
:10C9A00000200EF04FFE00200FE00000D4810010A8
:10C9B00054A70010F1E500003C82001001200FF0A8
:10C9C000AFFA03200EF03EFE02200EF05EFEC9E03C
:10C9D0009DF8000058B1FAF775FE022818BF01242F
:10C9E00005F0AAFF01460220FAF787FEBAE000210F
:10C9F0000620FAF782FE4DE79DF80000002818BFD8
:10CA0000012005F082FF9DF80000002818BF0120DA
:10CA100001F03EF9A6E0A1E099E093E062E05CE07D
:10CA20006CE057E063E00EE008E002E047E01CE065
:10CA30002DE09DF8000005F054FF93E0BDF80000E4
:10CA400006F02EF826E79DF8000020B1012840D01E
:10CA5000022805D086E04FF47F30F7F7D3FA81E063
:10CA600001F01CFE00210420C3E7F7F72FFF00F0C0
:10CA700008040820F7F725FF99F80300002808BFED
:10CA800089F802602046F7F717FF0121B0E79DF80B
:10CA90000000062805D2DFE800F004070A0C030FA7
:10CAA000A5E702210846A4E702210520A1E700210D
:10CAB00003E0002104209CE70421032099E79DF86E
:10CAC0000300009A002360F31F626221072004F034
:10CAD0004DFE47E0F9F7E6FCDCE69DF8000006F0C5
:10CAE0008BF8D7E69DF8000006F08EF8D2E69DF8A8
:10CAF000000000F00100FAF717FFCBE60CF001FB95
:10CB00009DF8004006F052F8012C13D0022C14D0EE
:10CB1000042C18BF082C7FF4BDAE40F0005005F087
:10CB200074FF042C18BF082C7FF4B4AE20460CF020
:10CB3000E3FAAFE605F069FFF8E740F0805005F052
:10CB400064FFF3E79DF800000FF083FB0AE09DF817
:10CB500000000CF0C8FA05F072FE03E09DF800003A
:10CB600000F06BF90CB101273FE0D9F808006D46E1
:10CB70004FF0FF3440B1D9F80820002301210846C6
:10CB800004F0F4FDC9F80860F7F7A0FE00F0080A09
:10CB90000820F7F796FE99F8030000B399F805000E
:10CBA00000EB4001401CC0B20BEB410189F80500CD
:10CBB000202828BF89F8056099F80300401E89F8ED
:10CBC00003004C7891F800800020002C05DD0A1845
:10CBD00092782A54401C8442F9DC0E704E70504604
:10CBE000F7F76AFE002CBFF624AEF7F76FFE00F0F1
:10CBF00008040820F7F765FE99F80310002908BF1C
:10CC000089F802602046F7F757FE002F14BF012075
:10CC10000020BDE8F88F000002460020022928BF4E
:10CC2000704752B1012A18BF704701EB4100C0EBB9
:10CC30004110FE4901EB8000704740F2DB10484391
:10CC4000FB49F7E770B5F7F741FE00F0080608204A
:10CC5000F7F737FEF74C00256078FF2806D240F63C
:10CC6000D861F34811F013FFA570E570A079FF2893
:10CC700005D2E821ED4811F00AFFE5712572304632
:10CC8000BDE87040F7F718BEDFF8ACC300FB01F356
:10CC90001CEB030C88BF7047E64BDA61C3E9050162
:10CCA0007047DFF890C30028DCF8143018BF036029
:10CCB000E0480029806918BF0860002A1CBFDCF822
:10CCC0001C10116058437047DA4801210171007847
:10CCD00040F2DB1180F001004843D54901EB8000B0
:10CCE0007047D4488278002132B1C27822B90278E4
:10CCF00082F001020270817001717047CD491E28D7
:10CD00004A78487008BF002003D01F2808BF0120C0
:10CD100000D1087010467047C648007840F2DB1119
:10CD200080F001004843C24901EB800070472DE9C3
:10CD3000F003DFF800C357009CF8004040F2DB1519
:10CD40006C43BB4DDCF8148005EB840403FB08F551
:10CD500004EB4504884534BF45460D46DCF818C051
:10CD6000ACEB0303934238BF1A464FF00009002A88
:10CD70008EBF0026BDE8F00370470023002D06D9C2
:10CD800030F813C024F813C05B1C9D42F8D8AC46A1
:10CD9000BD4205D224F81C600CF1010CBC45F9D34E
:10CDA00009F1010904EB480400EB41009145E4D38B
:10CDB000BDE8F00370472DE9F0419E4F14468C46C4
:10CDC00001467A7806981D468A4218BFBDE8F08170
:10CDD0000121F970012802D0022824D029E03878F6
:10CDE00040F2DB11484392497E6901EB8001A64283
:10CDF00034BF32462246B869A84238BF05460023F0
:10CE0000002D16D90020002A06D91CF8007021F840
:10CE10001070401C8242F8D85B1C01EB4601A44410
:10CE2000AB42EFD305E000232A4621466046FFF7D8
:10CE30007EFFBDE8F04100F036BD7E4A0128114674
:10CE40009072497808BF242004D0002806BF242906
:10CE5000FF207047507070477648807A704770B4F2
:10CE6000DFF8D8C1DCF800C0DCF818C01CF0040FF3
:10CE70001ABF012424EA0C060CF0010605680C68B0
:10CE8000002E1CBF1B1B5C1E1CF0020F1CBF521B84
:10CE9000551E1CF0040F19BF04600D6005600C6086
:10CEA00070BC7047002808BF70476249644B4A78DD
:10CEB00064491B88002A097818BF022A05D0042A71
:10CEC00018BF092A01D0012231E7012200F005BD77
:10CED0002DE9F04F574B93B00121D970DFF870C1A5
:10CEE00059495A4ABCF80070DFF854C15B78097898
:10CEF0001278BCF80090392B2DD2DFE803F01D64C6
:10CF00001D641D2C6464641D646464642C646E6E12
:10CF10006E6E642C2C2C2C2C2C2C2C642C2C2CFE8B
:10CF2000FE2CFD2C2C2C2C2C2C2C2C2C2C2C2C2C9E
:10CF30002C64646464646400464B1B78012B03D941
:10CF40004549464A0978127800281CBF002300F0A2
:10CF5000C4FC00F0A5B9002800F0A281354E0D46B2
:10CF6000317840F2DB135943314BD6F814C0002717
:10CF700003EB8103AC452CBF2C466446B16991425A
:10CF800038BF0A465FEA02084FF0000600F08881C9
:10CF90000021002C06D930F8112023F81120491C5B
:10CFA0008C42F8D82246644504D823F81270521CEB
:10CFB0006245FAD9761C03EB4C0300EB450046456D
:10CFC000E6D300F06DB9002800F06A8100234A46DC
:10CFD0003946FFF7ACFE00F063B9F5F7F6FEF5F75A
:10CFE00011FD0090002818BFF6F770F81948007876
:10CFF000012884BF194890F80090F5F7FEFF10F063
:10D00000020F18BF09F10109DFF854B000200290A7
:10D01000084890F801A0017840F2DB124A43044925
:10D02000406901EB8205B8421CE00000ECB600103C
:10D0300014A80010E48100104AFCFFFF2C830010AC
:10D0400058810010558100104C8100104D81001056
:10D05000568100104E8100104F8100105081001049
:10D060000000013038BF0746F6F7DDF801900020D8
:10D07000F6F742FD0026B9F1000F41DD0024002F34
:10D08000C4BF06EB460000EB061823DD01980057ED
:10D09000262824BF002025F8140018D200F0010132
:10D0A0000BEB813100EBD07001EB88014010BAF13D
:10D0B000100F51F820003CD0BAF1110F40D0BAF156
:10D0C000120F0CBFC0B2F6F71DFD25F81400641C4A
:10D0D000BC42DBDBFE49384649698F4298BF0022DB
:10D0E00004D825F81020401C8842FAD9F948761C4B
:10D0F000007805EB400501E031E027E04E45BDDB5F
:10D10000F348017840F2DB124A43F349406901EBEE
:10D11000820202994843F14902EB40000A78ED4946
:10D12000097811F0D2FC0098002818BFF5F7D1FF5C
:10D13000B6E010F4003FC0F34230C6D04042C4E72E
:10D1400010F4803FC0F30420F8D1BEE700287DD062
:10D15000002309F102023946FFF7E9FDA0E00028AB
:10D1600074D00646DE483D460068007E10F0040F8D
:10D170000EBF3C464C46B946032300934FEA590282
:10D1800061080993201F0A930B930C92CDE90110BB
:10D190000D920E92CDE90331A9F104020F92109283
:10D1A000CDE905031192CDE907104B46224609A9A6
:10D1B0006846FFF754FE4B46224609AF0AA9E846E7
:10D1C00001A8FFF74CFE4B46224607F1080108F183
:10D1D0000800FFF744FE4B46224607F10C0108F118
:10D1E0000C00FFF73CFE4B46224607F1100108F108
:10D1F0001000FFF734FE4B46224607F1140108F1F8
:10D200001400FFF72CFE4B46224607F1180108F1E7
:10D210001800FFF724FE4B46224607F11C0108F1D7
:10D220001C00FFF71CFE4B46224607F1200108F1C7
:10D230002000FFF714FEA648007840F2DB114843B7
:10D24000A549002201EB8000914600E028E020F88B
:10D25000129058F82210A1F1010C491C61451CD311
:10D2600057F822104B1E491C99420FD303FB05C1EE
:10D2700036F9114030F912108C42C8BF20F8124024
:10D2800057F822105B1C491C9942EFD258F8221023
:10D290000CF1010C491C6145E2D2521C092AD4D37D
:10D2A00013B0BDE8F04F00F0FEBA89480121417289
:10D2B000407980F0010000EB4001C1EB401089494A
:10D2C00001EB800070478248C279002132B1027AB6
:10D2D00022B9427982F001024271C17141727047F4
:10D2E0007B491E288A79887108BF002003D01F2837
:10D2F00008BF012000D1487110467047744840793A
:10D3000080F0010000EB4001C1EB4010754901EBDA
:10D31000800070472DE9F04F7349DFF8B48185B084
:10D320000F7872490E78012188F8081098F80610D5
:10D330006C4CDFF8ACC14FF00009092900F01381F3
:10D3400049DC002918BF022900F00D81042918BF0B
:10D35000052900F00881F8B198F80510730001EB79
:10D360004102C2EB411104EB8102002113EB57048F
:10D3700012D0DCF800301B8A5B08002E03BF30F8A7
:10D3800011500B4422F8135030F8113018BF22F816
:10D390001130491C8C42ECD8F7F798FA00F00804D9
:10D3A0000820F7F78EFA98F80900002801BF98F8CE
:10D3B000050080F0010088F8050088F807901CBF80
:10D3C000012088F807002046F7F776FA88F80890D9
:10D3D00005B0BDE8F08F102918BF112903D012291C
:10D3E00018BF1329B7D1F5F7F0FCF5F70BFB029046
:10D3F000002818BFF5F76AFE98F80650D8F8200004
:10D40000009098F8050000EB4001C1EB401004EBE0
:10D41000800BF4F783FB00287AD01120F3F77FFB11
:10D4200000280CBF1220112060F3070A0120F3F737
:10D4300076FB002814BF0120022060F30F2A0AF0B7
:10D44000FF000190F6F758FBF5F7EBFE0024039080
:10D45000002E1FD903980257142AA8BF143A02DAE3
:10D460000A2AA8BF1232262A28BF2BF814900ED2FF
:10D47000DDE90010F5F748F9102D5AD0112D5FD0D5
:10D48000122D0CBFC0B2F6F73DFB2BF81400641C44
:10D49000B442DFD30BEB4606CAF3072B5846F6F728
:10D4A0002BFBF5F7C0FE00248246002F2AD91AF97B
:10D4B0000420262A28BF26F8149020D25846009926
:10D4C000F5F722F9102D41D0112D46D0122D10E084
:10D4D000E48100104C81001014A800104D81001050
:10D4E0002C830010ECB60010518100105281001006
:10D4F0000EE00CBFC0B2F6F705FB26F81400641C62
:10D50000BC42D4D30298002818BFF5F7E2FD43E7E8
:10D510000120F3F704FB002814BF0120022060F370
:10D52000070A1120F3F7FBFA002814BF112012207C
:10D5300083E710F4003FC0F34230A6D04042A4E796
:10D5400010F4803FC0F30420F8D19EE710F4003FB0
:10D55000C0F34230D1D04042CFE710F4803FC0F357
:10D560000420F8D1C9E700283FF416AF98F8051059
:10D5700001EB4102C2EB411104EB81020021F419DD
:10D580003FF40AAFDCF80030002E5B8A03BF30F8AE
:10D5900011500B4422F8135030F8113018BF22F804
:10D5A0001130491C8C42EDD8F6E670B50D46F449B1
:10D5B0000122CA70F34A49781688F34A212914884F
:10D5C0001EBF2229232970BD002818BF002D11D0AD
:10D5D000002322463146FFF7AAFB631C01222146A5
:10D5E0002846FFF7A4FB05EB4400A31C01223146AB
:10D5F000FFF79DFBBDE8704000F055B970B50446DB
:10D60000C068DF4D40B1697831B9DF4901220B882C
:10D61000DE49097800F061F9A06820B16978002935
:10D6200008BFFFF755FC6878102804BF0020FFF7FB
:10D630004FFC6878112804BF0020FFF749FC687888
:10D64000122804BF0020FFF743FC6878132804BFAA
:10D650000020FFF73DFC206920B1A979002908BF0F
:10D66000FFF758FEA879102804BF0020FFF752FEEC
:10D67000A879112804BF0020FFF74CFEA8791228D2
:10D6800004BF0020FFF746FEA879132818BF70BD1D
:10D690000020BDE870403DE62DE9F04F83B0924692
:10D6A0000D4680460BF09FFC01900BF0A0FC009013
:10D6B00001980026B0FBF5F10098DFF8C49201FB59
:10D6C00000F70120344689F8030099F80C0099F816
:10D6D0000010DFF8BCB288420ED040F2DB114843A4
:10D6E0000BEB800199F8000040F2DB1250430BEB8A
:10D6F0008000920011F0D5F9BAF1000F2CD999F8F9
:10D700000DC00099BCFBF1F001FB10C2019951431F
:10D7100000FB05110020002D11D938F8142099F8CC
:10D72000003040F2DB1E03FB0EF301EB000E0BEBAF
:10D730008303401C641C23F81E208542EDD80CF1A5
:10D740000100C0B289F80D00B84224BF002089F85A
:10D750000D00761C5645D2D399F80D00401EC0B27C
:10D7600089F80D0087429CBF781E89F80D0099F852
:10D77000000089F80C0003B0BDE8F04F00F093B84A
:10D780007F48017800F1240281F0010132F8111084
:10D79000002918BF7047017881F001010170002154
:10D7A000C181037822F813107A4A00781154704727
:10D7B0007349C87270477248C07A704770B5704C30
:10D7C00000252570E572E581258240F6D861704814
:10D7D00011F05DF96562658270BD694908780022C3
:10D7E0000A8280F001001231095C69B140F2DB115C
:10D7F000674A414332F82110A1F55062B63A02BFA0
:10D80000654931F810007047002070475C4B18786C
:10D8100003F1120C80F001014FF6FF701CF801209B
:10D82000012A18BF704740F2DB104843584A02EB08
:10D8300080001A8A30F81200521C1A82564B33F8B4
:10D840001120521E1204120C23F8112004BF0022D2
:10D850000CF8012070475049A1F12402137801EB24
:10D8600043010B8803440B8092F800C0012102F1B0
:10D87000120303F80C10D1890844D0817047404A44
:10D88000D38903EB5000454B01445B1824BF0020B3
:10D890007047117840F2DB1251433D4A02EB81019F
:10D8A00001EB4000704770B5F7F710F800F008067C
:10D8B0000820F7F706F8324C20790025002801BF30
:10D8C000207880F001002070A5701CBF0120A0709E
:10D8D0003046F6F7F1FFE57070BD2DE9F0479A4646
:10D8E00090460F460646F5F7A3FC5FEA00091FD0F5
:10D8F0002349087840F2DB125043254A4D6902EB78
:10D9000080000AFB05F200EB4204AF4294BF3846A8
:10D9100028468969A1EB0A01414538BF88464FF086
:10D92000000AB8F1000F88BF002109D8BDE8F087D0
:10D930005346424639463046BDE8F047FFF7F7B94F
:10D940000023002808D919F9032036F8122024F8FA
:10D9500013205B1C9842F6D88446A84205D824F8C8
:10D960001C100CF1010CAC45F9D90AF1010A04EBC9
:10D97000450406EB4706C245E2D3BDE8F087000048
:10D98000E48100105681001058810010558100106C
:10D9900014A80010F6810010088200104AFCFFFF56
:10D9A0004149002814BF00200120087070473E48FC
:10D9B000007800280CBF01200020704701203A4960
:10D9C00048707047384800214170017800291ABF1B
:10D9D0004068002870473548016821F00101016066
:10D9E00070473148017821B130490A6842F001029C
:10D9F0000A60002141608160C160016170472A486E
:10DA0000017821B129490A6842F001020A60002127
:10DA100041608160C1600161704700B50178427862
:10DA200085B0890141EA82018DF800104188090919
:10DA30008DF80110818809098DF80210817801F0B4
:10DA40000F02017962F31F118DF80310017A8DF82E
:10DA50000410417A8DF805108179C27901F03F01F7
:10DA600002F00C0241EA02118DF80610C179827AA7
:10DA7000890102F0010241EA42118DF80710C17BD1
:10DA80008DF80810017C8DF80910407C00F00F0023
:10DA90008DF80A0000208DF80B000390684611F005
:10DAA0007DF805B000BD00000C820010144C004051
:10DAB000002818BF47484849886370474648806B2C
:10DAC000444988420CBF01200020704742487047FB
:10DAD000424B4FF0000C1C681B1F1D683E4B196029
:10DAE0005A603F49D963DC6214F0804F22D0290C80
:10DAF0005985290A83F8291083F82850598D19B1BE
:10DB0000598D012242EA014C93F8291039B193F85A
:10DB10002910022242EA014C32490C681C6393F836
:10DB2000281039B193F82810032242EA014C2E49FB
:10DB30000C685C632D490C60091DC1F800C02C4ABB
:10DB400081691160B0E816109960DA601C61C3F851
:10DB500014C090E807109861D9611A62C3F824C014
:10DB6000986B1C49884202D1234922480860FEE78D
:10DB70002249012804BF09607047022818BF704776
:10DB800008471548D0F8EC201C498A4204BFD0F859
:10DB9000F0208A4208D1D0F8F4208A4201BFD0F8A0
:10DBA000F8208A4201207047C0F8EC10C0F8F0104D
:10DBB000C0F8F410C0F8F8100020704706480F496C
:10DBC000C0F8EC10C0F8F010C0F8F410C0F8F8106D
:10DBD00070470000504D5544005F01102CED00E0EF
:10DBE000544C414638ED00E034ED00E0344C004048
:10DBF0003C4C0040AD2007B0304C0040ADDEADDE07
:10DC000070B50E460446F9F75DFD042811D1A4F560
:10DC1000BC7088280DD2A019A0F27910882808D2EB
:10DC200065020024002E04D92846F6F7EBF90128F6
:10DC300001D0002070BD641C05F50075B442F3D31B
:10DC4000012070BD70B50D460446F9F73BFD042870
:10DC50000AD1A4F5BC70882806D260022946F6F7DE
:10DC600073FA012808BF70BD002070BD10B5074CC5
:10DC7000FEF782FD012808BF10BD206800F0BFFD3F
:10DC8000002818BFF9F780FDF2E700002C83001090
:10DC9000F14A0028516814BF41F0010021F0010051
:10DCA00050607047EC4B59680A0E120721F07F4113
:10DCB00042EA0060084358607047E7484068C0F394
:10DCC00003607047E4484068000F7047E248322123
:10DCD000C0684843E149A1FB001080087047DE4856
:10DCE00000697047DC48006A7047DB490120086220
:10DCF0007047D949002008627047D74800787047BC
:10DD0000002818BF0120D44908707047D248406AE3
:10DD10007047D14800214162017070472DE9F04100
:10DD200086B040F20F31F9F78CFE002804BF06B030
:10DD3000BDE8F08110F037FF10F03AFFF7F768FF09
:10DD40005FEA000872D1F3F7F9FBC548F4F7A5FEC6
:10DD50000120F4F795FEF6F7DBFDC248F6F78DFEDD
:10DD6000F6F774FEF6F79DFEBF4E4000BA4D3168DF
:10DD7000B1F80E21B0FBF2F0401CC0F34F006880F8
:10DD800091F8101111F0FF0169700AD0F6F789FEC1
:10DD900031684000B1F80C11B0FBF1F0401CC0F349
:10DDA0004F00F6F7EEFDB14F17203860306890F85D
:10DDB0001E01A860F5F709F8F4F724FE002808BF53
:10DDC000F5F768F9687838B1401E10F0FF00687008
:10DDD00004BF6888F6F7D5FD6868C0F30364214680
:10DDE0000520F2F77EFAFEF7C7FC012807D0686825
:10DDF000C0F30360A04208BFB8F1000F1FD0F5F7D1
:10DE000076FC00203860F6F70CFE40B1F6F7F1FD25
:10DE1000F6F727FE0020F6F730FEF6F786FDF4F75A
:10DE2000D4FFF4F7F1FD0020F4F737FE10F0C0FE48
:10DE300010F0C3FEF9F7A3FF06B0BDE8F081684615
:10DE4000F5F7FEFB98B16846FFF7D8FBF9F73AFC07
:10DE50002146009A07F01CFD684610F0B3FE80468C
:10DE600007F08CFDF5F743FCF9F7A4FCBBE730683D
:10DE7000D0F8B00010F0704F02D0F9F785FCB2E78F
:10DE8000F9F79FFCAFE770B50546002404F0AEFD3E
:10DE900070B10BF036F908280AD0754800EB051070
:10DEA000C1686D48426B91421CBF0121816301240E
:10DEB000204670BD6E4A014602EB01110020CA687F
:10DEC00065494B6B9A4208BF7047012088637047D1
:10DED0002DE9F047DFF8909180005F4FD9F80010EE
:10DEE00000242646D1F8001121FA00F000F00F00BE
:10DEF000C1F30321C7E90A01884218BFBDE8F087D2
:10DF00000020DFF86C81B863D9F80000D0F8001168
:10DF100008EB041002799200D14001F00F050F2D9B
:10DF200004D0816820468847012806D0641C022C52
:10DF3000EAD3B86B01280AD102E02646BD62F8E7B1
:10DF400008EB0610C06878630020F7F7E0FE396B35
:10DF5000B86A814218BF3863BDE8F0872DE9F04107
:10DF600041480068B0F91611B0F9140110F0FDFD38
:10DF7000F2F775FC0120F7F7CAFE00200BF0CAF893
:10DF80000EF054F90420FFF7A3FFF7F77EFE002000
:10DF900004F090FE304D002601202E616E61C5E92F
:10DFA000066004F06DFF01200DF06FFB01200DF005
:10DFB00086FB10F00CFE0020EE6004F0ECFCF9F79C
:10DFC00081FB05282AD16868010FC0F30364A142D0
:10DFD00002D02E616E61AE612046FFF779FF0746E1
:10DFE0002146052003F086FC74B3022C28D0042CB3
:10DFF0002ED068680E2C4FEA106120F07F404FEA67
:10E00000017118BF41F0007108436860FEF7B4FB6E
:10E01000012803D0F9F756FB0528D4D00DF0A5FF51
:10E02000144C6068C0F3402004F0B5FCF7F76EFEB6
:10E030000EF003F9606820F400706060BDE8F081C4
:10E040003846FFF76BFEE1E7384610F0C5FDDDE727
:10E05000384604F0AFFFD9E720820010ABAAAAAA85
:10E0600071590010EB4E00102C8300101048004036
:10E070005C820010001000407047002808BF704705
:10E0800080220146014810F0FDBC7047D4BF00104B
:10E09000704705283CBFFE49087070470020FC49C6
:10E0A00088604860FB48006890F8CD00052838BFBC
:10E0B000087070470020F64948607047F4480078BF
:10E0C000704770B5F34D0024286890F8B80010F040
:10E0D000020F0BD0F9F7F6FA022807D1EC482968AD
:10E0E000007801EB8000B0F8D00084B2204670BD0B
:10E0F00070B5E84D4FF48054286890F8B80010F0DF
:10E10000020F0DD0F9F7DEFA022809D1E04829689C
:10E11000007801EB8000D0F8D000000CC0F31304AD
:10E12000204670BDDA488078002818BF012070476B
:10E130002DE9F041F9F7C6FA022803D104F049FBB2
:10E14000022803D04FF48050BDE8F0814FF4805591
:10E150002E4604F009FCDFF83C830446CC4FD8F887
:10E16000000090F8B81011F0010F0CD0B0F8C20008
:10E17000B9684042814206DC2CB10020641EB860C0
:10E18000204604F0F4FBD8F8001091F8B80010F025
:10E19000040F18BF002C0AD0B1F8C800621E9040CE
:10E1A000B1F8CA20824238BF1046C0F31306D1F836
:10E1B000F00010F0020F1CBFB978002902D0000C4B
:10E1C000C0F31305B54298BF35462846BDE8F08137
:10E1D0002DE9F04FDFF8BCA287B0DAF8001091F813
:10E1E000B82012F0020F0DD0DFF8A4B291F8CC9055
:10E1F00000289BF8007009DB484503D2B84218BFDD
:10E20000064643D107B00020BDE8F08F3E464FF0F0
:10E21000FF38F4F7F9FBF5F7BAFC0025B9F1000F68
:10E2200034D9DAF80000002400EB8500B0F8D00003
:10E2300081B22046F3F789FAF4F72CFF6846F5F728
:10E24000FFF9002863D0029878B10146924802781D
:10E25000924800785043421E07D331F9020B002840
:10E26000B8BF40420444521EF7D2F5F740FAF4F723
:10E27000CBFB002322469221072003F077FAA0452A
:10E2800084BF2E46A0466D1C4D45CAD3B74241D02F
:10E29000052E38BF8BF80060DAF80000B0F8CE1019
:10E2A00021B300EB870200EB8600B2F8D020B0F873
:10E2B000D00092B280B2801A484340F30F34F7F78F
:10E2C00041F9774BDFF8DCC100211A88BCF8005017
:10E2D0006A430BD030F81120224420F811201A880C
:10E2E000BCF80050491C6A438A42F3D84FF48000BE
:10E2F00004F093FCDAF80000002300EB8600802194
:10E30000B0F8D00082B2072003F030FA09E0F9F744
:10E310003BFA93E704F028FB03283CBF401C04F0C1
:10E3200026FB012007B0BDE8F08F5A485849006825
:10E33000B0F8C200424288688242BCBF401E88607A
:10E3400070472DE9F04F93B093460E4604464FF0C8
:10E35000000A04F009FBDFF83C814D4F0500D1466F
:10E3600010D110F03EFCD8F80010B1F8C41088426B
:10E3700008D30120C7F8089004F0F9FA13B001207F
:10E38000BDE8F08F002E1FDDB8680028B8BFC7F8C1
:10E39000089007DBD8F80010B1F8C0108842BCBF65
:10E3A000401CB860D8F80000B968B0F8C0008842D6
:10E3B00015DC032D13D2681CC7F8089004F0D7FAB7
:10E3C00013B00120BDE8F08F09D1D8F80000B0F8F3
:10E3D000C2004142B8688842C4BF401EB860B878E5
:10E3E00050B1D8F8000090F8F00010F0040F1EBFF4
:10E3F000002013B0BDE8F08FD8F80000B0F9BE10CF
:10E400008C420EDD796821447960B0F8BA00884208
:10E4100010DC4FF0FF30C7F80490FFF7D9FE8246BA
:10E4200008E07868002805DD002CD4BF01212146D2
:10E43000401A7860DFF8709099F8000007283CD106
:10E440001A48594600784200684610F02AFBADF899
:10E450000040ADF80260ADF804503889ADF8060010
:10E46000B888ADF80800D8F80000B0F8BE10ADF8D4
:10E470000A10B0F8C010ADF80C10B0F8BA10ADF832
:10E480000E10B0F8C200ADF8100099F800000FE0CF
:10E49000148300102C8300104C8100105081001058
:10E4A0005681001058810010E58100105581001040
:10E4B000072804BF6846FEF7F5FC504613B0BDE8D8
:10E4C000F08F474810B50068D0F8F00010F4807F56
:10E4D00006D0C0F30330012101FA00F0F5F714FF74
:10E4E000404900204870887010BD70B53D4D002433
:10E4F000A878002814BF01260026687828B904F0FF
:10E5000042FA002808BF002100D001218E4227D006
:10E510000A1C18BF0122AA7031480068D0F8F030F8
:10E5200013F0040F0ED021B1C3F30310052808D255
:10E5300006E00021A960696090F8CD00052800D2AE
:10E540002870012413F0020F18BF0124002A18BFFD
:10E55000012200238221072003F008F9F1F7F1FEE0
:10E56000204670BD2DE9F0411D4800270068D0F815
:10E57000F01011F4807F30D01A4E7078051C18BF4F
:10E580000125C1F30330184A5268012303FA00F051
:10E59000024011F4007F0AD092B10AF0B2FD0428C3
:10E5A00018BF08280AD002200AF0A6FD06E03AB1FA
:10E5B0000AF0A7FD042818BF0828F4D1012403E0BD
:10E5C000002401200AF098FDA54206D0201C18BFA7
:10E5D00001207070FFF789FF07463846BDE8F081DB
:10E5E0002C83001014830010001000407148007844
:10E5F00070477048406800F5407070476D4840684B
:10E6000000F58070704770B56A4C4FF444306A4A28
:10E6100060600168914204BF4168B1F50C7F3BD155
:10E620008168B1F5584F37D8644AC568954223D000
:10E630004FF0000C03466246BCEB910F0AD253F830
:10E64000046B521C86EA0C0CB2EB910FF7D3BCF1B1
:10E65000000F21D1026A7AB14FF0000C03466246E6
:10E66000BCEB910F06D253F8046B521CB444B2EBCE
:10E67000910FF8D365450FD1012500F5807000F0AA
:10E68000BEF848B1606800F5407000F0C7F8002897
:10E690001EBF2570012070BD002070BD45490020BF
:10E6A00008704FF44430F5F7ADBC4248017841B1F1
:10E6B0004068414A0168914202BF4168B1F50C7F50
:10E6C0007047002070473B4B5B6803F5807318442C
:10E6D000F5F78EBD374B5B6803F540731844F5F7CB
:10E6E00087BD3448406800F5A0607047314B5B68D7
:10E6F00003F5A0631844F5F77BBD2E484068006918
:10E7000070472C4949680A6982429CBF00207047C3
:10E7100000EB400001EB001000F5C0607047254A97
:10E72000526802EB8000436A406E1A4400FB0120ED
:10E7300070472049886070471E48806870472DE9FF
:10E74000F0011C4B00220127D3E9014690468318B3
:10E7500093F92030002B12DB07FA02FC1CEA060FAB
:10E760000DD002F0FF0C04EB8C0CDCF82450DCF82C
:10E7700064C0254403FB0C5341F8223001E041F80A
:10E780002280521C102AE2D3BDE8F0017047002914
:10E79000B8BF704730B49446064A526802EB800016
:10E7A000446A406E224401FB002030BC1A46614698
:10E7B000F5F71EBD2083001054465053EFBEADDE6A
:10E7C00010B5FFF720FFB0B1FFF713FF01464FF47C
:10E7D000BC72174810F056F9FFF710FF154C0146B0
:10E7E0004FF4E872206810F04DF92068C06BBDE866
:10E7F000104004F03AB80220F9F72CF8E1E758B1DC
:10E800000D4A0168914207D1406820F00F00B0F531
:10E81000407F04BF012070470020704730B100687E
:10E8200020F00F00802804BF0120704700207047AF
:10E83000B83101102C83001041505352FE494860FA
:10E840007047FD4880687047FB4948707047FA4838
:10E85000407870470200F9484FF008010068438A89
:10E86000008A03FB00101CBFC01C20F0030070478F
:10E870002DE9F04104460D460846F8F71DFF78B132
:10E88000012606FA04F010F0CA0F18BF002C07D0BA
:10E89000032C05D8E9494FF43C3201200B6802E013
:10E8A0000020BDE8F081A04213D006FA00F111F07B
:10E8B000CA0F0BD0598A1F8A4FF0080C01FB07C101
:10E8C000C91C21F0030C0CEB4C010A44401C03282A
:10E8D000E9D90120A8420CD0B3F812C01C8A082143
:10E8E0000CFB0411C91C21F00301401C0A4403283D
:10E8F000F0D91046BDE8F0812DE9F04F0E4690F8B2
:10E9000021A090F8209000F15005ADF20C4D174673
:10E91000012411463046FFF7ABFFA11E012E08BFB0
:10E92000C74906D0022E08BFC64902D0032E08BF31
:10E93000C5494FF0000830B102688A4204BF406800
:10E94000CDE9002001D0CDE90018C048022E0168B1
:10E950000CBFB1F98A00B1F93A0086460CBFB1F993
:10E960008820B1F93820934600230AFB09FCBCF14A
:10E97000000F0ED935F913107145D8BF8B4505DC52
:10E980009142C8BF0A468142B8BF08465B1C9C45FD
:10E99000F0D8104400EBD07042100023BCF1000FFF
:10E9A00088BFE94616D935F91300801A00EBD070FC
:10E9B00041107F29C8BF7F2105DC11F1800FB8BF4E
:10E9C0006FF07F0100DA002409EB03005B1C017289
:10E9D0009C45E8D88DF804409DF80500FF283CBF11
:10E9E000401C8DF80500ADF806206C4639463046CF
:10E9F000FFF73EFF78B19149082209684B8A098ADE
:10EA000003FB01222146F5F7F3FB01280CBF4FF071
:10EA100001084FF0000840460DF20C4DBDE8F08FA4
:10EA20002DE9F047984615460E468146F8F741FE17
:10EA3000F8F742FE002808BFBDE8F0877E4F844CFF
:10EA40003878814588BFBDE8F0870CD287F8009000
:10EA50004FF00000B8704FF0FF024FF014017C48F7
:10EA600010F03DF819E097F802C0BCF1050F28BF7F
:10EA7000BDE8F087BCF1000F18BF00200DDD14F8D1
:10EA80002010B14206D104EB80014978A94208BFA9
:10EA9000BDE8F087401C6045F1DBB87804EB8001ED
:10EAA00004F820604D70A1F80280401CB870BDE8E9
:10EAB000F08770B5054616460C460846F8F7FCFD8B
:10EAC00000281CBF681E032832BF022E002070BD24
:10EAD00004EBC400400105EB450100EB411006EBDF
:10EAE000460100EB011000F5203000F5FD4070BD3F
:10EAF0002DE9F04F97B04FF0000816460D46074637
:10EB0000CDF83080FF2230216846CDF834800FF0F8
:10EB1000E6FFDFF840A14FF47F30CDF800A0016898
:10EB2000880A424211EB822218BF401C404201EB8E
:10EB30008000C01C20F0030000F500504649428AC6
:10EB4000437C52BA007C63F31F4242EA00600190AA
:10EB50000888A1F1040940BAADF80A0038690390A9
:10EB600099F800008DF81800002231462846FFF77A
:10EB7000A0FF0446012231462846FFF79AFF4FF0D6
:10EB8000010C012D04D0022D18BF032D40D082E0CE
:10EB90000022114624B32368534521D1237A647A95
:10EBA00028B1D0F800B0D34504BF027A417A1819D1
:10EBB00002EB010A504583BFADF830C0ADF83430E8
:10EBC000ADF83640ADF830809CBFADF83420ADF8DC
:10EBD0003610BDF83400BDF836100844ADF83200E8
:10EBE000BDF83400BDF836109DF81820C0B28DF87D
:10EBF0000800C9B20CFA02F28DF8091012F00E0FDB
:10EC000019BF401C8DF80800481C8DF8090042E02F
:10EC1000002134B32268524523D1227A18B1036807
:10EC2000534508BF017A8A4286BFADF830C0ADF8BF
:10EC30003220ADF8308011E0308300102C830010BA
:10EC40004654525946544D3246544D335083001069
:10EC5000CEED0010464648533483001098BFADF8FF
:10EC60003210022D18BF032D15D1387C10F0300062
:10EC700004BF17B0BDE8F08FBDF832003146401C2C
:10EC80008DF808002846FFF7F3FD00280CBF40462A
:10EC900040798DF80900FE480DF1380A6B46B0E85E
:10ECA00016108AE8161090E8071012AC84E80710D6
:10ECB0009DF81800082813D20EA951F82000B0F1D1
:10ECC000FF3F0DD007EBC000D0E90A10CDE90410DA
:10ECD00099F80200EF49820003F11C000FF0E1FEF9
:10ECE000BDF830106C46CAB231462846FFF7E1FE47
:10ECF00048B130222146F5F77BFA01280CBF4FF0CE
:10ED000001084FF00008404617B0BDE8F08F01221F
:10ED10000021824012F0CA0F10D001281CBF022827
:10ED2000032804D0072808BF4FF4907106E0DA48A2
:10ED300008210068428A008A02FB001108467047D9
:10ED4000012310B50022834013F0CA0F0FD0012811
:10ED50001CBF0228032802D0072803D007E0FFF7D2
:10ED600087FD03E000220120FFF7A3FE02461046C4
:10ED700010BD2DE9F04106460127F8F79AFC8046C0
:10ED8000F8F79AFC002808BFBDE8F081C34D686819
:10ED900010F4807F18BF02240DD00120A04010F095
:10EDA000CA0F05D0424621463046FFF7A5FD07466B
:10EDB000306978B90BE010F4007F18BF0324ECD160
:10EDC00010F0070018BF0124E7D1BDE8F0812878D2
:10EDD000112805D2424621463046FFF789FE0746F4
:10EDE0003846BDE8F081AD49C8607047AB4810B403
:10EDF000C068002808BF4FF47C30A94A01689142DE
:10EE00001CD14168B1F5007F18D383680022844685
:10EE1000B3F5056F88BF4FF405630021B1EB930F85
:10EE200024BF10BC70475CF82140491C2244B1EB60
:10EE3000930FF8D3002A04BF10BC7047002010BC09
:10EE4000704770B50022C260D0F808C00121134697
:10EE50000446BCF5056F88BF4FF4056C0022B2EB89
:10EE60009C0F06D254F82250521C2B44B2EB9C0F3C
:10EE7000F8D35A42C260894A127912F0800F07D142
:10EE80004FF47C304FF405622146F5F7B1F90146A5
:10EE900001290CBF0120002070BDFF2270B50025A4
:10EEA000044605614FF4006150300FF018FEA58450
:10EEB000E584E562A56265632563E563A563656432
:10EEC0002564E5640120A56470BD2DE9F0414FF48F
:10EED0007C310446724E0868B04218D14868B0F5DB
:10EEE000007F14D38A6800230D46B2F5056F94BFE6
:10EEF00094464FF4056C0020B0EB9C0F26D255F8D9
:10EF00002070401C3B44B0EB9C0FF8D3F3B1FF22C0
:10EF10004FF4056120460FF0E2FD4FF40870C4E99C
:10EF200000604FF40560A0600020E06084F82000DD
:10EF300084F8210084F8220084F8230020616061B5
:10EF4000A061E0612046FFF7A8FF07E0B2F5056F7A
:10EF500088BF4FF4056220460FF094FD0120BDE804
:10EF6000F08170B402684FF408715160016801F1DA
:10EF7000500291F821C091F820300CFB03F102EB14
:10EF800041010022BCF1000F08D900EB4204521CE1
:10EF9000B4F8DE4021F8024B9445F6D80022002B4D
:10EFA00008D900EB4204521CB4F8064121F8024B88
:10EFB0009342F6D85D084FEA4C044FF0000208D0A7
:10EFC00000EB4206521CB6F8646021F8026B9542D1
:10EFD000F6D80022002C08D900EB4205521CB5F8E7
:10EFE0008C5021F8025B9442F6D8B0F8DA2021F870
:10EFF000022BB0F8DC2021F8022BB0F8D82021F841
:10F00000022B00240022BCF1000F0ED904EB4405B2
:10F0100005EB041500EB850505EB4206521CB6F81E
:10F02000526121F8026B6245F6D30022002B0ED903
:10F0300004EB440505EB041500EB850505EB4206E2
:10F04000521CB6F8826221F8026B9A42F6D3641C15
:10F05000042CD7D370BC70472DE9F74F88B000253A
:10F060000A992C462E460968049101F1500309992A
:10F07000002984BF0B49D1F8008029D9002200283B
:10F0800088BFB8F93A701AD933F9021B00290BE08E
:10F09000E4410200CEED00102C83001030830010FC
:10F0A00053454C4650830010B4BFC1F1000C8C4650
:10F0B000BC45BCBF0D44641C521C8242E4D3099978
:10F0C000761C8E42DAD3002CC8BF95FBF4FA08DC1C
:10F0D0004908414301EB5002049901EB4201B1F9A7
:10F0E00050A000210291019104995031009100211A
:10F0F00003910999002969D9FF49009E069609687C
:10F100004FF0000B4FF00109B1F81CE091F824100A
:10F110005F46D846CDF814B00791002829D9B6F932
:10F1200000204FF0000C06999344634600280DD947
:10F13000B1F90040A51A48BF151B7545B8BF0CF1C1
:10F14000010C01EB49015B1C8342F1D307998C450B
:10F1500003D305997F1C1144059108F1010806EBC2
:10F1600049068045DBD3002FC4BF059991FBF7F119
:10F1700001DC9BFBF0F1039B0A9A09B202EB43020C
:10F18000A2F86410DC4A1268538BAAEB030399427D
:10F1900009DD128B52448A4205DD019A1144019126
:10F1A0000299491C02910099099A01EB40010091D2
:10F1B0000399491C039191429ED30299002905DDD0
:10F1C000DDE9011291FBF2F1019102E05146CDF827
:10F1D00004A00A9AA2F8DA1000210291039104997E
:10F1E0005031009100210491002865D9C249009F47
:10F1F000069709684FF0000B099EB1F820E091F8DE
:10F200002510D846D946CDF814B00791002E2BD939
:10F21000B7F900204FF0000C069993446346002E86
:10F220000DD9B1F90040A51A48BF151B7545B8BFE7
:10F230000CF1010C01EB40015B1CB342F1D30799C7
:10F240008C4504D3059908F101081144059109F191
:10F25000010907EB4007B145DAD3B8F1000FC4BF8D
:10F26000059991FBF8F101DC9BFBF6F1049B0A9AEE
:10F2700009B202EB4302A2F88C109F4A1268538B2A
:10F28000AAEB0303994209DD128B52448A4205DD41
:10F29000039A114403910299491C02910099891C17
:10F2A00000910499491C049181429FD3029800283F
:10F2B000C4BF039991FBF0FA0A98A0F8DCA001986A
:10F2C0000A99504400B200EBD0704010A1F8D80069
:10F2D0000BB0BDE8F08F2DE9F04F8BB08146A1F166
:10F2E0002000146815460E464FF0010A00902029B0
:10F2F0003ABF0AFA06F0401E4FF0FF30049031BFCB
:10F30000002000980AFA00F0401E0390B9F1200F87
:10F310003BBF0AFA09F0401E4FF0FF30002205D330
:10F32000A9F120010AFA01F1A1F10102C6F12001BF
:10F330000591202E32BF20FA01F1009900FA01F167
:10F34000B2401143B040CDE90110206920F4FE60C5
:10F3500020616A48426812F0010F00F0F3804FEA22
:10F3600059084FEA59004FEA460BA0F12001B8F1C5
:10F37000200F3ABF0AFA08F0401E4FF0FF300A9003
:10F3800032BF00200AFA01F0401E0990BBF1200FA5
:10F390003BBF0AFA0BF0401E4FF0FF30002322BFA4
:10F3A000ABF120030AFA03F35B1EB8F1200F3ABF5A
:10F3B000C8F1200120FA01F100FA01F103FA08F383
:10F3C000194300FA08F0CDE9071012F4807F05D048
:10F3D0002A464146584601F0C7FC82E012F4007FFD
:10F3E0002A464146584602D001F0D6FE79E001F0A7
:10F3F0009BFB0020A86107466861BBF1000F20D984
:10F4000005EB4700B0F98C000028B8BF404200B2BD
:10F4100039490968B1F9381081420FDD7A0905EBE5
:10F42000820107F01F034A690AFA03F31A434A618B
:10F4300083B2FAB2FF210420FFF7F2FA7F1C5F4586
:10F44000DED30027BBF101001CBFDFF8ACB0069093
:10F4500047D005EB4703B3F98E20B3F98C10501A4F
:10F4600048BF881A00B2DBF800C0BCF932C084453E
:10F4700033DAB5F9DC00B1EB000C48BFA0EB010CAE
:10F480000FFA8CFC111A48BF811A08B2844511DBAF
:10F49000790905EB810007F01F0241690AFA02F2BF
:10F4A00011434161B3F88C30FAB2FF210420FFF719
:10F4B000B7FA12E0781C420905EB820100F01F0C3C
:10F4C0004A690AFA0CFC42EA0C024A61C2B2B3F879
:10F4D0008E30FF210420FFF7A3FA06987F1C874295
:10F4E000B7D36969E86901FA08F108432063AA699A
:10F4F000296A02FA08F203E05083001030830010FA
:10F50000114361636A69B8F1200F39BFC8F1200364
:10F51000DA40A8F120039A4011436163089A10422F
:10F5200004BF079A114203D0226942F010022261FF
:10F530000A9A104204BF0998014203D0206940F0A2
:10F5400020002061FE48007910F0040F00F0ED81EA
:10F550004FF0000BC5F830B05F46C5F82CB0002E58
:10F5600088BFDFF8E08320D9D8F8001005EB47000A
:10F57000B0F95201B1F95C20824203DCB1F95E10AE
:10F5800081420FDA7A0905EB820107F01F03CA6A8C
:10F590000AFA03F31A43CA6283B2F9B2FF220220C5
:10F5A000FFF73EFA7F1CB742DED3C5F828B000272C
:10F5B000C5F824B0B9F1000F88BFDFF8888320D9DF
:10F5C000D8F8001005EB4700B0F98202B1F95C20D1
:10F5D000824203DCB1F95E1081420FDA7A0905EB51
:10F5E000820107F01F034A6A0AFA03F31A434A62C8
:10F5F00083B2FAB2FF210220FFF712FA7F1C4F45B7
:10F60000DED3C5F840B00027C5F83CB0002E88BF57
:10F61000DFF830832DD9D8F8001005EB4700B0F99A
:10F620009E01B1F960208242DCBFB1F962209042B4
:10F630000EDD7A0905EB820107F01F03CA6B0AFA97
:10F6400003F31A43CA6383B2FF22F9B201200BE02D
:10F65000B1F96C208242DCBFB1F96E10884205DD41
:10F6600083B2F9B2FF221020FFF7DAF97F1CB7420C
:10F67000D1D3C5F838B00027C5F834B0B9F1000FC0
:10F6800088BFDFF8C0822DD9D8F8001005EB4700FD
:10F69000B0F9CE02B1F960208242DCBFB1F962203C
:10F6A00090420EDD7A0905EB820107F01F034A6BD9
:10F6B0000AFA03F31A434A6383B2FF21FAB2012024
:10F6C0000BE0B1F96C208242DCBFB1F96E108842C8
:10F6D00005DD83B2FAB2FF211020FFF7A1F97F1CEC
:10F6E0004F45D1D300202865E864A86407466864C4
:10F6F000002E88BFDFF84C8220D9D8F8001005EB27
:10F700004700B0F9EA01B1F96420824203DCB1F9A3
:10F71000661081420FDA7A0905EB820107F01F03B8
:10F72000CA6C0AFA03F31A43CA6483B2F9B2FF221D
:10F730000320FFF775F97F1CB742DED30027B9F12C
:10F74000000F88BFDFF8FC8120D9D8F8001005EB46
:10F750004700B0F91A03B1F96420824203DCB1F921
:10F76000661081420FDA7A0905EB820107F01F0368
:10F770004A6C0AFA03F31A434A6483B2FAB2FF21CD
:10F780000320FFF74DF97F1C4F45DED3696AE86A15
:10F79000B14040EA0108C4F83880A96A286BB1403A
:10F7A0000843E0636A6A202E39BF059922FA01F105
:10F7B000009902FA01F141EA0007E763696BE86B1F
:10F7C00001FA06F140EA01022264A96B286C01FAF1
:10F7D00006F140EA010060646B6B39BF059923FABA
:10F7E00001F1009903FA01F141EA000161646B6CD7
:10F7F000E86C03FA06F340EA0300A0640690AB6CE1
:10F80000286D03FA06F340EA0300E064D5F844C02B
:10F8100039BF059B2CFA03F3009B0CFA03F343EA70
:10F820000000E064059032EA080521EA070C48EA86
:10F8300005002564009047EA0C0E06EB0901C4F8A8
:10F8400044C008BFBCF1000F44D000231A4618463C
:10F8500000293FD94FEA501904EB890900F01F0B2A
:10F86000D9F840900AFA0BFB19EA0B0F03D0864235
:10F8700094BF521C5B1C401C8142EBD8012B11D160
:10F880000498284040EA0800A06303980CEA0000AE
:10F890003843E063049825EA0000206403982CEACA
:10F8A00000006064012A15D1206C029A00EA02036C
:10F8B000A26B1A43A263626C019BD4F83CC0134054
:10F8C00043EA0C03E363029B98432064019822EA15
:10F8D00000006064009A06989043A064059A22EAAA
:10F8E0000E02E26408BF002A1FD000231A46184601
:10F8F000002917D94FEA501C04EB8C0C00F01F05AF
:10F90000DCF848C00AFA05F51CEA050F03D0864268
:10F9100094BF521C5B1C401C8142EBD8002B18BFCB
:10F92000002A02D10020A064E064A06B0299084282
:10F9300003D1E26B01990A4209D0216904E0000079
:10F94000308300105083001041F040012161049980
:10F95000084203D1E16B0398014203D0206940F0D3
:10F9600080002061206C0299084203D1626C0199E9
:10F970000A4203D0216941F480712161049908424F
:10F9800003D1616C0398014203D0206940F40070F8
:10F990002061A06C002804BFE06C002803D020691F
:10F9A00040F4806020610BB00120BDE8F08FFE487C
:10F9B000006970472DE9F04FCBB017460D4604465D
:10F9C000F3F722F80120F1F7AAF806461120F1F723
:10F9D000A6F8304314BF012002208DF8180014BF90
:10F9E000112012208DF81900F2F798F838B19DF81F
:10F9F00018009DF819108DF818108DF819009DF851
:10FA00001800F1F78CF8002818BF284604909DF8DC
:10FA10001900F1F784F8002818BF20460590F3F785
:10FA200000FC0022002D88BF24A90BD98356142B7B
:10FA3000A8BF143B02DA0A2BA8BF12338B54521C06
:10FA4000AA42F3D3F3F7EFFB0021002C88BF24AACE
:10FA500007D9435C02EB010C491C8CF826308C4220
:10FA6000F7D8F3F7CAFA0390CF480DF1180A0079D6
:10FA700010F0200F55D007F1DE000090283000254F
:10FA8000E9460DF1100B01905BF825601AF80500AE
:10FA9000F4F732F80024002E1AD905EB450000EBEC
:10FAA000051024A901EB400818F90420262A28BFD4
:10FAB000002006D21AF805000021F2F725FEF4F71F
:10FAC00021F859F8251021F81400641CB442EBD336
:10FAD0006D1C022DD8D3B54C26781D2E21D10021C6
:10FAE0000A460DF11C085BF822500020002D88BF4B
:10FAF00059F822C007D93CF8103028F81130401CC2
:10FB0000491C8542F7D8521C022AECD31D2E08D17D
:10FB10004046FDF7FFFB20781D2804BF07A8FDF72E
:10FB2000F9FBA14D287910F00C0F00F0AE8303987B
:10FB300000F0F000F3F71FF99DF81800F1F7F1FD60
:10FB400007909DF81800F1F75BFE002437901AF833
:10FB50000400F2F721FD44A941F824001AF804003A
:10FB6000F1F78BFE0EA941F824001AF80400F1F712
:10FB7000D8FF20A941F824001AF80400F2F709F888
:10FB800022A941F824001AF80400F1F707F846A961
:10FB900018AA41F824001CA81AA902EB840200EB61
:10FBA000840001EB84010092CDE9011016A800EB5E
:10FBB000840314A800EB840212A800EB84011AF855
:10FBC0000400F2F7C8FA1AF80400F2F7F6FB1EA9CF
:10FBD00041F824001AF80400F2F72EFD10A941F8AC
:10FBE0002400641C022CB2D3714E3068B0F8481067
:10FBF0009DF81800F1F7A9FD002400211AF804006F
:10FC0000F2F7B0FC6A4E306890F84A101AF8040017
:10FC1000F1F747FE1AF804000021F1F79CFF1AF8EB
:10FC200004000021F1F7CFFF1AF804000121F0F7DA
:10FC30009BFF3068B0F84C101AF80400F2F747FB4D
:10FC40001AF804000021F2F7BFFC641C022CD4D384
:10FC500055484FF00009007910F0040F00F0DC81E6
:10FC60003446206890F84B3090F85920B0F8501086
:10FC70000091CDE9012390F84F3090F84E2090F894
:10FC800058109DF81800F2F7AAF8206890F84B3049
:10FC900090F85920B0F850100091CDE9012390F868
:10FCA0004F3090F84E2090F858109DF81900F2F758
:10FCB00096F89DF818000021F2F786FC9DF81900CF
:10FCC0000021F2F781FC3AADF3F7E4F9FCF754FDBB
:10FCD000012806D02846F3F7B3FC00286CD0F3F7D0
:10FCE00006FDF2F791FE3E99002204AD002055F882
:10FCF0002230002B0ED902EB420C0CEB021C07EB5E
:10FD00000C1C31F8026B0CEB4008401CA8F8526147
:10FD10008342F6D8521C022AE8D32648D0E90010C4
:10FD2000CDE90C109DF81800F0F7F9FE48909DF809
:10FD30001900F0F7F4FE49909DF8180040A9F1F77A
:10FD40004DFE9DF8190042A9F1F748FE9DF81800F4
:10FD500008A9F1F7B5FE9DF819000AA9F1F7B0FE60
:10FD6000134C206890F84B3090F85920B0F852109E
:10FD70000091CDE9012390F84F3090F84E2090F893
:10FD800058109DF81800F2F72AF8206890F84B30C8
:10FD900090F85920B0F852100091CDE9012390F865
:10FDA0004F3090F84E2008E030830010EA810010B8
:10FDB00050830010DC41020030E090F858109DF8AC
:10FDC0001900F2F70CF89DF818000CA9F1F756FE8F
:10FDD0009DF819000CA9F1F751FE00249DF81800B8
:10FDE0000021F2F7F1FB9DF819000021F2F7ECFB7E
:10FDF0009DF818000021F0F778FE9DF81900002109
:10FE0000F0F773FE1AF804000121F0F76EFE1AF8FD
:10FE10000400C0F3011001280AD102E0F7F7B4FC96
:10FE200054E784F0010001211AF80000F0F75DFEAC
:10FE3000CDF8E090CDF8E4909DF8180038A9F1F7DE
:10FE4000ADFD9DF8190038A9F1F7A8FD04A800211F
:10FE500050F824801AF80400F2F7FCFC0025019009
:10FE6000B8F1000F4CD904EB440000EB041024A9B6
:10FE700001EB400107EB001B0091009838AA00211C
:10FE80004657CDF8E090CDF8E4901AF80400F2F768
:10FE9000FEFB202E06DBA6F1200101208840CDE9E3
:10FEA000389003E00120B040CDE938091AF8040089
:10FEB00038A9F1F773FD389838AAC04338903998BB
:10FEC0000921C04339901AF80400F2F7E0FB3AAE7A
:10FED000F3F7E0F8FCF750FC012806D03046F3F7C2
:10FEE000AFFB00287ED0F3F702FCF2F78DFD0198FE
:10FEF00000880BEB45016D1CA1F89E014545BCD364
:10FF0000CDF8E090CDF8E4901AF8040038AA00216A
:10FF1000F2F7BDFB641C022CFFF460AF9DF81800E3
:10FF200008A9F1F7ABFD9DF819000AA9F1F7A6FDA4
:10FF30009DF818004899F0F7D8FD9DF819004999E7
:10FF4000F0F7D3FD9DF8180040A9F1F727FD9DF8C3
:10FF5000190042A9F1F722FDFE4C206890F84B30C1
:10FF600090F85920B0F854100091CDE9012390F891
:10FF70004F3090F84E2090F858109DF81800F1F787
:10FF80002EFF206890F84B3090F85920B0F85410AC
:10FF90000091CDE9012390F84F3090F84E2090F871
:10FFA00058109DF81900F1F71AFF9DF8180001216B
:10FFB000F2F70AFB9DF819000121F2F705FB3AACB4
:10FFC000F3F768F8FCF7D8FB012806D02046F3F7D2
:10FFD00037FB00287DD0F3F78AFBF2F715FD0022EE
:10FFE00004AC00E081E03E9954F822C00020BCF14E
:10FFF000000F0ED902EB420303EB021307EB0313CE
:020000021000EC
:1000000031F8025B03EB4006401CA6F8EA51844538
:10001000F6D8521C022AE7D3CF48007910F0080F17
:100020007ED0CC4C206890F84B3090F85920B0F836
:1000300056100091CDE9012390F84F3090F84E20F2
:1000400090F858109DF81800F1F7C9FE206890F854
:100050004B3090F85920B0F856100091CDE90123AB
:1000600090F84F3090F84E2090F858109DF81900F5
:10007000F1F7B5FE00210DF1100C00205CF82120F5
:10008000002A0CD901EB410303EB011307EB031327
:1000900003EB4005401CA5F836928242F8D8491C73
:1000A0000229EAD32068002590F86800B5EB400FDC
:1000B00036DA206890F86800A842D4BF01210021F8
:1000C0009DF81800F2F780FA206890F86800A842BE
:1000D00000E00DE0D4BF012100219DF81900F2F7E6
:1000E00073FA3AAEF2F7D6FF05E0F7F74DFBF1E60B
:1000F000F7F74AFB66E7FCF73FFB012805D03046DF
:10010000F3F79EFAD8B3F3F7F2FAF2F77DFC3E99D3
:100110004FF0000904AB0022104653F8296000E0BC
:1001200058E0002E05D931F91030401C1A4486429F
:10013000F9D8B2FBF6F2701E3DD009EB490303EB90
:10014000091307EB031B31F9103001EB400C3CF9AC
:10015000028CB3EB080348BF5B4231F91080B8EB67
:10016000020831F910804CBFA2EB0808A8EB020886
:100170003CF902EC3CF902CCBEEB020E00E00FE0D1
:100180004CBFA2EB0C0CACEB020CE0450BEB400CB3
:1001900009DDBCF936824345C8BFACF8363208E009
:1001A000F7F7F2FAA7E7BCF934829845B8BFACF884
:1001B0003432401EC7D109F1010901EB4601B9F102
:1001C000020FA7D320686D1C90F86800B5EB400FB4
:1001D000FFF66FAF9DF818000799F1F7B6FA9DF892
:1001E00018003799F1F71BFB00241CAD1EAE20AFA1
:1001F0000DF188080DF588790DF58C7B59F82410E0
:100200001AF80400F2F7AEF90EA850F824101AF804
:100210000400F1F746FB57F824101AF80400F1F730
:100220009AFC58F824101AF80400F1F7CCFC5BF89B
:1002300024101AF80400F0F797FC1AA918A851F82E
:10024000241055F8242050F82400CDE9000116A808
:10025000029250F8243014A850F8242012A850F824
:1002600024101AF80400F1F7BAFD56F824101AF811
:100270000400F2F72CF810A850F824101AF8040023
:10028000F2F7A2F9641C022CB8D30398F2F773FDBD
:100290004BB0BDE8F08F2DE9F04F04462F4887B0F2
:1002A0000F4600684FF0000890F8F80000F00F05C6
:1002B00001F072FB01280BD040F20F312846F7F70E
:1002C000C0FB012813D0002001F063FB00F02EBA20
:1002D00000210846F2F785FDF0F77AFE50B120487C
:1002E000D0F8401341F48031C0F8401302E00120FF
:1002F00001F04FFB1B4806781B480578002D18BFFE
:10030000002E00F011823868002180F8206080F80B
:10031000215080F8221080F82310F3F727FCF2F721
:100320006CFE0090002014F0030F18BF0F4814F06B
:10033000200F1CBF40F0F00040F00050DFF81480A8
:10034000002800F0E780009940F47F00084014F492
:10035000407F0DE050830010308300102C8300108C
:10036000005000404C8100104D810010070000102B
:1003700018BF20F47F00F2F7FEFC0020F8F7CFFF53
:1003800060F30F09824600210846F8F7B2FF022009
:10039000F8F7C5FF60F31F4900210220F8F7A9FF15
:1003A0001220F8F7BCFF60F30F0B00211220F8F7C2
:1003B000A0FF14F4407F17D00020F1F7B2F90690A7
:1003C0000020F1F71DFA05900020F1F756FA04908D
:1003D0000020F1F7A6FB03900020F1F7DAFB029072
:1003E0000020F1F76CFF019014F4807F2DD0D8F835
:1003F0000000B0F8841000291CBF0020F1F7A5F917
:10040000D8F8000090F8861000291CBF0020F1F7F2
:1004100048FAD8F8000090F8870010F00F0F05D0C8
:1004200000F00F00411E0020F1F795FBD8F8000006
:1004300090F8870010F0F00F3BD04FF0FF3101EB48
:1004400010110020F1F7BFFB33E014F4007F30D02F
:10045000D8F80000B0F8AC1000291CBF0020F1F75C
:1004600074F9D8F8000090F8AE1000291CBF0020E5
:10047000F1F717FAD8F8000090F8AF0010F00F0F5E
:1004800005D000F00F00411E0020F1F764FBD8F802
:10049000000090F8AF0010F0F00F06D04FF0FF31E1
:1004A00001EB10110020F1F78EFB00210846F1F757
:1004B000F9FE1F20F8F714F9F2F7A6FA14F4407FBA
:1004C00017D000200699F1F740F900200599F1F7BF
:1004D000A6F900200499F1F7E4F900200399F1F757
:1004E0003AFB00200299F1F76EFB00200199F1F729
:1004F000D9FE51460020F8F7FCFE4FEA29410220C0
:10050000F8F7F7FE0FFA8BF11220F8F7F2FE0098D9
:10051000F2F731FC14F02C0F04D03A46294630464D
:10052000FFF748FA14F0030F00F0FC800097D7F8AB
:1005300000A0A9460AF15004F2F775FE0746F2F74B
:1005400063FAFE4DA88810F4407F03D00020F1F735
:1005500094F90190686810F4807F05D0D8F8000005
:1005600090F8861059B107E010F4007F07D0D8F852
:10057000000090F8AE1011B10020F1F792F90020C0
:10058000F3F7BAFAED48006903280CD004284FF0BD
:10059000000847D0B9F1000F43D908EB4800002507
:1005A00000EB081B91E04FF00008B9F1010018BF03
:1005B000029024D008EB4800002500EB081B15E052
:1005C0007857262811D2C107490C00EBD07001EBF7
:1005D0008B01401001EB800000F1405000F58030AD
:1005E0000068F3F78FFA24F8020B6D1CB54201D2B4
:1005F000262DE5DB029808F101088045DAD3A9F140
:100600000101494538BF002268D2002002E024F8E9
:10061000022B401CB04201D22628F8DB491C494578
:10062000F3D35BE0B9F1020018BF029024D008EBCD
:100630004800002500EB081B15E07857262811D24A
:10064000C107490C00EBD07001EB8B01401001EBAE
:10065000800000F1405000F580300068F3F752FA56
:1006600024F8020B6D1CB54201D2262DE5DB029861
:1006700008F101088045DAD3A9F10201494538BFE4
:1006800000222BD2002002E024F8022B401CB042B2
:1006900001D22628F8DB491C4945F3D31EE07857E0
:1006A000262811D2C107490C00EBD07001EB8B0159
:1006B000401001EB800000F1405000F580300068F0
:1006C000F3F720FA24F8020B6D1CB54201D2262D57
:1006D000E5DB08F10108C845FFF45FAF9748808863
:1006E00010F4407F03D000200199F1F7DAF84A4670
:1006F00031460AF150000EF0E8F9914C20781D289F
:100700000AD10AF15000FCF7E3FB20781D2804BF52
:100710000AF15000FCF7DCFB71084FEA4900009A2F
:10072000FEF79AFC4FF00108F2F72AFC07B04046AA
:10073000BDE8F08F81480121816011210170002105
:100740008170FDF74EB97D490020886070477B4974
:10075000086170472DE9F04FDFF8E0A1ADF56F7D3E
:1007600001271120CAF808704FF000088AF800002D
:100770008AF80280FDF735F9DAF804004FF4407189
:1007800031EA000008BF002600F0A7811D20FCF719
:10079000B5FAED901D20FCF7A3FDEE904FF46D71BE
:1007A0006846DAF80C400EF072F90094BAF80400CA
:1007B00010F4804F1CBF2046FEF76FFBDAF80400F0
:1007C00010F4806F1CBF0120CAF810000BD110F488
:1007D000006F18BF022004D110F4805F18BF0320FF
:1007E0007DD0CAF8100000986A4690F8203090F842
:1007F00021C05E084FEA4C0506FB05F1503000EBC6
:1008000041000021BCF1000F08D902EB410B30F888
:10081000029B491CABF8DE908C45F6D80021002BDA
:1008200008D902EB410B30F8029B491CABF806914A
:100830008B42F6D80021002E08D902EB410B30F88C
:10084000029B491CABF864908E42F6D80021002D23
:1008500008D902EB410930F8026B491CA9F88C60F9
:100860008D42F6D830F8021BA2F8DA1030F8021BDD
:10087000A2F8DC1030F8021BA2F8D81000250021E5
:10088000BCF1000F0ED905EB450606EB051602EB91
:10089000860606EB410B30F8029B491CABF85291DF
:1008A0006145F6D30021002B0ED905EB450606EB7A
:1008B000051602EB860606EB410B30F8029B491C3D
:1008C000ABF882929942F6D36D1C042DD7D36146C2
:1008D0001846FEF7C1FB3E46DAF8040000E003E0EC
:1008E00010F4004F09D104E010F4005018BF0420A8
:1008F00077E76946FFF7CFFC0646ED98FCF7FEF96F
:10090000EE98FCF7EDFC94F8209094F82150002E1E
:100910001CBFB9F1000F002D00F0DF80DAF81000E5
:1009200000287AD19AF8040010F0020F05D04FEA9F
:10093000590168006A4600F0AEFD03E03083001004
:10094000E58100109AF8040010F0050F04D06A4603
:1009500029464846FEF7BFFC9AF8040010F0080F3D
:100960007BD0009ADFF8F8E66846116921F4C0519F
:1009700011610021CDF86080CDF85C80002D19D97F
:10098000DEF800C000EB4103B3F93632BCF96AC0AF
:100990009C450CDA4B0900EB830301F01F0BD3F8E5
:1009A0005CC007FA0BFB4CEA0B0CC3F85CC0491C9B
:1009B000A942E5D3C0F858800021C0F85480B9F1AD
:1009C000000F19D9DEF800C000EB4103B3F966331C
:1009D000BCF96AC09C450CDA4B0900EB830301F0BB
:1009E0001F0BD3F854C007FA0BFB4CEA0B0CC3F8EF
:1009F00054C0491C4945E5D3916BC36D1943436D00
:100A0000AB4019439163D16B036E1943836DAB40C7
:100A10000B43D363202D416D00E01EE039BFC5F1CB
:100A2000200C21FA0CF1A5F1200C01FA0CF119436C
:100A3000D163416D002904BF816D002903D0116984
:100A400041F400611161C16D002904BF006E0028EE
:100A500003D0106940F4805010619AF8040010F03F
:100A6000400F05D1DAF8100000B36846FEF779FAB6
:100A7000C4F80C80A36800222146A446B3F5056F94
:100A800088BF4FF405630020B0EB930F06D25CF8EB
:100A90002070401C3A44B0EB930FF8D35042C8602A
:100AA0009AF8040010F0800F14D10DE06069401C2A
:100AB00060612069002814BFE069A06900F10100AD
:100AC00014BFE061A061D0E74FF47C304FF40562C1
:100AD000F3F78EFB2046FEF74CF941208DF8B40366
:100AE000D6B1207C8DF8B503607C8DF8B603A07C70
:100AF0008DF8B703E07C8DF8B80300230522EDA93B
:100B0000072000F0C0FE0020CAF80880CAF81000D4
:100B10000DF56F7DBDE8F08FFF208DF8B5038DF8E2
:100B2000B6038DF8B703E6E72DE9F74F84B04FF031
:100B3000000AC2F820A00646C2F81CA00598DFF8FB
:100B40002085174654464FF00109002821D907EBAC
:100B50004400B0F964000028B8BF404200B2D8F8A1
:100B60000010B1F9381081420FDD610907EB8101F6
:100B700004F01F03CA6909FA03F31A43CA6183B276
:100B8000E1B2FF220420FDF74BFF0598641C84426C
:100B9000DDD3002401281CBF0598451E46D007EB75
:100BA0004403B3F96620B3F96410501A48BF881A99
:100BB00000B2D8F800C0BCF930C0844533DAB7F9C8
:100BC000DA00B1EB000C48BFA0EB010C0FFA8CFC73
:100BD000111A48BF811A08B2844511DB600907EB7E
:100BE000800004F01F02C16909FA02F21143C161D9
:100BF000B3F86430E1B2FF220420FDF711FF12E0E8
:100C0000601C410907EB810100F01F0CCA6909FA59
:100C10000CFC42EA0C02CA61C1B2B3F86630FF2292
:100C20000420FDF7FDFE641CAC42B8D3D8F80000E8
:100C300090F8361000297DD090F837003D68814249
:100C400088BF084600240599002984BF401C0090F5
:100C500070D94FF0010E00984FF000090121CA46EB
:100C6000012852D9FE4800680390B0F93A3004FBDD
:100C7000066002900EFB0660019004FB061005EB77
:100C80004000B0F950C0BCF1000FB4BFCCF100007F
:100C90006046834239DB0EFB061005EB4000B0F9DD
:100CA00050000028B4BF4242024693422DDB029A14
:100CB000521A05EB4202B2F94E80B8F1000FB4BFF0
:100CC000C8F10002424693421FDB019A521A05EB1B
:100CD0004202B2F94E20002AB4BFC2F1000B934683
:100CE0009B4512DCA0EB0C0C0398B0F93400604576
:100CF000B8BF09F10109A2EB08028242C8BF0AF19C
:100D0000010A491C00988142B7D3BAEB090048BFD9
:100D1000A9EB0A00D249096891F83610884214DB21
:100D2000600907EB800004F01F030121C2699940AC
:100D3000114300E014E0C16107EB4400E1B2B0F8F8
:100D40006430FF220420FDF76BFE0598641C84428A
:100D500006D2002C18BFA4F1010E7FF47CAF78E717
:100D600007B00120BDE8F08F2DE9F74F064688B0A7
:100D7000002017681062D06190615061B9480490FA
:100D80000020009001900290824603900998154639
:100D900047F6FF7BA0F10109A6F10108002871D9EF
:100DA0000024002E69D94FEAEA700AEBD06020F0E7
:100DB0001F01AAEB0101012202FA01F1401105EB2A
:100DC0008000CDE906011C3005900AFB064007EBC8
:100DD0004000BAF1000FB0F9500018BFCA450BD15E
:100DE000002C18BF444507D19D490968B1F99220EC
:100DF000B1F99010B2B911E09949049B0968984281
:100E0000B1F98A20B1F98810C4BF0294CDE903A0DA
:100E10005845BCBF8346CDE9004AEBE7904A1268CB
:100E2000B2F98A2019B98E490968B1F9881090423F
:100E300001DC88421EDA06994FF0010CCA69079955
:100E40000A4305990A60E11704EBD1614A1105EBE9
:100E5000820303F1140221F01F015B69611A0CFA8D
:100E600001F11943116083B2E2B20AF0FF010620DA
:100E7000FDF7D6FD641CB442A7D309980AF1010A14
:100E800082458DD3764C2068B0F88E00002846D07D
:100E90000499A1EB0B01814241DD039803994009BC
:100EA00005EB800001F01F03C269012101FA03F381
:100EB0001A43C2610198019A400905EB800002F0D3
:100EC0001F02C36901FA02F21A43C2610298029A30
:100ED000400905EB800002F01F02436901FA02F2AB
:100EE0001A4342610098009A400905EB800002F025
:100EF0001F024369914019434161049883B20298EB
:100F0000C2B20398C1B20620FDF78AFD00981FFA0D
:100F10008BF3C2B20198C1B20620FDF781FD5048A3
:100F2000006890F88C00002800F032814FF0000A31
:100F3000002E7DD90998801E009007EB4A00099980
:100F4000B0F950000024012973D04FEAEA710AEB8E
:100F5000D16121F01F02AAEB0202012303FA02F27F
:100F6000491105EB8101CDE9031214310291611C95
:100F7000019101FB06A107EB4101B1F950B0BBF1B2
:100F8000000FC8BF00285EDDBBEB000148BFA0EB2F
:100F90000B018345CCBF5A4602464FF448435943A0
:100FA00091FBF2F101F2FF114A0A002C1CBF0099DB
:100FB0008C420AD1BAF1000F18BFC24504D12849AA
:100FC000096891F88D100CE014B100998C4204D19D
:100FD0002349096891F8991003E02149096891F8BB
:100FE0008C1019B91E49096891F88C108A422ADDC3
:100FF000E11704EBD1614A1105EB820221F01F01D8
:1010000002F11C03A4EB010CD269012101FA0CF1DD
:1010100011431960039983B206204A6904990A436F
:1010200002990A600AF0FF02E1B2FDF7F9FC01E063
:1010300012E00CE001981FFA8BF3C1B20AF0FF0234
:101040000620FDF7EDFC641C58464C458FD30AF191
:10105000010AB245FFF471AF4FF0000A099803E0AE
:10106000508300100080FFFF002884BFB01E009056
:101070007DD90AFB06F007EB40000024B0F95000D0
:10108000012E7FD04FEAEA710AEBD16121F01F02F5
:10109000AAEB0202012303FA02F2491105EB8101D6
:1010A000CDE902121C3101910AFB064107EB410117
:1010B000B1F952B0BBF1000FC8BF00285EDDBBEB39
:1010C000000148BFA0EB0B018345CCBF5A46024646
:1010D0004FF44843594391FBF2F101F2FF114A0AE0
:1010E000BAF1000F18BFCA4509D1002C1CBF0099E6
:1010F0008C4205D1FE49096891F88D100CE014B1BD
:1011000000998C4204D1FA49096891F8981003E0DB
:10111000F749096891F88C1019B9F549096891F8EF
:101120008C108A422ADD02994FF0010CCA6903999A
:101130000A4301990A60E11704EBD1614A1105EBFA
:10114000820303F1140221F01F015B69611A0CFA9A
:1011500001F11943116083B2E2B20AF0FF010620E7
:10116000FDF75EFC601C1FFA8BF3C2B201E00FE0DA
:1011700008E00AF0FF010620FDF752FC641C584607
:10118000444591D309980AF1010A8245FFF471AFF1
:101190000BB00120BDE8F08F2DE9F04F05464FF070
:1011A000000087B017681062D06190615FEA0108A3
:1011B00082465061A8F101001646A5F10109009090
:1011C0005AD00024002D53D94FEAEA700AEBD060C0
:1011D00020F01F01AAEB0101012202FA01F14011E6
:1011E00006EB8000CDE9010100F11C0B0AFB054074
:1011F00007EB4000BAF1000FB0F950101CBF009887
:10120000824508D1002C18BF4C4504D1B84800686D
:10121000B0F9B20003E0B6480068B0F9B00018B900
:10122000B3480068B0F9B00081421EDD01984FF06C
:10123000010CC26902981043CBF80000E01704EBE0
:10124000D060421106EB820303F1140220F01F006C
:101250005B69201A0CFA00F0184310608BB2E2B2FE
:101260000AF0FF010720FDF7DBFB641CAC42BDD395
:101270000AF1010AC245A4D39D48006890F8B40061
:10128000002800F004814FF0000B002D84BFA8F16E
:10129000020005907AD907EB4B000024B0F950000A
:1012A000B8F1010F6ED04FEAEB710BEBD16121F079
:1012B0001F02ABEB0202012303FA02F2491106EB13
:1012C0008101CDE9031214310291611C019101FBEE
:1012D00005B107EB4101B1F950A0BAF1000FC8BF49
:1012E00000284ADDBAEB000148BFA0EB0A018245A5
:1012F000CCBF524602464FF44843594391FBF2F1AA
:1013000001F2FF114A0A002C1CBF05998C42784952
:1013100009680CBF91F8B51091F8B41019B9744967
:10132000096891F8B4108A4227DDE11704EBD16116
:101330004A1106EB820221F01F0102F11C03A4EB0B
:10134000010CD269012101FA0CF1114319600399D2
:1013500083B207204A6904990A4302990A600BF094
:10136000FF02E1B2FDF75CFB01981FFA8AF3C1B2FC
:101370000BF0FF020720FDF753FB0099641C504659
:101380008C42A2D30BF1010BAB4584D34FF0000B81
:10139000B8F1000F84BFA81E039078D90BFB05F0AD
:1013A00007EB40000024B0F95000012D6BD04FEA4C
:1013B000EB710BEBD16121F01F02ABEB02020123B9
:1013C00003FA02F2491106EB8101CDE901121C3149
:1013D00000910BFB054107EB4101B1F952A0BAF1B5
:1013E000000FC8BF00284ADDBAEB000148BFA0EBE0
:1013F0000A018245CCBF524602464FF44843594346
:1014000091FBF2F101F2FF114A0A002C1CBF039973
:101410008C42374909680CBF91F8B51091F8B410A7
:1014200019B93349096891F8B4108A4227DD019946
:101430004FF0010CCA6902990A4300990A60E1174A
:1014400004EBD1614A1106EB820303F1140221F08F
:101450001F015B69611A0CFA01F11943116083B233
:10146000E2B20BF0FF010720FDF7DAFA601CC2B20E
:101470001FFA8AF30BF0FF010720FDF7D1FA641C75
:1014800050464C45A5D30BF1010BC34586D307B09D
:101490000120BDE8F08F2DE9F04FD2F80090804692
:1014A00089B0D9F81000164620F00F00C9F81000D6
:1014B00047F6FF7003906FEA000002904FF0FF00C4
:1014C000049005904FF000001061F060B0605FEA9A
:1014D000010A09F1500B054670606AD005FB08F05F
:1014E0004FF0000E3BF9101073460A46174601E014
:1014F00050830010CDE9005E0120B8F1010F19D929
:1015000005FB080C3BF91C408C42C4BF21468646B3
:10151000BC42BCBF27460190B4EB020C48BFA2EB13
:10152000040C0FFA8CF29A42C8BF13462246401CA4
:101530004045E5D30298814202DDCDE9045E029187
:101540000398874203DA0198039707950690C81B12
:1015500048BF781A02B27F480068B0F91CC09445B1
:1015600003DBB0F91E00834220DDEA1705EBD262EF
:10157000531106EB830C22F01F020CF10C03AA1A84
:101580000120DCF80CC090404CEA000018608BB2DF
:101590000EF0FF02E9B20520FDF742FA0198BBB256
:1015A000C2B20098C1B20520FDF73AFA6D1C55454C
:1015B00094D30025B8F1000F57D93BF9151000203E
:1015C0008646034600900A46012017460195BAF167
:1015D000010F19D900FB085C3BF91C408C42C4BFC9
:1015E00021468646BC42BCBF27460090B4EB020CA5
:1015F00048BFA2EB040C0FFA8CF29A42C8BF134604
:101600002246401C5045E5D3C81B48BF781A02B299
:1016100050480068B0F920C0944503DBB0F92200BF
:1016200083421FDDEA1705EBD262531106EB8303F9
:1016300022F01F0203F1040CAA1A01205B689040FB
:1016400018438BB2CCF80000EAB20EF0FF0105207F
:10165000FDF7E6F90198BBB2C2B20098C1B205200D
:10166000FDF7DEF96D1C4545A7D3F068002804BFDF
:101670003069002805D0D9F8100040F00800C9F8FA
:1016800010007068002804BFB068002805D0D9F8A1
:10169000100040F00400C9F810007168F06801FA09
:1016A0000AF10843C9F82800B168306901FA0AF163
:1016B0000843C9F82C007168BAF1200F39BFCAF18C
:1016C0002002D140AAF1200291400843C9F82C0021
:1016D0000398A9F824000298A9F82600B6F9D810B2
:1016E0000298401A44BF0298081A1A4C2168B1F9AE
:1016F000181088420EDDD9F8100040F00200C9F839
:101700001000029883B20598C2B20498C1B20520B5
:10171000FDF786F9B6F9D8100398081A44BF039864
:10172000401A2168B1F91A1088420EDDD9F810006C
:1017300040F00100C9F81000039883B20698C2B2C5
:101740000798C1B20520FDF76BF909B00120BDE88B
:10175000F08F00005083001070474FF0FF3070474B
:101760007A484068704779494860704710B584B03E
:1017700007280BD14FEA111C012404FA0CFC734C0E
:1017800064681CEA040F04BF04B010BD9B0100F0A4
:101790000F0043EA800040F001008DF800008DF852
:1017A00001108DF80220100A8DF80300100C8DF83E
:1017B0000400100E8DF8050000208DF806008DF84D
:1017C00007000290039068460DF057F904B010BD71
:1017D0002DE9F04F0E464FF0000185B05FEA020898
:1017E0000091019102914FF001024FF006070D4662
:1017F0000C46039104BF05B0BDE8F08FEB467B01BA
:1018000000F0070943EA890040F0030A16F81400C3
:101810000BF80200501C36F81420C0B2120A0BF864
:101820000020401CC2B2481CC1B2B9420ED1681C93
:1018300085B28DF800A0FF2D94BF2846FF208DF8BB
:101840000D0068460DF019F900210122601C84B2D8
:101850004445DBD3002904BF05B0BDE8F08F480143
:1018600040EA890040F003008DF80000681C80B257
:10187000FF2888BFFF208DF80D0068460DF0FDF8A9
:1018800005B0BDE8F08F10B584B007280DD191F8F0
:1018900000C001244FEA1C1C04FA0CFC2B4C6468A9
:1018A0001CEA040F04BF04B010BD9B0100F00F0040
:1018B00043EA800040F001008DF800000F2A88BF45
:1018C0000F2200206B46002A09D911F800C01C180D
:1018D000401C84F801C09042F7D30F2805D20021A4
:1018E0001A18401C51700F28FAD318460DF0C5F88D
:1018F00004B010BD70B5154E40EA012502283488A9
:10190000224618BF052803D1002918BF022900D19B
:101910002C46A24209D051B17088002344EA00420B
:1019200090210720FFF722FF3480758070BDF3F708
:10193000B8F84FF47A71B0FBF1F044EA00420023AA
:1019400090210720FFF712FFEEE70000448300100C
:10195000FE4908707047FD480078704710B504468E
:10196000FCF7BFFE0146D02220460DF08BF8F74869
:10197000446010BD58B1F64A0168914207D14068F1
:1019800020F00F00B0F5807F04BF012070470020D9
:101990007047EE4948707047EC484078704710B582
:1019A000EC48EA4C86B000686178B0F84000042941
:1019B000C0F3032008D00421F6F743F801281CBF28
:1019C000002060700FD043E000210846F1F709FACB
:1019D000EFF7FEFA88B1E048D0F8401341F48031C7
:1019E000C0F8401309E00420607005210020EFF7E3
:1019F000ACFE00210846F0F77AF91F20F6F770FEDA
:101A00000DF0D1F80DF0D4F80020F4F7E7F9EFF776
:101A1000DFFA10F0010F04BF0120EFF78FFDF1F79F
:101A200000FBFAF7A9FE01280CD06846F1F708FE82
:101A300028B16846FBF7E2FDF1F759FEF1E7F5F74B
:101A4000A3FEEEE7F0F7E0FF0DF0B2F80DF0B5F809
:101A5000F1F796FA06B010BD2DE9F04FADF68C5DAA
:101A6000BA4E0020CDF8740D7088002804BF0DF622
:101A70008C5DBDE8F08FB748717800680229006C72
:101A8000C0F303253DD0B26840F20F3412F4007F5A
:101A90001EBFC0F303310F290D4612F0800F1EBF89
:101AA000C0F303110F290D4612F4004F0DD0C0F3FF
:101AB00003600F2818BF0546F5F727FFCDF8740D12
:101AC00000281CBF0020F5F705FFB06810F0040FD8
:101AD00008BF40F20B3410F0020F08BF24F00204DC
:101AE00010F0010F08BF24F0010421462846F5F745
:101AF000A8FF012814BF00200220707040F0D88396
:101B00000DE000210846F1F76CF9EFF761FA30B10A
:101B10009148D0F8401341F48031C0F84013F1F7F8
:101B20006CFACDF8780D307A10F0100F18BFF2F77C
:101B300015F8307A10F0080F04BF1F20F6F7D0FD1B
:101B4000864804888648B0F800908648B9F1000FAE
:101B500090F8008084480078CDF8440D18BF002C20
:101B60001AD00DF020F80DF023F8B06810F4803F83
:101B700004BF0020F4F732F9B06810F4003F04BF4E
:101B80000020F4F764F9307A10F0100F0BD0012028
:101B9000F4F76BF901200AE0002818BFB8F1000F34
:101BA000DFD100F085BB0020F4F75FF90020F4F7E7
:101BB0005CF9B06810F4803F18BFF4F7B8F8B0686B
:101BC00010F4003F18BFF4F731F9EFF701FA10F005
:101BD000010F04BF0120EFF7B1FCF1F722FA1E203C
:101BE000FBF78CF800210846FBF716F88346012125
:101BF0000020FBF711F8B568824615F4002F04D0D9
:101C00004FF4BE6102A80CF042FF15F4800F0AD019
